:100000000C9452300C9483300C9483300C948330D5
:100010000C9483300C94C98A0C9483300C948330F4
:100020000C945A8E0C9483300C9483300D94695246
:100030000C9483300D94A4230C9483300C9483305F
:100040000C9483300C94CBAD0C9483300C9483309F
:100050000C9483300C9483300D94D91A0D940C8732
:100060000C9483300C9439FA0C9483300C948330C4
:100070000C9483300C9483300C9483300C94833034
:100080000C9483300C9483300C9483300C94833024
:100090000C94F5F90C9483300C9483300C948330D9
:1000A0000C9483300C9483300C9483300C94833004
:1000B0000C9483300C9483300C9483300C948330F4
:1000C0000C9483300C9483300C9483300C94809C7B
:1000D0000C9483300C9483300C9483300C948330D4
:1000E0000C948330C8D0DED0F1D0FED008D120D11E
:1000F00041D147D155D16BD187D191D1A2D1B3D1C3
:100100003EDA47DA0ADAF3D9D5D99CDB69DAEBDAD9
:1001100072DB930187015D0179014701BF01750120
:100120007D01310165015B018D012701A901B50147
:100130007B01D3018901370155018B01BD01B30159
:100140009D0135014F018301C301CD016F013F01C5
:10015000B70143013501A3019901D90139016101B9
:1001600049013D0157016D015901A701AB01290169
:10017000CF017F016B0185016D01330163017301C3
:10018000084AD73B3BCE016E84BCBFFDC12F3D6CFE
:1001900074319ABD56833DDA3D00C77F11BED9E464
:1001A000BB4C3E916BAAAABE000000803F05A84C44
:1001B000CDB2D44EB93836A9020C50B99186880810
:1001C0003CA6AAAA2ABE000000803F07634236B7B9
:1001D0009BD8A71A39685618AEBAAB558C1D3CB7D8
:1001E000CC5763BD6DEDFD753EF6177231BF000053
:1001F00000803F08000000BE922449123EABAAAA2C
:100200002ABECDCCCC4C3E00000080BEABAAAAAA30
:100210003E00000000BF000000803F000000000022
:10022000084178D3BB4387D1133D190E3CC3BD426F
:1002300082AD2B3E68EC8276BED98FE1A93E4C8020
:10024000EFFFBE01C4FF7F3F0000000000000D94DF
:10025000084F0D94D8840D94F14F0D9456870D944A
:10026000BB0A0D94802B0D940F850D9478820D940C
:10027000C14F0D9496840D940F060D94AA840D948D
:100280005D820D941E000D9465820D944B9C0D941F
:10029000582B0D94A0840D946B090D945B220D9442
:1002A00045820D94DF220D94E1880D943E820D94D9
:1002B000B4840D94BE840D94A52B0D942A2B0D941B
:1002C000CA000D949B840D9419850D948E2B0D946A
:1002D000ED220D9466220D94FB840D942D850D94D2
:1002E00057820D94AF890D9423850D94642B0D9442
:1002F000FE880D943C2B0D94304F0D94722B0D9471
:10030000EC840D94D7870D9449820D9405850D9446
:10031000242B0D948A4F0D9441820D94044F0D941B
:100320008F890D9461220D94162B0D94E2050D9486
:100330003C0C0D946F820D9445880D943A820D9477
:10034000AD090D9472890D946B820D94FA0C0D9485
:10035000C6840D940E4F0D94CE840D949E890D94F9
:100360000A880D9456090D9434820D94174F0D94FC
:1003700061820D9455890D94C3880D9430820D943B
:100380005E2B0D941B890D944F820D94A9870D94BB
:10039000E0050D9438890D9457220D9453820D94E5
:1003A000E2840D943E050D944D4F0D94C0980D942C
:1003B0000B280D9473824E414E494E495459494E73
:1003C00046CDCCCC3D0AD7233C17B7D13877CC2BC0
:1003D000329595E6241FB14F0A000020410000C865
:1003E0004200401C4620BCBE4CCA1B0E5AAEC59DE6
:1003F000746364696E6F70737578585B0000407A3F
:1004000010F35A00A0724E18090010A5D4E800009D
:10041000E87648170000E40B54020000CA9A3B003B
:100420000000E1F505000080969800000040420FB2
:10043000000000A08601000000102700000000E876
:1004400003000000006400000000000A000000003B
:10045000000100000000002C76D888DC674F0823DC
:10046000DFC1DFAE59E1B1B796E5E3E453C63AE642
:1004700051997696E8E6C28426EB898C9B62ED4022
:100480007C6FFCEFBC9C9F40F2BAA56FA5F4900571
:100490005A2AF75C936B6CF9676DC11BFCE0E40DA5
:1004A00047FEF520E6B500D0ED902E030094357799
:1004B000050080841E080000204E0A000000C80CC1
:1004C000333333330F986E12831141EF8D2114892A
:1004D0003BE65516CFFEE6DB18D1844B381BF77C84
:1004E0001D901DA4BBE424203284725E228100C9C9
:1004F000F124ECA1E53D2725642062797465732021
:100500007772697474656E20746F20454550524F40
:100510004D206174206164647265737320307825A6
:10052000303478004433202D20526561642F577297
:1005300069746520454550524F4D0A0020436F7540
:100540006E7420583A20005344207072696E7469AA
:100550006E67206279746520004E6F7420696E208A
:100560006661726D206D6F64652E004163746976FB
:10057000652045787472756465723A2000496E761C
:10058000616C696420657874727564657200746D5D
:1005900063323133305F73675F7468725B25635D0C
:1005A0003D25640A005A204F666673657400556ED7
:1005B0006B6E6F776E20636F6D6D616E643A202293
:1005C000007A5F6D61783A20007A5F6D696E3A203B
:1005D00000795F6D61783A2000795F6D696E3A202D
:1005E00000785F6D61783A2000785F6D696E3A201F
:1005F000005265706F7274696E6720656E64737403
:100600006F7020737461747573000053494C454ECC
:1006100054004E4F524D414C002553204D4F444500
:100620003A2050657263656E7420646F6E653A207F
:1006300025643B207072696E742074696D65207248
:10064000656D61696E696E6720696E206D696E7394
:100650003A2025640A00456E642066696C65206C4A
:1006600069737400426567696E2066696C65206C09
:100670006973740025643A2025640A000A50494EC3
:1006800044412074656D70657261747572653A20BD
:10069000252E3166205A20736869667420286D6D96
:1006A000293A20252E3366000A537465703A2025B6
:1006B000642F360A000A537465703A2025642F3679
:1006C0002028736B6970706564290A50494E444153
:1006D0002074656D70657261747572653A20256469
:1006E000205A20736869667420286D6D293A300A93
:1006F000000A5A45524F3A20252E33660A00737479
:100700006172742074656D70657261747572653A9A
:1007100020252E31660A0025642020252E32660011
:10072000255320583A20252E356620593A20252E6B
:100730003566205A3A20252E35660A004E6F742001
:10074000696E206661726D206D6F64652E00256490
:100750000045303A25642052504D0A50524E303AEE
:1007600025642052504D0A002564004175746F00C5
:1007700020452F443D00416476616E6365204B3D0A
:10078000004D3232302053256900255346696C6193
:100790006D656E742073657474696E67733A204476
:1007A000697361626C65640A00255346696C616D0A
:1007B000656E742073657474696E67733A0A2553A5
:1007C0002020204D3230302044252E32660A00256C
:1007D00053526574726163743A20533D4C656E6781
:1007E000746820286D6D2920463A53706565642031
:1007F000286D6D2F6D29205A3A205A4C6966742055
:10080000286D6D290A25532020204D323037205382
:10081000252E32662046252E3266205A252E326637
:100820000A25535265636F7665723A20533D4578C9
:10083000747261206C656E67746820286D6D292064
:10084000463A537065656420286D6D2F6D290A2521
:10085000532020204D3230382053252E326620463A
:10086000252E32660A25534175746F2D52657472B8
:100870006163743A20533D3020746F206469736162
:10088000626C652C203120746F20696E7465727003
:1008900072657420657874727564652D6F6E6C79FD
:1008A000206D6F7665732061732072657472616369
:1008B0007473206F72207265636F766572696573F9
:1008C0000A25532020204D323039205325640A0058
:1008D00025535049442068656174626564207365DE
:1008E0007474696E67733A0A25532020204D3330A3
:1008F000342050252E32662049252E32662044258C
:100900002E32660A00255350494420736574746979
:100910006E67733A0A25532020204D333031205022
:10092000252E32662049252E32662044252E326639
:100930000A00255353746570732070657220756EBC
:1009400069743A0A255320204D39322058252E3219
:10095000662059252E3266205A252E3266204525DE
:100960002E32660A25534D6178696D756D20666576
:1009700065647261746573202D206E6F726D616C99
:1009800020286D6D2F73293A0A255320204D3230CF
:10099000332058252E32662059252E3266205A25BE
:1009A0002E32662045252E32660A25534D61786920
:1009B0006D756D20666565647261746573202D20A8
:1009C000737465616C746820286D6D2F73293A0A01
:1009D000255320204D3230332058252E32662059A1
:1009E000252E3266205A252E32662045252E326667
:1009F0000A25534D6178696D756D20616363656C7F
:100A000065726174696F6E202D206E6F726D616CFE
:100A100020286D6D2F7332293A0A255320204D323C
:100A200030312058256C752059256C75205A256C5D
:100A3000752045256C750A25534D6178696D756D76
:100A400020616363656C65726174696F6E202D202F
:100A5000737465616C746820286D6D2F7332293A48
:100A60000A255320204D3230312058256C752059ED
:100A7000256C75205A256C752045256C750A255303
:100A8000416363656C65726174696F6E3A20533DB2
:100A9000616363656C65726174696F6E2C20543D8F
:100AA0007265747261637420616363656C65726101
:100AB00074696F6E0A255320204D3230342053253F
:100AC0002E32662054252E32660A25534164766103
:100AD0006E636564207661726961626C65733A2049
:100AE000533D4D696E2066656564726174652028AA
:100AF0006D6D2F73292C20543D4D696E20747261E9
:100B000076656C20666565647261746520286D6D1C
:100B10002F73292C20423D6D696E696D756D2073B0
:100B200065676D656E742074696D6520286D732925
:100B30002C20583D6D6178696D756D205859206A7B
:100B400065726B20286D6D2F73292C20205A3D6D06
:100B50006178696D756D205A206A65726B20286D09
:100B60006D2F73292C2020453D6D6178696D756D61
:100B70002045206A65726B20286D6D2F73290A2528
:100B80005320204D3230352053252E3266205425F7
:100B90002E32662042252E32662058252E326620BF
:100BA00059252E3266205A252E32662045252E32B2
:100BB000660A2553486F6D65206F666673657420FD
:100BC000286D6D293A0A255320204D3230362058A1
:100BD000252E32662059252E3266205A252E326661
:100BE0000A004625642025640A004D4D55203C3DF1
:100BF0002027462564202564270A005049442041C7
:100C000075746F74756E652066696E697368656466
:100C1000212050757420746865206C617374204BBA
:100C2000702C204B6920616E64204B6420636F6ED2
:100C30007374616E74732066726F6D2061626F767B
:100C40006520696E746F20436F6E666967757261A7
:100C500074696F6E2E6800504944204175746F743A
:100C6000756E65206661696C6564212074696D65C7
:100C70006F75740020403A00543A00423A005049DF
:100C800044204175746F74756E65206661696C658A
:100C900064212054656D706572617475726520748D
:100CA0006F6F206869676800204B643A2000204B12
:100CB000693A2000204B703A200020436C61737326
:100CC00069632050494420002054753A2000204B8D
:100CD000753A2000206D61783A2000206D696E3AE7
:100CE000200020643A200020626961733A200020CD
:100CF000453A00205A3A0020593A0020453A00204F
:100D00005A3A0020593A00583A00005A30005A31F5
:100D100000593000593100583000583100456E6498
:100D20002073746F70732064696167002E004465DE
:100D30006C6574696F6E206661696C65642C204611
:100D4000696C653A200046696C652064656C657461
:100D500065643A004E6F74205344207072696E745B
:100D6000696E67005072696E742073617665640005
:100D70005344207072696E742070617573656400ED
:100D80000A002F000A002F2F20616374696F6E3AEA
:100D900063616E63656C0043524153485F43414E4B
:100DA00043454C0043524153485F5245434F5645DB
:100DB000520043524153485F5245434F56455200FB
:100DC00022283229005400496E76616C69642054EF
:100DD00020636F64652E00556E6B6E6F776E204DCD
:100DE00020636F64653A202573200A006E6F2076B9
:100DF000616C696420636F6D6D616E64002C20000E
:100E00002C20002C20006E2F61002C20002C2000B4
:100E10002C20006E2F61002F00503A00576169743A
:100E200020666F722050494E44412074617267659C
:100E3000742074656D70657261747572653A004CEA
:100E4000414E472053454C20464F524345440022D3
:100E50002831290030303030303030302D303030D3
:100E6000302D303030302D303030302D303030308B
:100E700030303030303030300020555549443A0061
:100E800031002045585452554445525F434F554E0A
:100E9000543A005072757361206933204D4B330012
:100EA000204D414348494E455F545950453A003121
:100EB0002E3000206261736564206F6E204D617278
:100EC0006C696E204649524D574152455F55524C10
:100ED0003A68747470733A2F2F6769746875622E5C
:100EE000636F6D2F707275736133642F50727573F9
:100EF000612D4669726D776172652050524F544F73
:100F0000434F4C5F56455253494F4E3A0046495263
:100F10004D574152455F4E414D453A507275736190
:100F20002D4669726D7761726520004D3131332035
:100F3000530020423A0020453A00543A0020413AFA
:100F40000020503A002042403A0020403A00202F32
:100F5000003A00205400202F0020423A00202F00A9
:100F60006F6B20543A002569206D696E2C2025692D
:100F70002073656300496E76616C6964204D20635F
:100F80006F64653A202573200A00556E6B6E6F778B
:100F90006E204720636F64653A202573200A004D58
:100FA00065736820626564206C6576656C696E6740
:100FB000206E6F74206163746976652E000A0020CC
:100FC00020000A4D6561737572656420706F696EEB
:100FD00074733A000A5A2073656172636820686509
:100FE000696768743A20002C004E756D20582C59A2
:100FF0003A2000206D6963726F6E730045786365F7
:10100000737369766520626564206C6576656C69CA
:101010006E6720636F7272656374696F6E3A200049
:101020004732382057300050494E44412070726F8B
:1010300062652063616C6962726174696F6E2073AE
:101040007461727400473238205730004D323400DA
:101050005345545F43484F505F005345545F5354CA
:1010600045505F005345545F574156455F00544D0E
:10107000435F0043524153485F00507265737320D1
:101080006B6E6F6220746F2070726568656174208A
:101090006E6F7A7A6C6520616E6420636F6E74691E
:1010A0006E75652E00506C65617365207072657396
:1010B0007320746865206B6E6F6220746F20756E8C
:1010C0006C6F61642066696C616D656E7400526559
:1010D0006D6F7665206F6C642066696C616D656EFE
:1010E0007420616E6420707265737320746865206B
:1010F0006B6E6F6220746F207374617274206C6FFA
:101100006164696E67206E65772066696C616D65E4
:101110006E742E00616E6420707265737320746843
:1011200065206B6E6F6200496E736572742066692C
:101130006C616D656E740046696C2E2073656E730C
:101140006F7220726573706F6E73652069732070A3
:101150006F6F722C2064697361626C652069743FE3
:1011600000436F6C6F72206E6F7420636F727265D4
:1011700063740046696C616D656E74206E6F7420D7
:101180006C6F61646564004368616E6765642063C9
:101190006F72726563746C793F004C6F6164696E45
:1011A0006720636F6C6F72004368616E67652073C0
:1011B0007563636573732100506C65617365206F9F
:1011C00070656E2069646C657220616E6420726562
:1011D0006D6F76652066696C616D656E74206D61FA
:1011E0006E75616C6C792E005761732066696C6155
:1011F0006D656E7420756E6C6F61642073756363CA
:1012000065737366756C3F00506C6561736520751E
:101210007067726164652E004E6577206669726D35
:10122000776172652076657273696F6E2061766191
:10123000696C61626C653A0057616974696E672018
:10124000666F722050494E44412070726F62652073
:10125000636F6F6C696E67004372617368206465C9
:101260007465637465642E20526573756D652070B6
:1012700072696E743F0043726173682064657465BF
:10128000637465642E0045787472756465720043FA
:10129000686F6F73652065787472756465723A0063
:1012A00043686F6F73652066696C616D656E743A33
:1012B000004D32303020496E76616C69642065786B
:1012C00074727564657220006F70656E00545249C7
:1012D000474745524544004E6F206D6F76652E009E
:1012E0005761697420666F7220757365722E2E2E99
:1012F00000426564206C6576656C696E6720666186
:10130000696C65642E2053656E736F722074726908
:1013100067676572656420746F6F20686967682EFF
:101320002057616974696E6720666F7220726573F9
:1013300065742E00426564206C6576656C696E6725
:10134000206661696C65642E2053656E736F722030
:10135000646973636F6E6E6563746564206F722079
:101360006361626C652062726F6B656E2E205761DF
:101370006974696E6720666F722072657365742E7A
:1013800000537461626C6520616D6269656E7420E2
:1013900074656D70657261747572652032312D32BD
:1013A0003643206973206E65656465642061207230
:1013B00069676964207374616E6420697320726563
:1013C0007175697265642E00506C65617365207279
:1013D000756E2058595A2063616C69627261746934
:1013E0006F6E2066697273742E00536C6565702E83
:1013F0002E2E0073746172740A006164635F696EFB
:1014000069740A001B5B324A1B5B313B31484F72E7
:101410006967696E616C2050727573612069331B56
:101420005B323B334850727573612052657365615E
:1014300072636800466163746F7279205245534548
:1014400054004F6374203238203230313800436FFB
:101450006D70696C65643A2000286E6F6E652C2093
:1014600064656661756C7420636F6E6669672900D8
:101470004F637420323820323031382032313A33E1
:10148000343A32340020332E342E322D313336307C
:101490000A002055706C6F616420696E2070726F55
:1014A000677265737300205A3A0020593A00205839
:1014B0003A0043524153485F4445544543544544E0
:1014C00058590043524153485F444554454354459D
:1014D00044590043524153485F44455445435445A1
:1014E0004458004D323900507275736120693320C1
:1014F0004D4B332072656164792E00426C61636BE1
:101500006F7574206F636375727265642E20526507
:10151000636F766572207072696E743F0053656CFC
:1015200066746573742077696C6C206265207275CF
:101530006E20746F2063616C6962726174652061F2
:10154000636375726174652073656E736F726C6529
:101550007373207265686F6D696E672E00546865DD
:101560007265206973207374696C6C2061206E65EC
:10157000656420746F206D616B65205A2063616C17
:101580006962726174696F6E2E20506C656173655B
:1015900020666F6C6C6F7720746865206D616E7566
:1015A000616C2C2063686170746572204669727387
:1015B000742073746570732C2073656374696F6E27
:1015C0002043616C6962726174696F6E20666C6F32
:1015D000772E005072696E74657220686173206E98
:1015E0006F74206265656E2063616C6962726174FC
:1015F0006564207965742E20506C65617365206682
:101600006F6C6C6F7720746865206D616E75616CAE
:101610002C2063686170746572204669727374204F
:1016200073746570732C2073656374696F6E2043E7
:10163000616C6962726174696F6E20666C6F772E7F
:10164000004F6C642073657474696E677320666FF5
:10165000756E642E2044656661756C742050494433
:101660002C20457374657073206574632E20776930
:101670006C6C206265207365742E005761726E6910
:101680006E673A20626F7468207072696E7465725A
:10169000207479706520616E64206D6F7468657266
:1016A000626F6172642074797065206368616E672F
:1016B00065642E005761726E696E673A20707269B8
:1016C0006E7465722074797065206368616E6765F9
:1016D000642E005761726E696E673A206D6F746890
:1016E0006572626F617264207479706520636861ED
:1016F0006E6765642E002020506C616E6E657242CC
:10170000756666657242797465733A200020467288
:101710006565204D656D6F72793A2000204C6173CC
:101720007420557064617465643A2000506F776569
:101730007255700045787465726E616C2053504923
:1017400020666C61736820573235583230434C2024
:101750006E6F7420726573706F6E64696E672E00B1
:101760006572726F722077726974696E6720746F28
:101770002066696C6500656E6473746F70732068B1
:1017800069743A20006F6B0043726173684465743A
:101790006563742044495341424C4544004372619F
:1017A000736844657465637420454E41424C4544FA
:1017B0002100207C20417574686F723A200020530C
:1017C0006F66747761726520526573657400205787
:1017D00061746368646F67205265736574002042AA
:1017E000726F776E206F7574205265736574002078
:1017F00045787465726E616C20526573657400443F
:101800006F6E6520736176696E672066696C652E00
:101810000058595A2063616C6962726174696F6E15
:1018200020616C6C2072696768742E20536B657739
:101830002077696C6C20626520636F7272656374D7
:101840006564206175746F6D61746963616C6C7936
:101850002E0058595A2063616C6962726174696F15
:101860006E20616C6C2072696768742E20582F5945
:1018700020617865732061726520736C6967687494
:101880006C7920736B657765642E20476F6F6420D9
:101890006A6F62210058595A2063616C69627261F3
:1018A00074696F6E206F6B2E20582F5920617865F8
:1018B00073206172652070657270656E646963750E
:1018C0006C61722E20436F6E67726174756C617407
:1018D000696F6E73210058595A2063616C69627296
:1018E0006174696F6E206661696C65642E2052694F
:1018F0006768742066726F6E742063616C696272CF
:101900006174696F6E20706F696E74206E6F7420E1
:10191000726561636861626C652E0058595A206374
:10192000616C6962726174696F6E206661696C6571
:10193000642E2046726F6E742063616C69627261FE
:1019400074696F6E20706F696E7473206E6F74208F
:10195000726561636861626C652E0058595A206334
:10196000616C6962726174696F6E206661696C6531
:10197000642E20506C6561736520636F6E73756CA7
:101980007420746865206D616E75616C2E00585905
:101990005A2063616C6962726174696F6E20636F53
:1019A0006D70726F6D697365642E2052696768741B
:1019B0002066726F6E742063616C69627261746913
:1019C0006F6E20706F696E74206E6F742072656127
:1019D000636861626C652E0058595A2063616C69B6
:1019E00062726174696F6E20636F6D70726F6D6982
:1019F0007365642E2046726F6E742063616C696239
:101A0000726174696F6E20706F696E7473206E6F8F
:101A10007420726561636861626C652E0058595A62
:101A20002063616C6962726174696F6E20666169BE
:101A30006C65642E204265642063616C696272612A
:101A400074696F6E20706F696E7420776173206E99
:101A50006F7420666F756E642E00506C65617365DF
:101A600020706C61636520737465656C20736865B4
:101A70006574206F6E20686561746265642E004332
:101A8000616C6962726174696E67205A004469739F
:101A900074616E6365206265747765656E20746934
:101AA00070206F6620746865206E6F7A7A6C65208E
:101AB000616E642074686520626564207375726667
:101AC00061636520686173206E6F74206265656E66
:101AD00020736574207965742E20506C6561736580
:101AE00020666F6C6C6F7720746865206D616E7511
:101AF000616C2C2063686170746572204669727332
:101B0000742073746570732C2073656374696F6ED1
:101B1000204669727374206C617965722063616C10
:101B20006962726174696F6E2E00206F66203400E6
:101B3000536561726368696E6720626564206361E2
:101B40006C6962726174696F6E20706F696E740087
:101B5000506C6163652061207368656574206F66F1
:101B600020706170657220756E646572207468659E
:101B7000206E6F7A7A6C6520647572696E67207466
:101B800068652063616C6962726174696F6E206F51
:101B900066206669727374203420706F696E747386
:101BA0002E20496620746865206E6F7A7A6C6520F5
:101BB0006361746368657320746865207061706523
:101BC000722C20706F776572206F6666207468656E
:101BD000207072696E74657220696D6D65646961EB
:101BE00074656C792E00506C6561736520636C655B
:101BF000616E20746865206E6F7A7A6C6520666FFE
:101C0000722063616C6962726174696F6E2E204329
:101C10006C69636B207768656E20646F6E652E005B
:101C2000506C656173652072656D6F7665207374A5
:101C300065656C2073686565742066726F6D2068D9
:101C40006561746265642E00497320737465656C08
:101C5000207368656574206F6E20686561746265C5
:101C6000643F004175746F20686F6D650078797A04
:101C700063616C5F6D656173737572655F656E74CA
:101C800065720A0078797A63616C5F73706972615A
:101C90006C382063783D25642063793D2564207A83
:101CA000303D256420647A3D256420726164697545
:101CB000733D25642061643D25640A0078797A6368
:101CC000616C5F7365617263685A206E6F2073691F
:101CD000676E616C0A20783D256C6420793D256C27
:101CE00064207A3D256C640A00204F4E2D534947ED
:101CF0004E414C20617420783D256420793D256457
:101D0000207A3D25642061643D25640A0078797A53
:101D100063616C5F7365617263685A20783D256CFE
:101D20006420793D256C64207A3D256C640A000AA4
:101D300000253032780078797A63616C5F73636173
:101D40006E5F706978656C735F333278333220630D
:101D5000783D25642063793D2564206D696E5F7A46
:101D60003D2564206D61785F7A3D25640A00202559
:101D700032642025640A000A002530327800206D84
:101D8000696E3D2564206D61783D25642064696637
:101D90003D25640A006D61785F633D253264206DE6
:101DA00061785F6C3D25640A006D61785F633D2555
:101DB00064206D61785F723D2564206D61785F6D90
:101DC000617463683D25640A0020783D25642079AC
:101DD0003D2564207A3D25640A0020706174746595
:101DE000726E20666F756E642061742025642025F4
:101DF000640A000000F000F801FC03FE07FE07FE85
:101E000007FE07FC03F801F000000073697A656FB4
:101E10006628746F74616C293D25640A0073697AC1
:101E2000656F6628626C6F636B5F6275666665726C
:101E3000293D25640A0078797A63616C5F6D65617C
:101E400073737572655F6C656176650A00706F69A2
:101E50006E743D256420783D256420793D256420FD
:101E60007A3D25640A0058025802584D584DB00476
:101E7000F055F055B00478797A63616C5F66696EED
:101E8000645F6265645F696E64756374696F6E5FD9
:101E900073656E736F725F706F696E745F787920AF
:101EA000783D256C6420793D256C64207A3D256C55
:101EB000640A00203C20005741524E494E473A20C8
:101EC00046726F6E7420706F696E74206E6F74202E
:101ED000726561636861626C652E205920636F6F63
:101EE0007264696E6174653A000000004041000050
:101EF000C04000005C430000C04000005C430000A4
:101F000046430000404100004643497465726174D5
:101F1000696F6E3A200000007F43008058439AD9D1
:101F20005143FFFFFF43616C6962726174696F6EB8
:101F3000206661696C65642120436865636B207469
:101F40006865206178657320616E642072756E200B
:101F5000616761696E2E004B494C4C45442E200050
:101F60005072696E7465722068616C7465642E20AD
:101F70006B696C6C28292063616C6C656421004D71
:101F800031303420496E76616C69642065787472F2
:101F90007564657220004D31303520496E76616C74
:101FA000696420657874727564657220004D313003
:101FB0003920496E76616C69642065787472756445
:101FC000657220004D32313820496E76616C69644B
:101FD00020657874727564657220004D323231204C
:101FE000496E76616C696420657874727564657297
:101FF00020005265636F766572696E672070726942
:102000006E7420202020004B494C4C3A2025640A55
:102010000055564C4F202D20656E642025640A0023
:102020007374707325640A00776F726C6420636F39
:102030006F7264696E617465733A2028252E336669
:102040002C20252E33662C20252E3366290A00707D
:102050006879736963616C20636F6F7264696E6124
:102060007465733A2028252E33662C20252E33667E
:102070002C20252E3366290A0043757272656E7412
:1020800020706F73205A5F415849533A252E3366AA
:102090000A43757272656E7420706F7320455F41DC
:1020A0005849533A252E33660A00416674657220FA
:1020B00077616974696E6720666F722074656D70F0
:1020C0003A0A43757272656E7420706F7320585FA0
:1020D000415849533A252E33660A43757272656E2C
:1020E0007420706F7320595F415849533A252E333D
:1020F000660A0020573A0020453A00543A005A2018
:102100006C6976652061646A757374206F757420DC
:102110006F662072616E67652E2053657474696EF8
:102120006720746F20302E20436C69636B20746FBE
:1021300020636F6E74696E75652E005A206C697627
:10214000652061646A757374206F7574206F6620F2
:1021500072616E67652E2053657474696E672074B2
:102160006F20300020423A0020453A00543A00499E
:102170004E5434007265636F7665725F6D6163689B
:10218000696E655F73746174655F61667465725FC3
:10219000706F7765725F70616E69632C20696E691C
:1021A0007469616C20007265636F7665725F6D6142
:1021B0006368696E655F73746174655F6166746599
:1021C000725F706F7765725F70616E69632C2069F2
:1021D0006E697469616C20004739322045005052A5
:1021E0005553412075766C6F004734205330004DB5
:1021F00032362053256C75004D3130362053004D5A
:102200003832004731204625640047312045322AC4
:1022100064656661756C745F72657472616374691C
:102220006F6E2046343830004731205A0020463245
:102230003030300020590047312058004D383300ED
:10224000506F736974696F6E207265616420667285
:102250006F6D20656570726F6D3A004D32332025C9
:1022600073002E67636F0046656564726174653A3A
:1022700000473120452D64656661756C745F726539
:102280007472616374696F6E204634383000473170
:102290002045352046313230004D3833004D31393C
:1022A0003020532564004D313039205325640047D8
:1022B000323820582059004731205A3235204638CC
:1022C000303000544D4320445249564552204F5619
:1022D000455254454D50005A25362E326620005A3C
:1022E0002020202D2D2D200025632533642F2564EB
:1022F00025630025632533642525002D2D2D00251C
:102300003368686400253353253373252500205333
:10231000440020202000555342002025753E25759D
:1023200000204625750020463020200025632D2DF5
:102330003A2D2D2020002563253032753A25303284
:10234000752563256300726573756C742076616C06
:1023500075653A2025640A0020693D2532642063B2
:102360006E743D2532642076616C3D2532640A002E
:10237000636C7573746572733A0A0020693D253287
:102380006420737465703D2532640A00736F727443
:1023900065642073616D706C65733A0A0055534132
:1023A0005254322072782046756C6C2121210A002B
:1023B0003A20002020202020202020202020202023
:1023C00020202020202000203A2000202020202033
:1023D000202020202020202020202020202020001D
:1023E00020202020202020202020202020002573B5
:1023F0000050494E44412048656174696E6700543D
:10240000656D702E2063616C2E20202020202020FE
:102410002020200043616C6962726174696F6E20D4
:10242000646F6E650042656420646F6E650042658E
:10243000642048656174696E670048656174696EFF
:102440006720646F6E652E0048656174696E670071
:10245000000E1315110E00000004120912040000F2
:10246000001C1F11111F00000006191803130C0097
:10247000040E1F041C000000040A0A0A0A11110EAF
:10248000001F1511151F0000000103161C08000095
:102490000000110A04110A040C12120C00000000C2
:1024A0002563252D3138532563002563252E3135CD
:1024B000533A2573253364002563252E3132533A70
:1024C00025732500457872656D65207370616E20F7
:1024D0006F6620746865205A2076616C756573217B
:1024E0000000004041000000400000E44200000005
:1024F000400000574300000040000057430000C464
:10250000420000E4420000C442000040410000C418
:102510004200004041000042430000E4420000420B
:10252000430000574300004243205B6F66665D0036
:10253000426564206C6576656C696E6720666169CA
:102540006C65642E2053656E736F72206469646ECF
:102550007420747269676765722E204465627269BF
:1025600073206F6E206E6F7A7A6C653F20576169B9
:1025700074696E6720666F722072657365742E00D1
:10258000206F662039004D6561737572696E672032
:102590007265666572656E636520686569676874F3
:1025A000206F662063616C6962726174696F6E206E
:1025B000706F696E740024F4D43050C38E20C2A2B0
:1025C0004017828B7011127A910D816CD90AA86123
:1025D000E108C7586607615143061E4B5D05C145BA
:1025E000A7041A411104093D98037139310340369B
:1025F000DB0265339102D4305402802E1D02632C1D
:10260000EE01752AC501B028A001102781018F2590
:1026100064012B244B01E0223401AC211F018D20E9
:102620000D01801FFC00841EED00971DDF00B81C0B
:10263000D200E61BC600201BBC00641AB200B2190F
:10264000A8000A19A0006A189900D1179100401734
:102650008B00B516840031167E00B31579003A154B
:102660007300C7146F0058146A00EE1366008813D5
:10267000630025135E00C7125B006C125700151231
:102680005400C111510070114F0021114B00D610A0
:1026900049008D1047004610440002104200C00F50
:1026A0004000800F3E00420F3C00060F3B00CB0E67
:1026B0003800930E37005C0E3500270E3400F30D02
:1026C0003200C10D3100900D3000600D2E00320D32
:1026D0002D00050D2C00D90C2B00AE0C2900850C0B
:1026E00029005C0C2700350C27000E0C2600E80B97
:1026F0002400C40B2400A00B23007D0B23005A0BE5
:102700002100390B2100180B2000F80A1F00D90AFC
:102710001E00BB0A1E009D0A1D00800A1D00630AE0
:102720001C00470A1B002C0A1B00110A1A00F7099B
:102730001A00DD091900C4091900AB091900920932
:1027400017007B091800630917004C0916003609A9
:102750001600200916000A091500F5081500E00802
:102760001400CC081400B8081400A4081400900841
:1027700013007D0812006B08130058081200460869
:10278000120034081100230811001208110001087A
:102790001100F0071000E0071000D0071000C0077C
:1027A0001000B0070F00A107100091070E0083076B
:1027B0000F0074070F0065070E0057070E0049074A
:1027C0000E003B070D002E070E0020070D0013071B
:1027D0000D0006070D00F9060C00ED060D00E006E1
:1027E0000C00D4060C00C8060C00BC060C00B00699
:1027F0000C00A4060B0099060C008D060B00820647
:102800000B0077060B006C060B0061060A005706EA
:102810000B004C060A0042060A0038060A002E0683
:102820000A0024060A001A060A0010060900070614
:102830000A00FD050900F4050900EB050900E205A1
:102840000900D9050900D0050900C7050900BE0522
:102850000900B5050800AD050800A50509009C059F
:102860000800940508008C050800840508007C0514
:102870000800740508006C050700650508005D0583
:102880000700560508004E050700470507004005EC
:10289000080038050700310507002A050700230551
:1028A00007001C050600160507000F0507000805B0
:1028B000060002050700FB040600F5040700EE040D
:1028C0000600E8040600E2040700DB040600D50465
:1028D0000600CF040600C9040600C3040600BD04B8
:1028E0000600B7040600B1040500AC040600A60407
:1028F0000600A00405009B04060095040500900452
:1029000006008A04050085040500800406007A0498
:10291000050075040500700405006B0405006604DD
:102920000500610405005C0405005704050052041D
:1029300005004D04050048040500430405003E045D
:1029400004003A04050035040500300404002C049A
:10295000050027040400230405001E0404001A04D3
:10296000040016040500110404000D040400090409
:1029700005000404040000040400FC030400F80340
:102980000400F4030400F0030400EC030400E80373
:102990000400E4030400E0030400DC030400D803A3
:1029A0000400D4030400D0030400CC030400C803D3
:1029B0000300C503030024F404D9201BC40C5C0EDF
:1029C0009804C4095F0265077101F405F900FB046E
:1029D000B30048048700C10369005803550003038E
:1029E0004500BE023A008402310053022A00290247
:1029F000250004022000E4011C00C8011900AF01F9
:102A00001700980114008401130071011000610186
:102A1000100051010E0043010D0036010B002B0187
:102A20000B0020010B00150109000C010900030136
:102A30000800FB000800F3000800EB000700E400BA
:102A40000600DE000600D8000600D2000600CC001A
:102A50000500C7000500C2000500BD000400B90064
:102A60000400B5000400B1000400AD000400A9009A
:102A70000400A5000300A20003009F0004009B00C7
:102A800003009800030095000200930003009000EB
:102A900003008D0002008B00030088000200860006
:102AA000020084000300810002007F0002007D001C
:102AB00002007B000200790002007700010076002E
:102AC00002007400020072000100710002006F0039
:102AD00002006D0001006C0002006A000100690044
:102AE000020067000100660001006500010064004B
:102AF00002006200010061000100600001005F004F
:102B000002005D0001005C0001005B0001005A0052
:102B10000100590001005800010057000100560053
:102B20000100550001005400010053000000530053
:102B300001005200010051000100500001004F004F
:102B400001004E0000004E0001004D0001004C004D
:102B500001004B0000004B0001004A000100490049
:102B60000100480000004800010047000100460045
:102B7000000046000100450000004500010044003F
:102B80000100430000004300010042000000420039
:102B900001004100000041000100400001003F0031
:102BA00000003F0001003E0000003E0001003D002B
:102BB00000003D0001003C0000003C0000003C0023
:102BC00001003B0000003B0001003A0000003A0019
:102BD0000100390000003900010038000000380011
:102BE0000000380001003700000037000100360007
:102BF00000003600000036000100350000003500FE
:102C000000003500010034000000340000003400F2
:102C100001003300000033000000330001003200E7
:102C200000003200000032000100310000003100DD
:102C300000003100010030000000300000003000D2
:102C400001002F0000002F0000002F0000002F00C7
:102C500001002E0000002E0000002E0001002D00BB
:102C600000002D0000002D0000002D0001002C00B0
:102C700000002C0000002C0000002C0001002B00A4
:102C800000002B0000002B0000002B0001002A0098
:102C900000002A0000002A0000002A00010029008C
:102CA0000000290000002900000029000000290080
:102CB0000100280000002800000028000000280073
:102CC0000000280001002700000027000000270066
:102CD0000000270000002700010026000000260059
:102CE000000026000000260000002600010025004C
:102CF0000000250000002500000025000000250040
:102D00000000250001002400000024000000240031
:102D10000000240000002400010023000000230024
:102D20000000230000002300000023000000230017
:102D30000000230001002200000022000000220009
:102D400000002200000022000000220001002100FB
:102D500000002100000021000000210000002100EF
:102D600000002100000021000100200000002000E0
:102D700000002000000020000000200000002000D3
:102D8000000020000000200001001F0000001F00C4
:102D900000001F0000001F0000001F0000001F00B7
:102DA00000001F0001001E0000001E0000001E00A9
:102DB00000001E0000001B5B313B31485057523A67
:102DC00020202020202025642E2530316456001B31
:102DD0005B303B314842656C742073746174757369
:102DE0001B5B313B3248582025641B5B323B324829
:102DF0005920256400464C4558202D20203234307F
:102E00002F35300050502020202D20203235342FF7
:102E10003130300048495053202D20203232302F9D
:102E20003130300041425320202D20203235352FC3
:102E30003130300050455420202D20203233302FA7
:102E4000383500504C4120202D20203231352F368E
:102E50003000414253202020202D20203235352FB4
:102E6000313030006E6F7A7A6C65202D202032353B
:102E7000302F30006661726D2020202D20203235E9
:102E8000302F363000466C617368416972204950BA
:102E900020416464723A004D4D553220202020209C
:102EA00020204E2F4100756E6B6E6F776E0025648B
:102EB0002E25642E25642D2564002046573A004DAA
:102EC0004D553220636F6E6E6563746564004F63A9
:102ED000742032382032303138004533447636663B
:102EE000756C6C0045494E53795F31306100315F3C
:102EF00037356D6D5F4D4B33002D2D2D2D2D2D2D27
:102F00002D2D2D2D2D00207265706F20556E6B6E4E
:102F10006F776E0020332E342E322D313336300051
:102F20004669726D776172653A0025642E25642EBC
:102F300025642E2564004D373032004D3730310086
:102F40004578747275646572006D6D0000590058A3
:102F500000580059005A002563252E3132533A2576
:102F600073252B30362E336600436F6F6C646F779A
:102F70006E00566F6C74616765730054656D7065A3
:102F8000726174757265730042656C74207374614C
:102F900074757300457874727564657220696E6625
:102FA0006F0058595A2063616C2E20646574616902
:102FB0006C7300446174653A00686F77746F2E70AB
:102FC0007275736133642E636F6D00666F72756D19
:102FD0002E707275736133642E636F6D007072753D
:102FE000736133642E636F6D004175746F6C6F6134
:102FF00064696E672066696C616D656E74206973C3
:10300000206163746976652C206A75737420707210
:1030100065737320746865206B6E6F6220616E64E7
:1030200020696E736572742066696C616D656E747B
:103030002E2E2E00546F74616C207072696E742095
:1030400074696D6500546F74616C2066696C616DA4
:10305000656E74005072696E742074696D65004607
:10306000696C616D656E742075736564005072657E
:103070006865617420746865206E6F7A7A6C65216A
:10308000004552524F523A005269676874004C65CD
:10309000667400592064697374616E63652066729A
:1030A0006F6D206D696E0053657665726520736B78
:1030B000657700536C6967687420736B6577004DA2
:1030C0006561737572656420736B6577005B303B77
:1030D000305D20706F696E74206F66667365740072
:1030E00041646A757374696E67205A00526573652E
:1030F0007400526561722073696465205B756D5D53
:103100000046726F6E7420736964655B756D5D0057
:10311000526967687420736964655B756D5D004C06
:103120006566742073696465205B756D5D00536529
:10313000742074656D70657261747572653A001BF8
:103140005B324A2553203A1B5B313B394825382EE8
:103150003266206D0A2553203A0A25376C646420B4
:103160003A253268686468203A25303268686420FD
:103170006D001B5B324A25533A1B5B313B364825B9
:10318000382E32666D200A2553203A1B5B333B38BC
:10319000482532646820253032646D202530326441
:1031A000730025362E32666D6D004E2F41001B5B7D
:1031B000303B304825533A0A25530A25533A0A250D
:1031C000533A001B5B303B3135484E2F41001B5BAF
:1031D000303B31354825342E326601001B5B303BD5
:1031E000304825533A0A25530A25533A20202535DD
:1031F0002E3266010A25533A202025352E326601EB
:103200000052756E6E696E672057697A617264202C
:1032100077696C6C2064656C657465206375727287
:10322000656E742063616C6962726174696F6E208F
:10323000726573756C747320616E6420737461724F
:10324000742066726F6D2074686520626567696EB0
:103250006E696E672E20436F6E74696E75653F00F0
:1032600050726568656174696E67206E6F7A7A6CFA
:10327000652E20506C6561736520776169742E003E
:10328000596F752063616E20616C7761797320726C
:103290006573756D65207468652057697A6172641D
:1032A0002066726F6D2043616C6962726174696F30
:1032B0006E202D3E2057697A6172642E00506C6535
:1032C00061736520636865636B206F757220686148
:1032D0006E64626F6F6B20616E6420666978207423
:1032E00068652070726F626C656D2E205468656E23
:1032F00020726573756D65207468652057697A6101
:103300007264206279207265626F6F74696E6720E3
:10331000746865207072696E7465722E00416C6C01
:1033200020697320646F6E652E204861707079206B
:103330007072696E74696E672100506C65617365A7
:1033400020636C65616E20686561746265642061EC
:103350006E64207468656E20707265737320746883
:1033600065206B6E6F622E00446F20796F75207739
:10337000616E7420746F20726570656174206C6179
:103380007374207374657020746F20726561646A51
:103390007573742064697374616E6365206265740B
:1033A0007765656E206E6F7A7A6C6520616E642039
:1033B000686561746265643F00492077696C6C20C0
:1033C000737461727420746F207072696E74206CF3
:1033D000696E6520616E6420796F752077696C6C09
:1033E000206772616475616C6C79206C6F776572AF
:1033F00020746865206E6F7A7A6C6520627920721D
:103400006F746174696E6720746865206B6E6F629B
:103410002C20756E74696C20796F752072656163FC
:1034200068206F7074696D616C2068656967687485
:103430002E20436865636B2074686520706963742F
:103440007572657320696E206F75722068616E6495
:10345000626F6F6B20696E206368617074657220A3
:1034600043616C6962726174696F6E2E004E6F7792
:1034700020492077696C6C2063616C6962726174A9
:10348000652064697374616E636520626574776535
:10349000656E20746970206F6620746865206E6F99
:1034A0007A7A6C6520616E64206865617462656417
:1034B00020737572666163652E00497320697420FC
:1034C000504C412066696C616D656E743F004C6FB5
:1034D0006164696E672066696C616D656E74005029
:1034E0006C6561736520696E7365727420504C4120
:1034F0002066696C616D656E7420746F20746865F8
:103500002065787472756465722C207468656E200D
:103510007072657373206B6E6F6220746F206C6FB6
:1035200061642069742E00506C6561736520696E5A
:103530007365727420504C412066696C616D656ED4
:103540007420746F207468652066697273742074C7
:10355000756265206F66204D4D552C207468656E30
:1035600020707265737320746865206B6E6F6220C3
:10357000746F206C6F61642069742E00456A656306
:103580007400556E6C6F61640055736520756E6CC8
:103590006F616420746F2072656D6F766520666957
:1035A0006C616D656E7420312069662069742070CD
:1035B000726F747275646573206F75747369646576
:1035C000206F66207468652072656172204D4D55CC
:1035D00020747562652E2055736520656A65637475
:1035E0002069662069742069732068696464656E67
:1035F00020696E20747562652E0053656C65637476
:10360000206E6F7A7A6C65207072656865617420CF
:1036100074656D7065726174757265207768696331
:1036200068206D61746368657320796F7572206DB1
:103630006174657269616C2E004E6F772049207746
:10364000696C6C2070726568656174206E6F7A7A3F
:103650006C6520666F7220504C412E0049732066C5
:10366000696C616D656E74206C6F616465643F00A8
:1036700049732066696C616D656E742031206C6FD2
:10368000616465643F00492077696C6C2072756ED7
:10369000207A2063616C6962726174696F6E206E5A
:1036A0006F772E00492077696C6C2072756E2078D8
:1036B000797A2063616C6962726174696F6E206EE1
:1036C0006F772E2049742077696C6C2074616B656C
:1036D00020617070726F782E203132206D696E73A8
:1036E0002E0046697273742C20492077696C6C2017
:1036F00072756E207468652073656C66746573748A
:1037000020746F20636865636B206D6F7374206332
:103710006F6D6D6F6E20617373656D626C79207073
:10372000726F626C656D732E0048692C20492061B0
:103730006D20796F7572204F726967696E616C20B8
:103740005072757361206933207072696E7465728E
:103750002E20576F756C6420796F75206C696B65CE
:10376000206D6520746F20677569646520796F75B9
:10377000207468726F75676820746865207365745B
:1037800075702070726F636573733F00452D636FB2
:103790007272656374005A2D636F72726563740090
:1037A000592D636F727265637400582D636F727266
:1037B00065637400536F756E642020202020205BA9
:1037C0006C6F75645D00536F756E6420202020203F
:1037D000205B6D7574655D00536F756E64202020ED
:1037E000205B73696C656E745D00536F756E642049
:1037F00020202020205B6F6E63655D00536F756E27
:10380000642020202020205B6C6F75645D00536F66
:1038100072743A2020202020205B6E6F6E655D0060
:10382000536F72743A20205B616C706861626574DA
:103830005D00536F72743A2020202020205B746951
:103840006D655D005344206361726420205B6E6F80
:10385000726D616C5D0053442063617264205B662D
:103860006C73684169725D0052506920706F7274A8
:1038700020202020205B6F6E5D0052506920706F09
:103880007274202020205B6F66665D0054656D7049
:103890002E2063616C2E2020205B6F6E5D005465CE
:1038A0006D702E2063616C2E20205B6F66665D005C
:1038B0004C696E2E20636F7272656374696F6E005F
:1038C00046616E7320636865636B20205B6F66667C
:1038D0005D0046616E7320636865636B2020205B2A
:1038E0006F6E5D004175746F206465706C65746502
:1038F0005B6F66665D004175746F206465706C6512
:103900007465205B6F6E5D00462E204F51206D6503
:103910006173732E5B6F66665D00462E204F5120EB
:103920006D656173732E205B6F6E5D00462E2061A6
:1039300075746F6C6F6164205B6F66665D00462E08
:10394000206175746F6C6F616420205B6F6E5D0029
:10395000462E206175746F6C6F6164205B4E2F4141
:103960005D0046696C2E2073656E736F72205B4E2E
:103970002F415D0044697361626C652073746570EA
:1039800070657273004D6F766520617869730054BD
:10399000656D70657261747572650054656D702E29
:1039A0002063616C6962726174696F6E0052657345
:1039B00065742058595A2063616C6962722E0053F5
:1039C000686F772070696E6461207374617465003C
:1039D0005049442063616C6962726174696F6E0062
:1039E000426564206C6576656C20636F72726563F6
:1039F00074004D65736820426564204C6576656C83
:103A0000696E670043616C696272617465205A0077
:103A100043616C6962726174652058595A0053653C
:103A20006C667465737420202020202020202000E4
:103A30004669727374206C617965722063616C2EC3
:103A40000057697A617264004C6F61642066696C2A
:103A5000616D656E742035004C6F61642066696C21
:103A6000616D656E742034004C6F61642066696C12
:103A7000616D656E742033004C6F61642066696C03
:103A8000616D656E742032004C6F61642066696CF4
:103A9000616D656E742031004C6F616420616C6CE7
:103AA00000456A6563742066696C616D656E74209B
:103AB0003500456A6563742066696C616D656E7476
:103AC000203400456A6563742066696C616D656EBB
:103AD00074203300456A6563742066696C616D65A6
:103AE0006E74203200456A6563742066696C616D8E
:103AF000656E74203100556E6C6F61642066696C70
:103B0000616D656E74203500556E6C6F6164206662
:103B1000696C616D656E74203400556E6C6F616404
:103B20002066696C616D656E74203300556E6C6F34
:103B300061642066696C616D656E74203200556E3B
:103B40006C6F61642066696C616D656E7420310014
:103B5000556E6C6F616420616C6C00457874727591
:103B60006465722034004578747275646572203320
:103B700000457874727564657220320045787472FD
:103B800075646572203100506C65617365207075D5
:103B90006C6C206F75742066696C616D656E742045
:103BA000696D6D6564696174656C7900556E6C6FE3
:103BB0006164696E672066696C616D656E7400573B
:103BC000697A61726420656E642073746174653A09
:103BD0002025640A0057697A6172642073746174E5
:103BE000653A2025640044697361626C65206661F2
:103BF000726D206D6F6465004661726D206E756D2B
:103C0000626572004D3834004D343400473238203C
:103C100057004739390044697361626C65206661F9
:103C2000726D206D6F64653F0043686F6F73652030
:103C3000636F6C6F723A006F6B0A00737461727419
:103C40000A004D4D5532206669726D7761726520AC
:103C500076657273696F6E20696E76616C69642E29
:103C60002052657175697265642076657273696F3B
:103C70006E3A206275696C64206E756D62657220A3
:103C80002564206F72206869676865722E006E6F08
:103C9000745F6F6B0A004D363030004D3630302087
:103CA0004155544F004653454E534F525F52454382
:103CB0004F56455200256868750050300A00523052
:103CC0000A004525640A0055300A0043300A004CBA
:103CD00025640A005425640A004D4D55202D2045C9
:103CE0004E41424C454400256868750050300A003A
:103CF00050300A004D4D552076657273696F6E2005
:103D000076616C69640025750053320A00257500E0
:103D10004D4D55206E6F7420726573706F6E6469BF
:103D20006E67202D2044495341424C454400533195
:103D30000A004D4D5520737461727473207265735F
:103D4000706F6E64696E670A004D4D55206E6F741A
:103D500020726573706F6E64696E670A0000008080
:103D60003F555585410000803F0000C841000000DC
:103D700040555505420000C03F0000484200002069
:103D80004055558542000070C1ABAAA642000060B4
:103D9000C10000A0410000C0C00000204100002080
:103DA00041ABAA3A41000020C15555D5400000481A
:103DB000C2555505424D373031204530004D373022
:103DC00031204531004D373031204532004D3730FC
:103DD00031204533004D373031204534004D3730E8
:103DE00031204534004D373031204533004D3730D8
:103DF00031204532004D373031204531004D3730CC
:103E0000312045300046696C616D656E74206E72BC
:103E1000206F7574206F662072616E676521007770
:103E20003235783230636C5F63666D0A0077323505
:103E3000783230636C5F656E7465720A005041546D
:103E4000393132355F5245535F593D256868750AEF
:103E500000504154393132355F5245535F583D254A
:103E60006868750A00062833D036C23E013F154106
:103E700032423B43F2443B45F24622473B48F2493B
:103E80003B4AF05898590C5A085B0C5C0861106763
:103E90009B6E2271077208FF095A0D000EF019047B
:103EA0005E0820642B6D322FFF506C6561736520B6
:103EB000757064617465206669726D7761726520E2
:103EC000696E20796F7572204D4D55322E205761E5
:103ED0006974696E6720666F722072657365742EEF
:103EE000004D4D55204F4B2E20526573756D696EF8
:103EF000672E2E2E004D4D55204F4B2E20526573B0
:103F0000756D696E6720706F736974696F6E2E2EA0
:103F10002E004D4D55204F4B2E20526573756D6907
:103F20006E672074656D70657261747572652E2E92
:103F30002E004D4D55206E65656473207573657256
:103F400020617474656E74696F6E2E2046697820E6
:103F500074686520697373756520616E6420746888
:103F6000656E20707265737320627574746F6E2055
:103F70006F6E204D4D5520756E69742E00506C6526
:103F80006173652072656D6F76652066696C616D21
:103F9000656E7420616E64207468656E2070726551
:103FA000737320746865206B6E6F622E00456A65BE
:103FB0006374696E672066696C616D656E7400621A
:103FC0007573793A2070617573656420666F72202D
:103FD000696E70757400627573793A2070617573DB
:103FE000656420666F7220757365720062757379FF
:103FF0003A2070726F63657373696E6700204600C4
:104000004731205A0020460047312045004D3833C3
:10401000006F6B0A0000002110422063308440A52D
:1040200050C660E770088129914AA16BB18CC1AD7F
:10403000D1CEE1EFF13112100273325222B5529417
:1040400042F772D662399318837BB35AA3BDD39CCF
:10405000C3FFF3DEE36224433420040114E664C7A3
:1040600074A44485546AA54BB528850995EEE5CF1F
:10407000F5ACC58DD55336722611163006D776F6B7
:10408000669556B4465BB77AA719973887DFF7FE6F
:10409000E79DD7BCC7C448E5588668A77840086143
:1040A0001802282338CCC9EDD98EE9AFF9488969BF
:1040B000990AA92BB9F55AD44AB77A966A711A5057
:1040C0000A333A122AFDDBDCCBBFFB9EEB799B580F
:1040D0008B3BBB1AABA66C877CE44CC55C222C03E3
:1040E0003C600C411CAEED8FFDECCDCDDD2AAD0B5F
:1040F000BD688D499D977EB66ED55EF44E133E32F7
:104100002E511E700E9FFFBEEFDDDFFCCF1BBF3AAE
:10411000AF599F788F8891A981CAB1EBA10CD12D9D
:10412000C14EF16FE18010A100C230E320045025A0
:104130004046706760B9839893FBA3DAB33DC31C14
:10414000D37FE35EF3B1029012F322D232354214F0
:104150005277625672EAB5CBA5A89589856EF54F60
:10416000E52CD50DC5E234C324A014810466744740
:104170006424540544DBA7FAB79987B8975FE77EB4
:10418000F71DC73CD7D326F2369106B01657667690
:1041900076154634564CD96DC90EF92FE9C899E900
:1041A000898AB9ABA94458654806782768C018E1E0
:1041B000088238A3287DCB5CDB3FEB1EFBF98BD854
:1041C0009BBBAB9ABB754A545A376A167AF10AD030
:1041D0001AB32A923A2EFD0FED6CDD4DCDAABD8BA0
:1041E000ADE89DC98D267C076C645C454CA23C8380
:1041F0002CE01CC10C1FEF3EFF5DCF7CDF9BAFBAF4
:10420000BFD98FF89F176E367E554E745E932EB2CF
:104210003ED10EF01E7C3C3E5E2B3D3F2F5B5D3B56
:104220002C2A225C0043757272656E7400557365AA
:104230006420647572696E67207072696E740050D4
:1042400049442063616C2E2066696E6973686564F9
:10425000005049442063616C2E2020202020202023
:104260002020202000506C6561736520776169749F
:10427000004D313137204669727374206C61796565
:10428000722063616C2E005072696E7420706175CB
:1042900073656400496E76616C69642050494420FE
:1042A00063616C2E20726573756C74732E204E6F73
:1042B000742073746F72656420746F20454550528A
:1042C0004F4D2E004D353030004731205A313520CA
:1042D00046313530300047393100473120583530CC
:1042E00020593139302045302046373030300047B2
:1042F0003930004D373032004D3730322043004DD9
:104300003730322055004D373032004D37303220B3
:1043100043004731205A313520463135303000478F
:104320003931004731205835302059313930204556
:1043300030204637303030004D38330047393000B8
:104340004D3834004D313034205330004D38340076
:104350004D37303220430047312058313020593119
:104360003830204634303030004731205A31302048
:1043700046313330302E303030004D313430205320
:1043800030004D31303420533000473120452D303E
:104390002E30373530302046323130302E3030300C
:1043A0003030004D313037004731205835302059FA
:1043B00035352045332E36323737330047312058D4
:1043C000323030205935352045302E3439333836A7
:1043D0000047312058323030205937352045332EB0
:1043E000363237373300473120583530205937358A
:1043F0002045302E34393338360047312058353097
:10440000205939352045332E36323737330047317E
:104410002058323030205939352045302E34393348
:10442000383600473120583230302059313135206C
:1044300045332E3632373733004731205835302058
:10444000593131352045302E343933383600473133
:104450002058353020593133352045332E36323708
:10446000373300473120583230302059313335202E
:1044700045302E363631373400473120583230300F
:1044800020593135352045322E3632373733004703
:1044900031205831303020593135352045320047F0
:1044A000312058373520593135352045322E3500E9
:1044B0004731204631303830004731205A302E31D4
:1044C00035302046373230302E3030300047312002
:1044D0005835302059313535004731204634303099
:1044E00030004D32303420533130303000473120ED
:1044F0005A352046373230302E30303000473120A8
:10450000452D312E35303030302046323130302E8E
:104510003030303030004D383300473930004732CA
:1045200031004739322045302E3000473120583194
:1045300030302E30204531322E352046313030306B
:104540002E30004731205836302E302045392E305D
:104550002046313030302E300047312058352E3053
:104560002045342E302046313030302E3000473157
:10457000205A302E32302046313030302E30004735
:1045800031205835352E30204532352046313430F3
:10459000302E3000473120592D322E302046313018
:1045A00030302E3000473120583234302E30204504
:1045B00032352E30202046323230302E300047390E
:1045C000322045302E30004731205A302E332046DD
:1045D000313030302E30004731205835352E3020E4
:1045E00045382E302046323030302E3000473120D2
:1045F00058352E30204533322E3020463138303079
:104600002E30004731205835352E30204533322E9C
:10461000302046313037332E30004731205A302E8B
:10462000342046313030302E3000473120592D3380
:104630002E302046313030302E30004D3833004798
:1046400039322045302E3000473238004D31303974
:104650002053323135004D31393020533630004D42
:1046600031343020533630004D3130342053323124
:1046700035004D3130370053657474696E677320AF
:1046800053746F7265640053746F72656420736550
:104690007474696E67732072657472696576656497
:1046A0000048617264636F64656420446566617587
:1046B0006C742053657474696E6773204C6F616409
:1046C000656400563200000000C8420000C8420085
:1046D00000C84300008C43000048430000484300EA
:1046E0000040410000F042E8030000E8030000C879
:1046F0000000008813000000409C4400409C4400DF
:1047000000000000000000204E00000000204100DA
:10471000002041CDCCCC3E00002040000000000035
:1047200000000000000000CDCCCC3E3D0A8141FFDE
:1047300008433EB099AB438F42FC42E65A343F4CAB
:1047400062B045000000000040400000344200001C
:1047500000000000000000000041000000E03F00F9
:1047600000C8420000C842000040410000F042C0C2
:10477000030000C0030000C80000008813000045CB
:104780004550524F4D204572726F7200436F6E74E8
:10479000696E7565207769746820616E6F746865ED
:1047A0007220626F7764656E3F0025002020202014
:1047B0002020002020202020200045524153494E37
:1047C0004720616C6C206461746100466163746FA2
:1047D00072792052455345540000007F43008054B5
:1047E000430000524300000000000080C09A991965
:1047F0003E00000000000080C09A99193E20003E53
:10480000003E0020003E003E0054656D7065726100
:10481000747572652063616C6962726174696F6E30
:10482000206661696C65642E20436F6E74696E75D5
:10483000652077697468207072657373696E67208C
:10484000746865206B6E6F622E0054656D706572C2
:1048500061747572652063616C6962726174696FFD
:104860006E20646F6E652E20436F6E74696E756581
:104870002077697468207072657373696E6720743D
:104880006865206B6E6F622E005A3020284C4544BC
:10489000206F6E2920005A3120284C4544206F6635
:1048A000662900502E492E4E2E442E412E20737420
:1048B00061746500473830004D3435004D34352083
:1048C0005A004737360054656D70657261747572B1
:1048D000652063616C6962726174696F6E206661E4
:1048E000696C65640054656D70657261747572659C
:1048F0002063616C6962726174696F6E20697320F4
:1049000066696E697368656420616E6420616374B2
:104910006976652E2054656D702E2063616C696226
:10492000726174696F6E2063616E206265206469D4
:104930007361626C656420696E206D656E752053CD
:10494000657474696E67732D3E54656D702E2063B7
:10495000616C2E004578747275646572004D6F76D7
:1049600065205A004D6F76652059004D6F766520A1
:1049700058001B5B324A437261736820646574653A
:104980006374696F6E2063616E1B5B313B304862FC
:1049900065207475726E6564206F6E206F6E6C7921
:1049A00020696E1B5B323B30484E6F726D616C202C
:1049B0006D6F6465001B5B324A5741524E494E474A
:1049C0003A1B5B313B304843726173682064657405
:1049D000656374696F6E1B5B323B30486469736159
:1049E000626C656420696E1B5B333B3048537465B1
:1049F000616C7468206D6F6465004175746F6C6FD5
:104A00006164696E672066696C616D656E742061B2
:104A10007661696C61626C65206F6E6C7920776875
:104A2000656E2066696C616D656E742073656E736A
:104A30006F72206973207475726E6564206F6E2EBC
:104A40002E2E004552524F523A2046696C616D65D8
:104A50006E742073656E736F72206973206E6F744D
:104A600020726573706F6E64696E672C20706C6560
:104A700061736520636865636B20636F6E6E656349
:104A800074696F6E2E0043616C69627261746500B7
:104A9000506C65617365206C6F616420504C4120DF
:104AA00066696C616D656E742066697273742E0040
:104AB000497320504C412066696C616D656E7420AD
:104AC0006C6F616465643F0043616E63656C0046B2
:104AD000696C616D656E740053656C65637420501C
:104AE0004C412066696C616D656E743A0052657365
:104AF000756D696E67207072696E740053757070A1
:104B00006F727400537461746973746963732020E5
:104B10000043616C6962726174696F6E0041757403
:104B20006F4C6F61642066696C616D656E740043E3
:104B300068616E676520657874727564657200558A
:104B40006E6C6F61642066696C616D656E740045A2
:104B50006A6563742066696C616D656E74004C6F84
:104B600061642066696C616D656E74004E6F2053E0
:104B7000442063617264005072696E742066726FC3
:104B80006D20534400526573756D65207072696EB7
:104B900074005061757365207072696E7400507294
:104BA00065686561740054756E65004C69766520B2
:104BB00061646A757374205A00496E666F2073636E
:104BC0007265656E0046696E697368696E67206D0F
:104BD0006F76656D656E747300536F756E6420201B
:104BE000202020205B6C6F75645D00536F756E64D0
:104BF0002020202020205B6D7574655D00536F754B
:104C00006E64202020205B73696C656E745D0053B8
:104C10006F756E642020202020205B6F6E63655DC1
:104C200000536F756E642020202020205B6C6F7510
:104C3000645D004372617368206465742E20205B9C
:104C40004E2F415D004372617368206465742E20AD
:104C500020205B6F6E5D0043726173682064657431
:104C60002E20205B6F66665D004D6F6465202020FE
:104C7000205B537465616C74685D004D6F646520E2
:104C8000202020205B4E6F726D616C5D0046696C68
:104C90002E2073656E736F7220205B6F6E5D004611
:104CA000696C2E2073656E736F72205B6F66665D34
:104CB000004368616E67652066696C616D656E743E
:104CC00000466C6F770053706565640046616E2026
:104CD000737065656400426564004E6F7A7A6C6536
:104CE0000053657474696E6773005072696E742046
:104CF00061626F7274656400596573004E6F005392
:104D0000746F70207072696E740046696C652069FA
:104D10006E636F6D706C6574652E20436F6E746981
:104D20006E756520616E797761793F004D61696EBE
:104D3000004661696C207374617473004D373032C2
:104D40002043004661726D206E756D626572004D84
:104D5000363030004D3234004D323320257300059B
:104D60002E2E0043616E6E6F7420656E7465722026
:104D70007375626469723A200053442063617264FF
:104D8000206F6B006F70656E526F6F742066616983
:104D90006C656400766F6C756D652E696E69742044
:104DA0006661696C656400534420696E69742066AD
:104DB00061696C00536F7274696E672066696C6517
:104DC0007300536F6D652066696C65732077696C3D
:104DD0006C206E6F7420626520736F727465642E30
:104DE000204D61782E204E6F2E206F662066696CF4
:104DF000657320696E203120666F6C646572206671
:104E00006F7220736F7274696E672069732031301E
:104E1000302E001F1F1F1F1F1F1F1F2E002E004E92
:104E20006F772066726573682066696C653A20004A
:104E30004E6F7720646F696E672066696C653A20F3
:104E4000002220706F73002220706172656E743AC8
:104E50002200535542524F5554494E452043414C30
:104E60004C207461726765743A2200747279696EBD
:104E70006720746F2063616C6C207375622D6763AB
:104E80006F64652066696C65732077697468207447
:104E90006F6F206D616E79206C6576656C732E2066
:104EA0004D4158206C6576656C2069733A005772E5
:104EB0006974696E6720746F2066696C653A2000BA
:104EC00046696C652073656C656374656400205386
:104ED000697A653A200046696C65206F70656E6579
:104EE000643A20001000C90210012C014001220187
:104EF00070011801B0010E01F00104015002FA0026
:104F0000B002F0003003E600D003DC009004D200D1
:104F10007005C800A006BE000008B400B009AA00D1
:104F2000D00BA000600E960060118C00001582006E
:104F300020197800C01D6E00A0226400B0275A001E
:104F4000902C500000314600E0343C001038320014
:104F5000903A2800603C1E00A03D1400803E0A00EC
:104F6000203F000070012C0190012701B0012201B7
:104F7000C0011D01F00118011002130130020E01E1
:104F80006002090190020401C002FF000003FA0060
:104F90004003F5008003F000D003EB002004E6009E
:104FA0007004E100E004DC004005D700C005D20039
:104FB0004006CD00D006C8008007C3003008BE0000
:104FC000F008B900C009B400B00AAF00B00BAA00E5
:104FD000D00CA500000EA000500F9B00C010960042
:104FE0005012910000148C00C0158700B017820089
:104FF000B0197D00D01B7800001E730040206E00A9
:1050000090226900F024640040275F0090295A0034
:10501000E02B5500102E500020304B00103246007F
:10502000E033410090353C001037370070383200D3
:10503000A0392D00B03A2800A03B2300603C1E00A0
:10504000103D1900903D1400103E0F00703E0A0004
:10505000C03E0500003F000090137D00B0157800B1
:10506000F0177300601A6E00F01C6900A01F640046
:1050700050225F0020255A00E0275500902A50005A
:10508000202D4B00A02F4600F031410010343C0091
:10509000F0353700A037320020392D00603A280063
:1050A000703B2300603C1E00203D1900C03D1400F1
:1050B000403E0F00A03E0A00F03E0500403F0000C9
:1050C000703FFBFF903FF6FFB03FF1FFC03FECFFAA
:1050D000D03FE7FFE03FE2FFF03FDDFFF03FD8FFCA
:1050E00020484F54454E4420544845524D414C2091
:1050F00052554E415741590020484541544245447C
:1051000020544845524D414C2052554E415741592B
:1051100000544845524D414C2052554E415741593B
:105120000042454420544845524D414C2052554E72
:10513000415741590020544845524D414C20525549
:105140004E4157415920282050524548454154204E
:10515000484F54454E44290020544845524D414C37
:105160002052554E4157415920282050524548451C
:105170004154204845415442454429005052454835
:10518000454154204552524F52004245442050520E
:105190004548454154204552524F52004572723A9B
:1051A000204D415854454D50003A20457874727551
:1051B000646572207377697463686564206F6666DE
:1051C0002E204D415854454D5020747269676765D3
:1051D0007265642021004572723A204D4158544551
:1051E0004D50204245440054656D70657261747580
:1051F00072652068656174656420626564207377F8
:10520000697463686564206F66662E204D4158544A
:10521000454D50207472696767657265642021008E
:105220004572723A204D494E54454D5020424544F6
:105230000054656D70657261747572652068656192
:10524000746564206265642073776974636865645B
:10525000206F66662E204D494E54454D5020747285
:10526000696767657265642021004572723A204D56
:10527000494E54454D50003A204578747275646526
:1052800072207377697463686564206F66662E2088
:105290004D494E54454D502074726967676572657B
:1052A00064202100746D63323133305F686F6D6547
:1052B0005F656E74657228617865735F6D61736B8D
:1052C0003D307825303278290A00746D63323133ED
:1052D000305F686F6D655F6578697420746D6332E7
:1052E0003133305F73675F686F6D696E675F6178D8
:1052F00065735F6D61736B3D3078253032780A00DD
:1053000046696C616D656E742073656E736F7200B3
:10531000537761707065640046726F6E742F6C65B0
:1053200066742066616E7300417869730041786924
:1053300073206C656E677468004C6F6F73652070C6
:10534000756C6C657900456E6473746F70206E6F58
:10535000742068697400456E6473746F70004D6FDB
:10536000746F7200456E6473746F70730057697266
:10537000696E67206572726F7200426564202F202B
:10538000486561746572004E6F7420636F6E6E6560
:1053900063746564004865617465722F5468657252
:1053A0006D6973746F7200506C656173652063681A
:1053B00065636B203A0053656C6674657374206591
:1053C00072726F7220210046696C616D656E742087
:1053D00073656E736F723A005072696E7420666105
:1053E0006E3A0045787472756465722066616E3A33
:1053F0000053656C6674657374206661696C6564DE
:10540000202000416C6C20636F72726563742020F1
:105410002020202000436865636B696E67207365F8
:105420006E736F72732000436865636B696E6720EB
:10543000626564202020202000436865636B696EEC
:1054400067205A2061786973202000436865636B88
:10545000696E672059206178697320200043686570
:10546000636B696E67205820617869732020004360
:105470006865636B696E6720686F74656E64202071
:1054800000436865636B696E6720656E6473746F53
:105490007073004572726F72202D2073746174698D
:1054A00063206D656D6F7279206861732062656538
:1054B0006E206F7665727772697474656E004361F1
:1054C00072642072656D6F7665640043617264205A
:1054D000696E736572746564002D2D2D2D2D2D2D33
:1054E0002D2D2D2D2D2D2D2D2D2D2D2D2D004361CF
:1054F0006C6962726174696E6720686F6D65000027
:1055000000000000110A04505255534133444657DD
:10551000002079303D25640A002078303D25640A5A
:10552000004F4B0A004552524F522061643D2564A2
:105530000A002020207A303D25640A00207A303D80
:1055400025640A002079303D25640A002078303D2A
:1055500025640A0078797A63616C5F66696E645FBE
:10556000706F696E745F63656E746572320A0020D5
:10557000746F6F206C6F6E672065787472757369D5
:105580006F6E2070726576656E7465640020636F5F
:105590006C6420657874727573696F6E20707265C3
:1055A00076656E74656400332E342E3200726300AB
:1055B0006265746100616C70686100646576007892
:1055C000797A63616C5F73706972616C32206378A1
:1055D0003D25642063793D2564207A303D25642093
:1055E000647A3D2564207261646975733D25642089
:1055F00061643D25640A0001021020200808102083
:10560000401020408002010201080402010102044E
:10561000081020408080402010080402018004020D
:105620000180402010080402010804020101020464
:105630000810204080010204081020408010080457
:105640000880102040044080102040048000002288
:1056500000250028002B002E00310034000201003C
:1056600000050108010B01050505050705080808E7
:1056700008020202020A0A080804040404010101E3
:1056800001010101010303030303030303040707EB
:10569000070C0C0C0C0C0C0C0C0202020206060689
:1056A00006060606060B0B0B0B0B0B0B0B07070A6C
:1056B0000A0A0A0A0A050505040404080802746DAA
:1056C00063323133305F676F746F5F73746570205E
:1056D0002564202564202564202564200A002E00EE
:1056E0006F70656E206661696C65642C2046696C1C
:1056F000653A20006673656E736F725F73746F70C6
:105700005F616E645F736176655F7072696E740A63
:10571000006673656E736F725F726573746F726526
:105720005F7072696E745F616E645F636F6E7469DF
:105730006E75650A0044495341424C45440A004590
:105740004E41424C4544004653656E736F722025AE
:10575000530A00504154393132355F696E69743AE9
:10576000256868750A00504154393132355F696ED9
:1057700069743A256868750A0050415439313235E8
:105780005F696E69743A256868750A0046530A00B5
:105790006673656E736F725F6F715F6D6561737352
:1057A0007572655F73746172740A006673656E73F7
:1057B0006F725F6F715F6D656173737572655F7333
:1057C000746F702C20256868752073616D706C652E
:1057D000730A004E4721004F4B005041543931327B
:1057E00035206E6F7420726573706F6E64696E67BA
:1057F0002028256429210A004D36303000465345C3
:105800004E534F525F5245434F56455200667365A3
:105810006E736F725F757064617465202D204D36F4
:1058200030300A006673656E736F725F6572725F07
:10583000636E74203D20300A0047312045332046F6
:1058400032303000473120452D3320463230300091
:105850006673656E736F725F6175746F6C6F616490
:105860005F636865636B5F7374617274202D206180
:1058700075746F6C6F616420454E41424C45440A1B
:10588000006673656E736F725F6175746F6C6F61C4
:10589000645F636865636B5F73746F70202D206154
:1058A00075746F6C6F61642044495341424C4544A8
:1058B0000A006673656E736F725F636865636B5F22
:1058C0006175746F6C6F6164203D20747275652022
:1058D0002121210A002079645F6D696E3D257520C4
:1058E00079645F6D61783D25752079645F617667C5
:1058F0003D25752073685F6176673D25750A002038
:1059000073745F73756D3D25752079645F73756D74
:105910003D25752065725F73756D3D257520657237
:105920005F6D61783D256868750A006673656E7302
:105930006F725F6F715F726573756C742025530AA7
:10594000002073685F617667203D202568687520B8
:1059500025530A002079645F717561203D2025750B
:105960002025530A002079645F646576203D202558
:10597000750A002079645F6D696E203D20257520D1
:1059800025530A002079645F6D6178203D202575DC
:105990002025530A002079645F617667203D202529
:1059A0006868752025530A002065725F6D61782054
:1059B0003D20256868752025530A002065725F73B5
:1059C000756D203D2025752025530A006673656E90
:1059D000736F725F6F715F726573756C740A00220A
:1059E000206661696C65643A20427566666572205E
:1059F00066756C6C21002200256920686F757273D2
:105A0000202569206D696E757465730054494D4594
:105A10004F55543A004D3131300046756C6C205270
:105A2000582042756666657200656E717565696EAF
:105A30006720220053544F505045442E200050728E
:105A4000696E7465722073746F707065642064751C
:105A50006520746F206572726F72732E20466978AC
:105A600020746865206572726F7220616E642075A3
:105A70007365204D39393920746F207265737461F4
:105A800072742E202854656D70657261747572652C
:105A90002069732072657365742E205365742069C4
:105AA00074206166746572207265737461727469C2
:105AB0006E6729004E6F20436865636B73756D20B8
:105AC00077697468206C696E65206E756D626572A9
:105AD0002C204C617374204C696E653A2000636819
:105AE00065636B73756D206D69736D617463682C8C
:105AF000204C617374204C696E653A2000446F6ECF
:105B000065207072696E74696E672066696C6500E5
:105B10004E6F204C696E65204E756D626572207700
:105B200069746820636865636B73756D2C204C61C4
:105B30007374204C696E653A20004C696E65204E86
:105B4000756D626572206973206E6F74204C61738D
:105B500074204C696E65204E756D6265722B312C18
:105B6000204C617374204C696E653A20000000A0DF
:105B7000400000A04000000040253364207374659D
:105B8000703D253264206D73636E743D2534640A64
:105B90000046696C616D656E74206F7574206F6668
:105BA0002072616E6765202564200A0067636F6458
:105BB000655F4D37303120626567696E0A0046695E
:105BC0006C2E2073656E736F7220726573706F6ECA
:105BD000736520697320706F6F722C206469736124
:105BE000626C652069743F0046696C616D656E7416
:105BF00020657874727564696E67202620776974F1
:105C00006820636F727265637420636F6C6F723F9C
:105C10000057616974696E6720666F72206E6F7AD3
:105C20007A6C6520616E642062656420636F6F6CBE
:105C3000696E670053656C662074657374204F4B02
:105C40000053656C6620746573742073746172749C
:105C50002020006C63645F73656C66636865636BCA
:105C60005F617869732025642C2025640A004D3813
:105C700034004731205A313520463130303000472A
:105C8000323820570025632041584953205347316B
:105C90003D25640A0041786973206C656E677468FD
:105CA00020646966666572656E63653A252E3366A3
:105CB0000A004D65617375726564206178697320AF
:105CC0006C656E6774683A252E33660A004D32346F
:105CD000004D3233202573006175746F25692E677E
:105CE0000022206661696C65643A204275666665CB
:105CF000722066756C6C2100456E717565696E6702
:105D000020746F207468652066726F6E743A20226A
:105D1000004572726F723A002200456E71756569B6
:105D20006E6720746F207468652066726F6E743AB7
:105D30002022006563686F3A004572723A20505223
:105D4000494E542046414E204552524F5200507207
:105D5000696E742066616E20737065656420697376
:105D6000206C6F776572207468656E206578706549
:105D700063746564004572723A20455854522E206F
:105D800046414E204552524F520045787472756418
:105D900065722066616E207370656564206973208A
:105DA0006C6F776572207468656E206578706563C6
:105DB000746564002F2F20616374696F6E3A70619F
:105DC00075736500526573656E640048656174693A
:105DD0006E672064697361626C6564206279207308
:105DE00061666574792074696D65722E0025533A79
:105DF00020256C640A25530A00004D37303100001D
:105E0000002100240027002A002D0030003300016B
:105E1000010000040107010A010000200023002600
:105E20000029002C002F00320000010000030106B1
:105E300001090100000A0B02090C0D0E08070304FA
:105E40000100000000000000000000000000000051
:105E50000000000000000000000000000000001230
:105E60001110000000000000000000000000000011
:105E70000000000000000000000000000000000022
:105E80000000000000000000002563252E31325381
:105E90003A2573252B30362E316600202020202015
:105EA0002020202020202020202020202020200012
:105EB0003E003E0020003E003E0020004E6F742059
:105EC0007370696E6E696E67005370696E6E696E8D
:105ED00067004C65667420686F74656E6420666147
:105EE0006E3F0046726F6E74207072696E74206629
:105EF000616E3F0046616E20746573740046696C84
:105F00002E2058643A2533642059643A2533640AB4
:105F1000496E743A202533642020536875743A2002
:105F20002533640046696C616D656E742073656E1F
:105F3000736F720A69732064697361626C65642EA1
:105F4000001B5B303B30484E6F7A7A6C65204641CF
:105F50004E3A202534642052504D0A5072696E74B6
:105F60002046414E3A20202534642052504D0A00EC
:105F70001B5B303B3048546F74616C206661696C08
:105F8000757265731B5B313B3148506F77657220CA
:105F90006661696C757265732020252D33641B5B07
:105FA000323B314846696C616D2E2072756E6F759B
:105FB00074732020252D33641B5B333B31484372BF
:105FC00061736820205820252D3364202059202516
:105FD0002D3364001B5B303B30484C617374207080
:105FE00072696E74206661696C757265731B5B31D2
:105FF0003B3148506F776572206661696C757265D8
:10600000732020252D33641B5B323B314846696C7D
:10601000616D2E2072756E6F7574732020252D337F
:10602000641B5B333B314843726173682020582006
:10603000252D336420205920252D336400546F749E
:10604000616C004C617374207072696E74001B5B2C
:10605000323B3148416D6269656E743A2020256497
:1060600025631B5B333B314850494E44413A202065
:10607000202025642563001B5B303B31484E6F7A3E
:106080007A6C653A202020256425631B5B313B3107
:10609000484265643A2020202020202564256300A2
:1060A0004501D50111241FBECFEFD1E2DEBFCDBF28
:1060B00000E00CBF16E0A0E0B2E0E2EEFFE603E095
:1060C0000BBF02C007900D92A43BB107D9F729E19D
:1060D000A4EBB6E001C01D92A33DB207E1F710E3C7
:1060E000C1E5D0E300E006C021970109802FFE0141
:1060F0000F9408B7C035D10780E00807A9F70F94BF
:10610000DF890D94E0B70C9400002F923F924F92DC
:106110005F926F927F928F929F92AF92BF92CF9237
:10612000DF92EF92FF920F931F93CF93DF93CDB740
:10613000DEB7C857D1090FB6F894DEBF0FBECDBF8A
:1061400080916F1390917013892B11F40C946E70E1
:1061500082E090E090932802809327028FE393E0FF
:106160000E94B3F48823B1F080913D1390913E13C7
:106170006AE270E005960F945FB7009711F0DC01BA
:106180001C9280913D1390913E1305960F946E29B9
:106190000C947B6BC0905E15D0905F1586010C58F7
:1061A0001C4E46E050E063E770E1C8010F94C0A7C1
:1061B000892B09F0EDC084E493E00E94B3F48823B6
:1061C00009F49BC088E50F94EB99182F89E50F948B
:1061D000EB99811112600F94AB7F8091B50601E0BD
:1061E000080F0093B506811105C08BE396E10F946B
:1061F000405E0EC048EC5FEA60E070E08BE396E141
:106200000F94FB5D882331F010923B161092B50677
:1062100001E007C0033049F710923B161092B50613
:1062200000E081E00E9463AD0E9459AD82E00E94CF
:106230005CA510FF15C086E69FE00F948EB161E06B
:10624000680F86E69FE00F94A0B185E09FE00F9471
:106250009BB1BC016F5F7F4F85E09FE00F94BAB1A7
:1062600011FF15C088E69FE00F948EB161E0680FC2
:1062700088E69FE00F94A0B183E09FE00F949BB16C
:10628000BC016F5F7F4F83E09FE00F94BAB181E064
:106290000E9463AD82E00E945CA586E792E10F94C4
:1062A000FC2740E061E081E00F94F96A0F94AB7F36
:1062B000002321F061E082EB9DE01BC0E0911A0D0C
:1062C000F0E0EE0FFF1FE05AFA4E1182108240E01C
:1062D00060E088E592E10F949C04182F81E00E9411
:1062E00063AD61E0112319F084EA9DE002C087E903
:1062F0009DE00F94685C0C947B6B83E593E00E94B7
:10630000B3F4882379F08091B70E882331F060E0F0
:1063100070E080E89FE30E94EDE281E080930D024F
:106320000C947B6B81E693E00E94B3F4882311F414
:106330000C947B6B81E080930D028091310E811172
:1063400004C00F94800C0C947B6B813011F00C9482
:106350007B6BE6E8FDE084918F01882339F00E9491
:106360007DFA0F5F1F4FF8018491F7CF8AE00E94FA
:106370007DFAE5E8F7E184918F01882311F40C940C
:10638000086A0E947DFA0F5F1F4FF8018491F5CFD4
:1063900044E050E06EE670E1C8010F94C0A7892B7D
:1063A00009F00EC1860108581C4E49E050E064E631
:1063B00070E1C8010F94C0A7892BD9F4F601EF57FB
:1063C000FC4E1081153431F01855143010F00C9437
:1063D0007B6B01C013E04AE050E060E070E0C60172
:1063E0008E579C4E0F944EA6812F0F94FB430C9416
:1063F0007B6B49E050E06AE570E1C8010F94C0A7EB
:10640000892B61F5F601EF57FC4E1081153431F000
:106410001855143010F00C947B6B01C013E04AE067
:1064200050E060E070E0C6018E579C4E0F944EA67F
:10643000E12FF0E0E45EF84F40E051E0008002C060
:10644000569547950A94E2F7842F880F880F81505C
:106450006823812F0F94DD450C947B6B49E050E05D
:1064600060E570E1C8010F94C0A7892B11F00C946E
:106470007B6BF601EF57FC4E8081853449F008EACA
:10648000902E980EF3E0F91510F40C947B6B02C07B
:1064900013E0912EE92CF12C5701AA0CBB1CF5013D
:1064A000E35DFD4F1081012F0F70712E7294BFE0DC
:1064B0007B22272D2770722E111F1127111F61813A
:1064C0006770660F162BF501E25DFD4F8081882E07
:1064D000869486948694382D3370832E1A8219827E
:1064E000C6018E579C4EDC012C912223E1F14AE03B
:1064F00050E0BE016F5F7F4F0F944EA6062F0F70C6
:1065000089819A81009779F1FC012081222359F138
:106510004AE050E0BE016F5F7F4F0F944EA6677058
:10652000762E89819A810097F1F0DC012C9122234B
:10653000D1F04AE050E0BE016F5F7F4F0F944EA64E
:10654000162F1F7089819A81009769F0FC012081C4
:10655000222349F04AE050E0BE016F5F7F4F0F9465
:106560004EA66370862EF501E35DFD4F972D977063
:106570009295907F612F679566276795902B962B54
:106580009083612F66951181107E882D8370880F0E
:10659000880F880F162B182B1183C701865E9D4F1D
:1065A000D701A25EBD4FB701645E784FFC01208128
:1065B0004C91DB016C91892D0E94099F0C947B6B9F
:1065C0008EE693E00E94B3F4882321F00F942D55BA
:1065D0000C947B6B8EE793E00E94B3F4882309F45C
:1065E000B5C184E893E00E94B3F4882391F08091D0
:1065F000F00E882311F40C947B6B0F944E866093FD
:1066000051167093521680935316909354160C940F
:106610007B6B89E893E00E94B3F4882349F0809172
:10662000A50E8F938091A40E8F9388E697E03DC0CE
:106630008DE893E00E94B3F4882329F140914F1331
:10664000509150132CE3249FC001259F900D1124DD
:106650009F938F9340914D1350914E13249FC001EF
:10666000259F900D11249F938F9381E597E09F9331
:106670008F930F949AA80F900F900F900F900F90F8
:106680000F900C947B6B81E993E00E94B3F4882314
:10669000C9F08091F00E882391F0809136078F9396
:1066A000809135078F938EE497E09F938F930F949B
:1066B0009AA80F900F900F900F900C947B6B8CE327
:1066C00097E0F0C084E993E00E94B3F4882321F0BE
:1066D000109234070C947B6B88E993E00E94B3F42A
:1066E000882349F060E085EA9FE00F94A0B161E063
:1066F0008CE490E1FECD8DE993E00E94B3F4882311
:1067000021F00E9457D90C947B6B84EA93E00E949D
:10671000B3F4882319F18091F00E8823C9F08AEA36
:1067200095E5DC018093FC1F9093FD1FA093FE1F55
:10673000B093FF1F88E08093FB1F98E10FB6F89499
:10674000A895909360000FBE80936000F894FFCFEF
:106750008AEA93E00E94B6FB0C947B6B8CEB93E08F
:106760000E94B3F4882339F180913D1390913E1338
:1067700041E061E003960F94C50E809185189091D9
:106780008618A0918718B091881880933219909339
:106790003319A0933419B09335198DE798E10E940D
:1067A00015E18C010E947DFA0A30110531F70F9432
:1067B000C73F0C947B6B8FEB93E00E94B3F488236C
:1067C00081F00F94FD6281E08093470780913D1333
:1067D00090913E1341E060E004960F94C50E0C9436
:1067E0007B6B83EC93E00E94B3F4882309F45EC0D2
:1067F0008091F00E882309F453C0109262156091C5
:10680000CD197091CE198BE390E00F94CBB06091CD
:10681000CD197091CE1983E590E00F94CBB0198219
:106820001B821A82CE0101960F94EF5D00E010E00A
:10683000FF24F3948091D50D9091D60D2091D70D22
:106840003091D80D821B930B8F779927892B81F07C
:106850000E94D9F9F09262156091CD197091CE190C
:1068600090E00F94CBB00F5F1F4F10926215E2CFF4
:1068700064E670E0CE0101960F94C65D811103C0FD
:1068800003311105BCF281E0809362156091CD194E
:106890007091CE198AE090E00F94CBB00C947B6B92
:1068A00089E595E00F94C1A80C947B6B86EC93E08E
:1068B0000E94B3F4882361F00AEC13E0F80181919F
:1068C0008F01882311F40C94086A0E947DFAF6CF98
:1068D00085ED93E00E94B3F4882361F009ED13E0A5
:1068E000D8018D918D01882311F40C94086A0E94BF
:1068F0007DFAF6CF88EF93E00E94B3F481110C94F7
:106900007B6B8DEF93E00E94B3F4882341F060E04D
:1069100070E088EF9FE00E944FC60C947B6B80E094
:1069200094E00E94B3F4882321F00F944E860C94D7
:106930007B6B85E094E00E94B3F4882311F40C94FF
:106940007B6B80E00E94A9F60C947B6B8EE50F9424
:10695000EB998AAF81110C947B6B87E40F94EB99D0
:10696000F82E882311F40C94F3410F94E2990F94BC
:1069700079B36C34710509F404C27CF56430710597
:1069800009F4FCC054F46230710509F4E2C00CF063
:10699000E9C077FF6DC00C94E7416C31710509F4D3
:1069A0003FC15CF46A30710509F435C16B30710583
:1069B00011F00C94E74180E02FC16E31710509F4AC
:1069C00071C16B34710511F00C94E74108E210E0DD
:1069D000F7E1EF2EF7E0FF2EB5C16835710511F430
:1069E0000C947B6BECF46135710511F40C94AE40A2
:1069F00054F46F34710509F431C76035710509F439
:106A000059C70C94E7416635710511F40C94574150
:106A10006735710511F00C94E74181E00C94584101
:106A20006C35710511F40C9460417CF46A35710584
:106A300011F40C945C416B35710511F00C94E74135
:106A400081E0809362190C947B6B6236710511F4BE
:106A50000C94C0416336710511F00C94E74110921B
:106A6000F00E60E084EC9FE00F94A0B10C94E24142
:106A700080910B0F81110C947B6B0F9408A3609194
:106A8000C00E7091C10E8091C20E9091C30E0F94F2
:106A900032A96B017C014090EB0F5090EC0F60909D
:106AA000ED0F7090EE0F8090140D9090150DA0904A
:106AB000160DB090170DA5019401C301B2010F94FA
:106AC00019B220E030E048EC52E40F9426A49B0178
:106AD000AC01C701B6010F9465B41816D4F4A30134
:106AE0009201C501B4010F9419B220E030E048ECE6
:106AF00052E40F9426A4A70196010F941AB20F94A2
:106B00007FB36093C00E7093C10E8093C20E9093BA
:106B1000C30E8091A510882311F40C94796B88E53D
:106B20000F94EB9981110C94796B89E50F94EB9993
:106B300081110C94796B8AE50F94EB9981110C9477
:106B4000796B85E40F94EB9981110C94506B0C9444
:106B5000796B80910B0F81110C947B6B0F94C8A300
:106B600081E008C080910B0F81110C947B6B0F9416
:106B7000C8A380E00F94559D0C947B6B80E50F9427
:106B8000EB99882339F00F94E2990F947FB36B014E
:106B90007C0103C0C12CD12C760183E50F94EB99C5
:106BA000882361F00F94E29920E030E04AE754E452
:106BB0000F9426A40F947FB36B017C01C114D10400
:106BC000E104F10421F08AEE93E10F94FC270F9485
:106BD000AB7F0F944E86C60ED71EE81EF91E0F948B
:106BE0004E86609367197093681980936919909322
:106BF0006A190F944E866C157D058E059F0510F061
:106C00000C947B6B0F94CD7980E00F940C8080E026
:106C10000E945CA5EECF81E00F94609A0C947B6B90
:106C200088E50F94EB998EAF0F94D7991B012C0137
:106C300089E50F94EB99682E0F94D79926966CAF3F
:106C40007DAF8EAF9FAF26978AE50F94EB99D82E34
:106C50000F94D7994B015C0187E50F94EB99782E3F
:106C600083E40F94EB997F928F93CD2C2696ECAC16
:106C7000FDAC0EAD1FAD2697262DB201A1018EAD44
:106C80000F9417680F900F90BEADB1110C947B6BF1
:106C900061100C947B6B71100C947B6BD1100C9475
:106CA0007B6B08C60F94AB7F81E00E941AF48C01C5
:106CB00080E090E0A8E4B4E4809322029093230261
:106CC000A0932402B093250260E070E080E291EC92
:106CD0000F947D0D8091EA0F8F938091E90F8F9330
:106CE0008091E80F8F938091E70F8F938091E60F4B
:106CF0008F938091E50F8F938091E40F8F93809114
:106D0000E30F8F938091E20F8F938091E10F8F9328
:106D10008091E00F8F938091DF0F8F9386ED9CE43D
:106D20009F938F9380E297E09F938F930F949AA8FD
:106D3000C8010E94F9F30FB6F894DEBF0FBECDBFB5
:106D40000C947B6BB801012E000C880B990B0F94EF
:106D500034A90E941F8F9F938F937F936F931F93EC
:106D60000F93FF92EF920F949AA80F5F1F4F0FB6E9
:106D7000F894DEBF0FBECDBF0F36110519F70C9486
:106D80007B6B0E94D5F98A3F30F088EC93E10F9439
:106D900079050C947B6B80911B0D882341F08091C9
:106DA0001C0D882321F080911D0D811106C081E00A
:106DB00080936E1385E490E197C581E893E10F9489
:106DC000790540E060E088E49CE10F949C0488230E
:106DD00009F493C080E090E0A0EAB0E48093E70F6C
:106DE0009093E80FA093E90FB093EA0F2091E30F7F
:106DF0003091E40F4091E50F5091E60F6091DF0F65
:106E00007091E00F8091E10F9091E20FFAE16F2E07
:106E1000FDE07F2E7F926F92812C912CA8E4AA2E08
:106E2000A2E4BA2EBBEECB2EBFE0DB2EE12CF12C80
:106E300000EA10E40F94C52E8092E70F9092E80FBD
:106E4000A092E90FB092EA0F80E090E0A4E3B3E4EF
:106E50008093E30F9093E40FA093E50FB093E60FB8
:106E60006091DF0F7091E00F8091E10F9091E20F40
:106E70007F926F928501740120E030E044E353E497
:106E80000F94C52E0F94AB7F80E29CE10F9479059F
:106E9000EEEEFEE125913591459154912093E30F5B
:106EA0003093E40F4093E50F5093E60FEAEEFEE1D6
:106EB00065917591859194916093DF0F7093E00FC8
:106EC0008093E10F9093E20FE090E70FF090E80FCE
:106ED0000091E90F1091EA0F7F926F920F94C52EE7
:106EE0000F94AB7F41E060E080E00F94F96A0F906F
:106EF0000F900F900F900F900F9020E030E04CE03B
:106F000052E46091C3197091C4198091C519909190
:106F1000C6190F9465B418160CF0A4C08091F00E39
:106F20008111A0C080E090E0A8ECB2E48093E70F6C
:106F30009093E80FA093E90FB093EA0F2091E30F2D
:106F40003091E40F4091E50F5091E60F6091DF0F13
:106F50007091E00F8091E10F9091E20FEAE1FDE086
:106F6000FF93EF93812C912C18E4A12E12E4B12E03
:106F70000BEEC02E0FE0D02EE12CF12C08EC12E429
:106F80000F94C52E80E090E0ACE0B2E48F8F98A320
:106F9000A9A3BAA30E947EA819821A821B821C820E
:106FA000CE0101960F94BD7210921F0D10921E0D0E
:106FB00019821A821B821C821D82CE0101960F94B7
:106FC000405E0F900F902F8D38A149A15AA160917A
:106FD000C3197091C4198091C5199091C6190F9465
:106FE00065B4181694F588E392E10F948F0464E079
:106FF00080E00E94AAA882E00F94BE4E83EC99E143
:107000000F94F5560E944CA788E094E00E944CA78C
:10701000CE014F960F94F5560E944CA78AE094E05B
:107020000E944CA788EE93E00E94A5940E94C98E0E
:1070300040E053E567E070E0CE0101960F94FB5D00
:10704000882309F4C0CF10E001C011E06FEF74E5B0
:1070500081E00E945FA881E00E9463AD111102C02F
:1070600080E0F8C381E00E9463AD81E090E09093FE
:10707000280280932702E7E2F0E184918F018823C0
:1070800039F00E947DFA0F5F1F4FF8018491F7CF0E
:107090008AE00E947DFA1A821982C090C319D090AA
:1070A000C419E090C519F090C61920E030E040EA1C
:1070B00050E4C701B6010F9408B30F9479B325E0EB
:1070C000269FA001279F500D1124BA01550F880B50
:1070D000990B0F9434A93B01382E292E20E030E083
:1070E0004CE052E40F942EA987FF06C0612C712C4E
:1070F000ACE03A2EB2E42B2EC101262D372D492FBC
:10710000522DC701B6010F9465B4181674F420E02F
:1071100030E040EA50E4F101662D772D8F2F922D5B
:107120000F941AB23B01382E292E2F923F927F9254
:107130006F928EEF96E09F938F930F949AA820E022
:1071400030E040EF51E4F101662D772D8F2F922D25
:107150000F9419B220E030E04CE852E40F941AB2D8
:107160000F9479B370931F0D60931E0D84E090E02F
:107170009093B90E8093B80E81E090E09093600EEA
:1071800080935F0E8FEF93E20F94FC2780E090E0F6
:10719000A0EAB0E48093E70F9093E80FA093E90F83
:1071A000B093EA0F2091E30F3091E40F4091E50F87
:1071B0005091E60F6091DF0F7091E00F8091E10F29
:1071C0009091E20FBAE14B2EBDE05B2E5F924F92A1
:1071D000812C912C18E4A12E12E4B12E0BEEC02EBE
:1071E0000FE0D02EE12CF12C00EA10E40F94C52E14
:1071F00080E090E0A0EAB1E48093DF0F9093E00F8D
:10720000A093E10FB093E20F80E090E0A0E7B2E43A
:107210008093E30F9093E40FA093E50FB093E60FF4
:10722000E090E70FF090E80F0091E90F1091EA0F5E
:107230005F924F929C01AD0160E070E080EA91E4C2
:107240000F94C52E8AE999E9A9E1BEE38093E70F7F
:107250009093E80FA093E90FB093EA0F2091E30F0A
:107260003091E40F4091E50F5091E60F6091DF0FF0
:107270007091E00F8091E10F9091E20F5F924F9239
:107280001AE9E12E19E9F12E09E11EE30F94C52E4A
:107290000F94AB7F0FB6F894DEBF0FBECDBF209129
:1072A000C3193091C4194091C5195091C619F10103
:1072B000662D772D8F2F922D0F9465B418163CF400
:1072C00088EE93E00E94A5940E94C98EE8CF60E00A
:1072D00086EA9FE00F94A0B180E090E0A0EAB0E4DD
:1072E0008093E70F9093E80FA093E90FB093EA0F14
:1072F0002091E30F3091E40F4091E50F5091E60F9C
:107300006091DF0F7091E00F8091E10F9091E20F9B
:107310000AE1402E0DE0502E5F924F92812C912C6D
:10732000E8E4AE2EE2E4BE2EFBEECF2EFFE0DF2E31
:10733000E12CF12C00EA10E40F94C52EEAEEFEE1F8
:1073400065917591859194916093DF0F7093E00F33
:107350008093E10F9093E20FEEEEFEE125913591DF
:10736000459154912093E30F3093E40F4093E50F40
:107370005093E60FE090E70FF090E80F0091E90FCF
:107380001091EA0F5F924F920F94C52E0F94AB7F2E
:1073900060E070E080E89FEB0F947D0D0F900F9000
:1073A0000F900F90882309F45BCE3091E70F27965A
:1073B0003FAF27974091E80F2B964FAF2B975091F7
:1073C000E90F2F965FAF2F976091EA0F63966FAF2B
:1073D00063976F935F934F933F9381EF96E09F93F3
:1073E0008F930F949AA80F900F900F900F900F907B
:1073F0000F908EEA9FE09FAF8EAF44244A94542CA6
:1074000013E2C12ED12CE12CF12C8201B6010D2CFE
:10741000000C880B990B0F9434A94B015C01970168
:107420002F5F3F4F3BAF2AAFDF92CF923F932F9317
:1074300045EB56E05F934F930F949AA80F900F90EF
:107440000F900F900F900F908FEF4816580611F481
:107450000C945F70BE016F5F7F4F8EAD9FAD0E9439
:107460004FC6A5019401F101662D772D8F2F922D26
:107470000F942EA91816A4F495E0E916F10471F002
:1074800095E0C90ED11CAFEF4A1A5A0AEEADFFAD16
:107490003296FFAFEEAFEAACFBACB7CF05E010E041
:1074A000C8018752984FDC01AA0FBB1FBFAFAEAF18
:1074B0003801B3E06B0E711C25E0209FC001219FB5
:1074C000900D11241BAE1AAEFC01BD966596FFAF60
:1074D000EEAF6597AAE14A2EADE05A2EC30102979E
:1074E00005970CF0B6C165966EAD7FAD65978AAC19
:1074F0009BAC680D791D072E000C880B990B0F941F
:1075000034A926966CAF7DAF8EAF9FAF26977F9242
:107510006F92B8EAAB2EB6E0BB2EBF92AF920F943B
:107520009AA87092600E60925F0E20E030E040EF0B
:1075300051E426966CAD7DAD8EAD9FAD26970F9430
:1075400019B220E030E040E251E40F9426A420E09C
:1075500030E040EA50E40F9408B320E030E048E423
:1075600052E40F941AB20F9479B370931F0D609385
:107570001E0D80E090E0A0EAB0E48093E70F9093C6
:10758000E80FA093E90FB093EA0F2091E30F309139
:10759000E40F4091E50F5091E60F6091DF0F70917D
:1075A000E00F8091E10F9091E20F5F924F92812C5A
:1075B000912C18E4A12E12E4B12E0BEEC02E0FE098
:1075C000D02EE12CF12C00EA10E40F94C52E80E0BF
:1075D00090E0A0EAB1E48093DF0F9093E00FA093D6
:1075E000E10FB093E20F812C912CF0E7AF2EF2E483
:1075F000BF2E8092E30F9092E40FA092E50FB0921D
:10760000E60FE090E70FF090E80F0091E90F10917E
:10761000EA0F5F924F92812C912C28E4A22E22E453
:10762000B22E20E030E040E752E4BC01CD010F94DF
:10763000C52E2AE939E949E15EE32093E70F30934B
:10764000E80F4093E90F5093EA0F2091E30F309138
:10765000E40F4091E50F5091E60F6091DF0F7091BC
:10766000E00F8091E10F9091E20F5F924F921AE943
:10767000E12E19E9F12E09E11EE30F94C52E0F94B6
:10768000AB7F0FB6F894DEBF0FBECDBF2091C319FC
:107690003091C4194091C5195091C61926966CAD08
:1076A0007DAD8EAD9FAD26970F9465B418163CF452
:1076B00088EE93E00E94A5940E94C98EE7CF80E0F7
:1076C00090E0A0EAB0E48093E70F9093E80FA093D6
:1076D000E90FB093EA0F2091E30F3091E40F40914E
:1076E000E50F5091E60F6091DF0F7091E00F8091F0
:1076F000E10F9091E20F5F924F92812C912CE8E480
:10770000AE2EE2E4BE2EFBEECF2EFFE0DF2EE12C0C
:10771000F12C00EA10E40F94C52EEAEEFEE165912B
:107720007591859194916093DF0F7093E00F809332
:10773000E10F9093E20FEEEEFEE125913591459138
:1077400054912093E30F3093E40F4093E50F50934F
:10775000E60FE090E70FF090E80F0091E90F10912D
:10776000EA0F5F924F920F94C52E0F94AB7F60E0AB
:1077700070E080E89FEB0F947D0DAAADBBAD159630
:10778000BBAFAAAFBFEF6B1A7B0A0F900F900F90A1
:107790000F90811103C00F94099A5BC027967FADAB
:1077A00027972B966FAD2B972F969FAD2F976396AC
:1077B0008FAD6397272F362F492F582F6091E70FF2
:1077C0007091E80F8091E90F9091EA0F0F9419B230
:1077D000162F072FF82EE92E20912F103091301000
:1077E0004091311050913210D801F7016B2F7A2F50
:1077F0008F2F9E2F0F9426A40F9479B37A836983D9
:10780000EF92FF920F931F938091C6198F938091EF
:10781000C5198F938091C4198F938091C3198F9349
:10782000ECE7F6E0FF93EF930F949AA8BE016F5F29
:107830007F4F8EAD9FAD0E944FC62EAD3FAD2E5FE8
:107840003F4F3FAF2EAF0FB6F894DEBF0FBECDBF98
:1078500045CE81E00F94099A0C947B6B0FEF10E0FA
:1078600094E7C92E96E0D92E1093B0190093AF1962
:1078700084E6E82EF12C84E690E00E94A59451E085
:10788000E51AF108C1F7809150138F9380914F133F
:107890008F931F930F93DF92CF920F949AA8055066
:1078A00011090F900F900F900F900F900F90E1F62D
:1078B0000C947B6B81E08093D10E20911B0D809105
:1078C0009A0F90919B0F222341F020911C0D2223AF
:1078D00021F050901D0D51100FC0029749F081E02A
:1078E00080936E1380E290E10F94C2720C947B6BD4
:1078F0001092D10E0C947B6B0297D1F38091B80E4D
:107900009091B90E28969FAF8EAF2897A0915F0EE9
:10791000B091600E2C96BFAFAEAF2C9781E090E097
:107920009093B90E8093B80E83E190E09093600E2F
:1079300080935F0E81E00E945CA50F94B9490E947C
:10794000F6DB80E090E0A0EAB0E48093E70F90934C
:10795000E80FA093E90FB093EA0F2091E30F309165
:10796000E40F4091E50F5091E60F6091DF0F7091A9
:10797000E00F8091E10F9091E20F0AE1602E0DE09F
:10798000702E7F926F92E5E58E2E982CA82CE1E464
:10799000BE2EFBEECF2EFFE0DF2EE12CF12C00EA15
:1079A00010E40F94C52EE1EEF4E265917591859196
:1079B00094916093DF0F7093E00F8093E10F9093A9
:1079C000E20FE5EEF4E22591359145915491209333
:1079D000E30F3093E40F4093E50F5093E60FE090F0
:1079E000E70FF090E80F0091E90F1091EA0F7F92F6
:1079F0006F92812C912CB8ECAB2EB2E4BB2E0F947D
:107A0000C52E0F94AB7F0F900F900F900F9005EC49
:107A10001FE0C8010F949BB1019639F00E5F1F4F14
:107A2000053DEFE01E07A9F75AAE80E00E941AF468
:107A300060969FAF8EAF609711EE412E14E2512EEB
:107A4000612C712CC30163E070E00F94D9B62496C9
:107A50007FAF6EAF24971C0160FF06C0B2E08B2E93
:107A6000912C881A990A14019AAC9920A1F16114F9
:107A7000710489F124968EAD9FAD2497880F991FCC
:107A80002496AEACBFAC24978A0D9B1D820D931D2E
:107A9000880F991F8D53904F0F949BB1BC01990F84
:107AA000880B990B0F9434A92AE037ED43E25CE38D
:107AB0000F9426A4209164153091651540916615A8
:107AC000509167150F941AB222966CAF7DAF8EAFAE
:107AD0009FAF229706C022961CAE1DAE1EAE1FAEF3
:107AE000229720E030E040EA50E42093E70F309303
:107AF000E80F4093E90F5093EA0F2091E30F309184
:107B0000E40F4091E50F5091E60F6091DF0F709107
:107B1000E00F8091E10F9091E20FAAE1BDE0BF93E9
:107B2000AF93812C912CE0EAAE2EE1E4BE2EFBEE69
:107B3000CF2EFFE0DF2EE12CF12C00EA10E40F94B1
:107B4000C52E0F94AB7FF20185919591A591B491CB
:107B50008093DF0F9093E00FA093E10FB093E20FBB
:107B6000F201349685919591A591B4918093E30F9C
:107B70009093E40FA093E50FB093E60F63EE7FE0E0
:107B80008FED9FE00E9475F5E090E70FF090E80F11
:107B90000091E90F1091EA0F2091E30F3091E40F6B
:107BA0004091E50F5091E60F6091DF0F7091E00F6B
:107BB0008091E10F9091E20FBAE18B2EBDE09B2EF8
:107BC0009F928F92812C912CE6E1AE2EE3E4BE2EA3
:107BD0000F94C52E0F94AB7F0F900F900F900F90C6
:107BE000BAACBB2081F06114710469F020E030E090
:107BF00040E85FE322966CAD7DAD8EAD9FAD2297E0
:107C00000F9419B204C060E070E080E291EC0F9430
:107C10007D0D882309F48EC0C090E70FD090E80F47
:107C2000E090E90FF090EA0FA701960160E070E0A4
:107C300080EA90E40F9419B22DEC3CEC4CEC5DE33F
:107C40000F942EA987FD7BC02AAD2223A1F0A701A6
:107C5000960122966CAD7DAD8EAD9FAD22970F94AF
:107C600019B29F7720E030E040E85FE30F9465B4FD
:107C700018160CF469C0C090C319D090C419E090D4
:107C8000C519F090C61980911B078823A9F00E949E
:107C90009AF6882389F0C701B6010E941F8F2091B0
:107CA0002F103091301040913110509132100F94BC
:107CB00008B39B01AC0103C020E030E0A901A7E0BC
:107CC00024968EAD9FAD2497A89F8001A99F100D8B
:107CD0001124020D131D000F111F000F111F0D594C
:107CE0001A4E6091E70F7091E80F8091E90F909123
:107CF000EA0F0F9419B2F80161837283838394832E
:107D000080915F0E9091600E01979093600E80932A
:107D10005F0EFFEF6F1A7F0A81E00E945CA528E0EA
:107D2000420E511C39E06316710409F08BCE412CD0
:107D3000512C0EC000E3402E05E2502E09C014E382
:107D4000412E13E1512E04C0B1EF4B2EB2E15B2E58
:107D500080E090E0A0EAB0E48093E70F9093E80F12
:107D6000A093E90FB093EA0F2091E30F3091E40F55
:107D70004091E50F5091E60F6091DF0F7091E00F99
:107D80008091E10F9091E20FEAE1FDE0FF93EF9324
:107D9000812C912CE0EAAE2EE1E4BE2EFBEECF2E3C
:107DA000FFE0DF2EE12CF12C00EA10E40F94C52E49
:107DB0000F94AB7F0F900F9049E06416710421F08F
:107DC00060E0C2010C94E14960968EAD9FAD609772
:107DD0000E94F9F30E94A3DB6091180D7091190DB8
:107DE000072E000C880B990B0F9434A99058209102
:107DF0002F103091301040913110509132100F946B
:107E000008B30E94B4DB80EC9FE00F948EB1082F82
:107E1000CE0101969BAF8AAF10E0809091029090C6
:107E20009202A0909302B090940222968CAE9DAEE6
:107E3000AEAEBFAE229750E7252E55E1352E67EB4B
:107E4000862E65E1962E22962CAD3DAD4EAD5FADF2
:107E5000229729833A834B835C83AAADBBAD8D9176
:107E6000BBAFAAAF0F94EB99882319F00F94D79961
:107E70001BC0013009F026C1123028F4112341F053
:107E80008EEB9FE00AC0123031F08CEB9FE005C012
:107E90008FEB9FE002C08DEB9FE00F948EB1682FB7
:107EA000880F770B880B990B61157105810591057A
:107EB00009F408C10F9434A92FE632E143E85AE3EC
:107EC0000F9426A46B017C019F7727E139ED4EECDE
:107ED0005DE30F9465B418160CF033C0E1E1FDE5E5
:107EE00084915F01882341F00E947DFAFFEFAF1A71
:107EF000BF0AF5018491F6CFECEFFFE084915F01BA
:107F0000882341F00E947DFAFFEFAF1ABF0AF50106
:107F10008491F6CF42E0C701B6010E9420FBE3EF57
:107F2000FFE084917F01882341F00E947DFAFFEFFA
:107F3000EF1AFF0AF7018491F6CF8AE00E947DFADA
:107F4000C1C020E030E040E05FE3C701B60112307D
:107F500009F463C0133009F48AC0113071F10F9431
:107F600026A42B013C0143E6A42E45E1B42EA30137
:107F70009201D50115966D917D918D919C911897E7
:107F80000F941AB2F5016583768387839087A701E2
:107F9000960161817281838194810F941AB2D50117
:107FA00011966D937D938D939C931497BCE1AB0ECA
:107FB000B11C8A149B04D9F685C00F9426A42B010A
:107FC0003C0133E6A32E35E1B32EA3019201F50166
:107FD00065817681878190850F941AB2D5011596B7
:107FE0006D937D938D939C931897A7019601199695
:107FF0006D917D918D919C911C970F941AB2F50112
:108000006187728783879487FCE1AF0EB11C27EBF1
:10801000A21625E1B206C9F655C00F9426A42B017D
:108020003C0124E6A22E25E1B22EA3019201D50146
:108030005C966D917D918D919C915F970F941AB292
:10804000F501648F758F868F978FA70196016081E8
:108050007181828193810F941AB2D5016D937D93C2
:108060008D939D935D012A163B06F9F62BC00F9464
:1080700026A42B013C0190E8A92E95E1B92EA3017D
:108080009201F50160817181828193810F941AB20E
:10809000D5016D937D938D939D935D01A70196010D
:1080A00058966D917D918D919C915B970F941AB22A
:1080B000F501608F718F828F938FFCE8AF16F5E129
:1080C000BF06E9F61F5F143009F0BDCE0F94D14909
:1080D00081E0809363150E948AA0E0911A0D24E04C
:1080E000E29FF0011124EB58F04F20E030E04FE226
:1080F00053E460817181828193810F9465B4181675
:1081000084F480911B07882361F00E949AF68823EB
:1081100041F080911E0D90911F0DC29714F00C94A8
:10812000D16B81E090E0909328028093270287EE44
:1081300094E10F94FC2728964EAD5FAD289750939D
:10814000B90E4093B80E2C968EAD9FAD2C979093A0
:10815000600E80935F0E1092D10E34C18091631532
:10816000882309F495C0E9EEFFE084918F0188230C
:1081700039F00E947DFA0F5F1F4FF8018491F7CF0D
:1081800067E070E080E090E00E9406FBE7EEFFE031
:1081900084918F01882339F00E947DFA0F5F1F4F71
:1081A000F8018491F7CF67E070E080E090E00E94F2
:1081B00006FBE4EDFFE084918F01882339F00E94F3
:1081C0007DFA0F5F1F4FF8018491F7CF65E070E0F3
:1081D00080E090E00E9406FBE2ECFFE084918F01DA
:1081E000882339F00E947DFA0F5F1F4FF8018491B8
:1081F000F7CF8AE00E947DFA00E010E0BFEB6B2E23
:10820000BFE07B2E8DEBA82E8FE0B82EE12CF12C59
:108210004801F8EA8F0E911CF3018491AFEBCA2E4E
:10822000AFE0DA2E882341F00E947DFAFFEFCF1AEB
:10823000DF0AF6018491F6CFF401EE0DFF1DED5932
:10824000FA4E618172818381948145E00E9420FB16
:10825000F4E0EF0EF11C2CE1E216F104E9F6F50171
:108260008491FDEBEF2EFFE0FF2E882341F00E946A
:108270007DFAFFEFEF1AFF0AF7018491F6CF0C5158
:1082800011090C33FFEF1F0709F0C0CF0C947B6B73
:10829000EFE9FFE084918F01882311F40C94086AC0
:1082A0000E947DFA0F5F1F4FF8018491F5CF86EE93
:1082B0000E94A4F60C947B6B109262190C947B6B59
:1082C00085E40F94EB99811102C00F94AB7F66E3B4
:1082D000662E63E0762E7FEDA72E7FE0B72EEBE7CC
:1082E0008E2EE0E19E2ED12CD3018D913D010F9475
:1082F000EB998823C9F1B3E0DB120CC00F94E2992B
:10830000F50160837183828393838BEE9FE00E94EB
:1083100083BA2AC00F94E2999B01AC01D4016D91FC
:108320007D918D919C910F941AB2F50160837183B8
:1083300082839383E090E70FF090E80F0091E90FBC
:108340001091EA0F2091E30F3091E40F4091E50F77
:108350005091E60F6091DF0F7091E00F8091E10F77
:108360009091E20F0F944A42D394F4E0AF0EB11C07
:1083700024E0820E911C34E0D312B6CF0C947B6BB8
:1083800081E08093F00E0F944E86609351167093A7
:10839000521680935316909354166091F00E84EC0D
:1083A0009FE00F94A0B165E377E081EC9FE00E942D
:1083B0004FC61092BA0E60E08FEF9FE00F94A0B10D
:1083C0000C947B6B82E00E945CA50C947B6B80918B
:1083D0005E1590915F158C589C4E9F938F938AE801
:1083E0009FE00C9455338DE40F94EB99882311F49E
:1083F0000C942469E0913D13F0913E1331968191E4
:108400008032E9F38930D9F380538A3060F080916B
:108410005E1590915F158C589C4E9F938F9385E7C6
:108420009FE00C9455330F94E2990F9479B3AB010C
:10843000BC01CA0150931E0E40931D0E4B3C5105CA
:1084400011F40C940C520CF05CC14135510511F43F
:108450000C940C4D0CF0C1C04A31510509F4EEC327
:10846000ACF54431510509F453C394F4413151053D
:1084700009F444C334F44230510508F48CC20C941E
:108480000D694231510511F40C942A4D0C940D697B
:108490004731510509F480C37CF44531510509F495
:1084A00077C34631510511F00C940D69109257169F
:1084B000109258160C941F694831510509F484C371
:1084C0004931510509F4ADC30C940D694032510591
:1084D00009F4AEC50CF05AC04D31510511F40C949D
:1084E0001F6954F44B31510509F4B6C34C315105A1
:1084F00009F4A1C40C940D694E31510509F4C7C4A7
:108500004F31510511F00C940D690F944E86009176
:10851000C80E1091C90E2091CA0E3091CB0E6B017E
:108520007C01C01AD10AE20AF30AC701B60128EE9B
:1085300033E040E050E00F94DEB1CA01B9012CE312
:1085400030E040E050E00F94DEB17F936F93C701BD
:10855000B60120E63AEE40E050E00F94DEB13F93E2
:108560002F9386E69FE09F938F938E010F5F1F4F9F
:108570001F930F930F94F2A8E3E3FDE584910FB6E8
:10858000F894DEBF0FBECDBF7F01EDC54D32510562
:1085900009F44BC6C4F44A32510509F4FFC54C3204
:1085A000510511F00C940D698FEF0E94A4F660E064
:1085B00070E088EF9FE00F94BAB10E94E2A20E949F
:1085C000C4A20C941F694F32510509F435C64934D1
:1085D000510509F477C60C940D694E36510511F416
:1085E0000C942F4E0CF042C04C35510511F40C94F4
:1085F000AB4D0CF54435510511F40C942A4D7CF427
:108600004235510511F40C94264D4335510511F0B6
:108610000C940D6981E08093230E0C941F694535FD
:10862000510511F40C94714D4635510511F40C941B
:108630008C4D0C940D694A36510511F40C94D64CAE
:1086400054F44836510509F49AC64936510509F4DF
:10865000CBC60C940D694B36510511F40C94064DA4
:108660004D36510509F4DFC70C940D6948375105A3
:1086700011F40C9439500CF54237510511F40C9457
:10868000584F5CF44037510509F498C641375105FD
:1086900011F40C94424E0C940D694337510511F4BA
:1086A0000C947F4E4737510511F00C940D69E1EFA2
:1086B000F5E084918F010C9442504E3B510511F42A
:1086C0000C94AD4B5CF44937510511F40C943D50BA
:1086D0004C38510509F477C60C940D69483C510596
:1086E00011F40C945B51493C510511F00C940D6947
:1086F00046E3E42E43E0F42E03E210E1D12C0C9487
:10870000C751873F41E0940711F40C94785A0CF05C
:108710008AC08C3261E0960711F40C94C154C4F500
:10872000803D910511F40C94AF53A4F48D3C910558
:1087300011F40C94AA5214F40C9465528E3C9105D9
:1087400011F40C9459538F3C910511F40C94785307
:108750000C940D698D3D910511F40C943D5464F415
:10876000813D910511F40C94D7538C3D910511F482
:108770000C942C540C940D69823E910511F40C94C8
:108780005E54803F910511F40C941F690C940D699F
:108790008F35B1E09B0711F40C941F690CF58F32F3
:1087A000F1E09F0711F40C9462566CF48D3231E0C5
:1087B000930711F40C94F9548E32914011F40C94F7
:1087C0004D560C940D69803351E0950711F40C94CB
:1087D000B5558E35914011F40C9422680C940D69B6
:1087E000843FA1E09A0711F40C94705A6CF480391C
:1087F000E1E09E0711F40C94285A8339914011F45A
:108800000C942C5A0C940D69853F21E0920711F4C9
:108810000C94745A863F914011F00C940D690E949B
:10882000F9FB0C941F698D3843E094070CF04FC09E
:108830008B3853E0950714F00C941F698D3B62E070
:10884000960711F40C94BF680CF58835B2E09B07CD
:1088500011F40C94075E5CF48D3F914011F00C9480
:108860000D69E3E3FDE584918F010C94305D89355A
:1088700022E0920711F40C94E7628A35924011F0DD
:108880000C940D690F943C0C0C941F698C3543E0DB
:10889000940711F40C94EA626CF48E3B62E0960744
:1088A00011F40C94CB688335934011F40C94485D1B
:1088B0000C940D698D35B3E09B0711F40C94BB63E8
:1088C0008438934011F40C94D7650C940D69833966
:1088D000F3E09F0711F40C9464673CF5803933E0B2
:1088E000930711F40C9432676CF48E3853E09507BB
:1088F00011F40C94FD668F38934011F40C940067CA
:108900000C940D698139A3E09A0711F40C941F6946
:108910008239934011F00C940D69109224070E9443
:1089200067BA0F945D180C941F698639E3E09E07BF
:1089300011F40C94F2676CF4843923E0920711F47B
:108940000C946C678539934011F40C94C2670C94B5
:108950000D69803A43E0940709F4D6C3873E9340FB
:1089600011F00C940D6910920B0F10928E0F8091E4
:10897000200D9091210DA091220DB091230D809397
:108980003F1390934013A0934113B09342130F945D
:10899000F5810C941F69E0913D13F0913E138F0116
:1089A0000E5F1F4F80E50F94EB99882371F00F94B1
:1089B000E2990F947FB36B017C01AA24A394672BE7
:1089C000682B692B31F4A12C04C0A12CC12CD12C13
:1089D000760183E50F94EB99882391F00F94E29947
:1089E00020E030E04AE754E40F9426A40F947FB3CC
:1089F0006B017C01BB24B394672B682B692B09F4B2
:108A0000B12C6AE270E0C8010F945FB7009711F0D3
:108A1000DC011C92F801CF0121912032E1F3A11079
:108A200007C0B11005C0222319F00F946E2904C0AD
:108A300080EE92E10F94FC2781E08093BF0E1092AC
:108A4000BE0E0F94AB7F0F944E86609367197093A0
:108A500068198093691990936A19C114D104E104CB
:108A6000F10419F10F944E86C60ED71EE81EF91EAA
:108A700084E090E090932802809327020F944E8622
:108A80006C157D058E059F0510F00C94136C0E94EB
:108A900034A681110C94136C0F94CD7981E00F945E
:108AA0000C8080E00E945CA5E9CF84E090E0909388
:108AB0002802809327020E9434A6811109C00F94D6
:108AC000CD7981E00F940C8080E00E945CA5F3CF0B
:108AD00082E090E0909328028093270280915716BD
:108AE000882331F08DEE9AE40F94FC270C941F69D3
:108AF00087EE94E10F94FC270C941F6987ED92E1B7
:108B00000F94FC2717981698159814980C941F69C1
:108B1000E4E6F6E084918F01882339F00E947DFA23
:108B20000F5F1F4FF8018491F7CF8AE00E947DFA12
:108B300010923819109237198BEA96E10E9457DE8D
:108B40008BE1EBEAF6E1DE01119601900D928A9538
:108B5000E1F740E050E0BE016F5F7F4F8BE094E0B3
:108B60000F948977CE0101960E94C7F4E6E5F6E0FE
:108B700084918F01882339F00E947DFA0F5F1F4F87
:108B8000F8018491F7CF8AE00E947DFA0C941F6966
:108B90000F949B130C941F6980913D1390913E1389
:108BA0006AE270E004960F945FB7009711F0DC0161
:108BB0001C9280913D1390913E1341E061E0049638
:108BC0000F94C50E0C941F6980915916811114C021
:108BD00060E086E69FE00F94A0B160E088E69FE049
:108BE0000F94A0B160E085E69FE00F94A0B160E033
:108BF00084E69FE00F94A0B180915816882329F055
:108C000081E080935716109259160F944E86609308
:108C1000C80E7093C90E8093CA0E9093CB0E0C941D
:108C20001F6980915716882311F40C941F691092C4
:108C3000571681E0809359160C941F69809158163D
:108C4000882311F40C941F6983E50F94EB9981112B
:108C50000C941F6C0C941F6980915716882309F49B
:108C6000B8C003E716E1F80181918F01882319F05C
:108C70000E947DFAF8CFE4E8FDE084918F0188231B
:108C800039F00E947DFA0F5F1F4FF8018491F7CFF2
:108C9000E7E4F5E084918F01882339F00E947DFAA2
:108CA0000F5F1F4FF8018491F7CF609132197091D7
:108CB000331980913419909135194AE00E9495FA40
:108CC000E2E8FDE084918F01882339F00E947DFA6B
:108CD0000F5F1F4FF8018491F7CF60912A197091AF
:108CE0002B1980912C1990912D194AE00E9495FA28
:108CF0008AE00E947DFA0F944E8640E6C42E4AEE2A
:108D0000D42EE12CF12CA70196010F94DEB149017C
:108D10005A016091C80E7091C90E8091CA0E90914F
:108D2000CB0EA70196010F94DEB18401021B130B39
:108D3000C8016CE370E00F94C5B6CB019927EAE057
:108D4000F0E0BF010F94D9B6282FCB01BF010F94DB
:108D5000D9B6805D8093A719205D2093A819109241
:108D6000A91957EAE52E59E1F52E6701D6018D9133
:108D70006D01882319F00E947DFAF8CF8AE30E94E2
:108D80007DFAC8016CE370E00F94C5B66AE070E04C
:108D90000F94D9B6605D6093A719805D8093A81980
:108DA0001092A919F70181917F01882319F00E947F
:108DB0007DFAF8CFE0E8FDE084918F01882311F47B
:108DC0000C941F690E947DFA0F5F1F4FF801849178
:108DD000F5CF80915916882371F0E0E7FDE084918A
:108DE0008F01882309F4CFCE0E947DFA0F5F1F4FB9
:108DF000F8018491F6CF8091B70E882371F0E4E6F4
:108E0000FDE084918F01882309F4BDCE0E947DFA94
:108E10000F5F1F4FF8018491F6CFE4E5FDE08491E8
:108E20008F01882309F4AFCE0E947DFA0F5F1F4F98
:108E3000F8018491F6CF80913D1390913E136AE240
:108E400070E004960F945FB78C01892BA9F0809194
:108E50005E1590915F156EE470E08C589C4E0F94F7
:108E60005FB760E270E00F945FB7019690933E1396
:108E700080933D13D8011C9280913D1390913E1335
:108E800041E060E004960F94C50E0C941F69809138
:108E90005816882311F40C941F690F94C73F8091D2
:108EA0003D1390913E136AE270E004960F945FB711
:108EB0008C01892BA9F080915E1590915F156EE46D
:108EC00070E08C589C4E0F945FB760E270E00F9496
:108ED0005FB7019690933E1380933D13F801108283
:108EE000C0903D13D0903E1386010C5F1F4F8091C0
:108EF0005816882311F40C941F698DE798E10E949D
:108F0000FADC109257161F8E1AA28BEA96E1909304
:108F1000C7168093C6160115110591F0D601149657
:108F20008C918F3239F4BE01615E7F4FC8010F947E
:108F3000BB4106C088EC96E19093C7168093C61695
:108F40006091C6167091C71619821C8222E0A80192
:108F5000CE0101960E9480E68823A1F0CE01019601
:108F60000F94F776882371F061E0CE0101960E949C
:108F700003DD009739F025EEFC0120831C820F945D
:108F80004E5EF82ECE0101960E94C7F4FF2021F11B
:108F9000E6E4FDE084917F01882341F00E947DFAA0
:108FA000FFEFEF1AFF0AF7018491F6CFD8018D91F8
:108FB0008D01882319F00E947DFAF8CF8AE00E9483
:108FC0007DFA1092321910923319109234191092BE
:108FD00035190F94881126C0EEE2FDE084917F01DF
:108FE000882341F00E947DFABFEFEB1AFB0AF701DC
:108FF0008491F6CFD8018D918D01882319F00E94BC
:109000007DFAF8CFECE2FDE084918F01882339F0FE
:109010000E947DFA0F5F1F4FF8018491F7CF8AE01D
:109020000E947DFACE014F960E94C7F40C941F69EE
:109030008091571681110F94AB7F00913D131091D1
:109040003E130C5F1F4F6AE270E0C8010F945FB7D8
:109050007C0161E270E0C8010F945FB7009719F0DE
:109060008C010F5F1F4FE114F10411F0D7011C9226
:1090700080E50F94EB99F82E80913D1390913E136B
:109080000817190708F4F12C80915816882311F459
:109090000C941F6941E04F2561E0C8010F94C50E93
:1090A00083E50F94EB998823B9F080913D1390915B
:1090B0003E138017910780F40F94D799AB01BC0140
:1090C00040933219509333196093341970933519C2
:1090D0008DE798E10E9410DC80915816882329F0D2
:1090E00081E08093571610925916F1100C941F6965
:1090F0000F944E866093C80E7093C90E8093CA0E6B
:109100009093CB0E0C941F6980913D1390913E1368
:109110006AE270E005960F945FB78C01892BA9F085
:1091200080915E1590915F156EE470E08C589C4EB6
:109130000F945FB760E270E00F945FB70196909371
:109140003E1380933D13F801108280913D1390915E
:109150003E1321E02093561641E060E005960F94FF
:10916000C50E0C941F69882341F00E947DFA3FEFE1
:10917000E31AF30AF7018491F6CF7801D7018D91B4
:109180007D01882319F00E947DFAF8CF8AE00E94C1
:109190007DFAC8010F946E290C941F6983E50F9422
:1091A000EB99882311F40C941F690F94E2990F94A2
:1091B00079B3F62EE72E862F9E2D8C0180E50F9435
:1091C000EB99882331F00F3F110509F010F40C944E
:1091D000306C0DE010E0E5E9F2E0819191918017AB
:1091E000910711F40C941F69B2E0ED3CFB07A9F75D
:1091F0000630110539F48F2D9E2D9093B019809370
:10920000AF1904C017FF02C00C941F6961E0802FE2
:109210000F9433846F2D802F0F9405846F2D7E2D36
:10922000802F0F946F840C941F698AE50F94EB993B
:109230000E9488700C941F6984E090E0909328024B
:10924000809327020E9459AD0F94CD7981E00F944D
:109250000C8060E080E00E94AAA88DE19DE00E9461
:10926000D1A761E080E00E94AAA81E9903C087E10F
:109270009DE002C08AE19DE00E94D1A762E080E00B
:109280000E94AAA81D9903C081E19DE002C084E16B
:109290009DE00E94D1A763E080E00E94AAA81C99EB
:1092A00003C08BE09DE002C08EE09DE00E94D1A74C
:1092B0000E9434A6882341F20E9459AD0F94B388CE
:1092C0000C941F6980E50F94EB99882331F00F947B
:1092D000E2990F947FB360933E0282E50F94EB997D
:1092E000882341F00F94E2990F947FB37093420268
:1092F0006093410281E50F94EB99882331F00F943C
:10930000E2990F947FB360933D0283E50F94EB994C
:10931000882341F00F94E2990F947FB37093400239
:1093200060933F02809142028F93809141028F931C
:1093300080913E021F928F9382E196E09F938F93DC
:1093400009E116E01F930F930F949AA880914002B1
:109350008F9380913F028F9380913D021F928F9354
:109360008BE096E09F938F931F930F930F949AA88F
:109370000FB6F894DEBF0FBECDBF0C941F69BE01BF
:109380006F5F7F4F88E690E00F941A9681110C94DE
:109390001F6983E50F94EB99882311F40C941F69DE
:1093A00019810F94E29911110C941F690F9479B3EC
:1093B00070936115609360150C941F6963E08AE0F7
:1093C00096E00E94F89583E50F94EB99882311F4B9
:1093D0000C941F690F94E2990F9479B370931F0D49
:1093E00060931E0D0C941F69BE016F5F7F4F89E66D
:1093F00090E00F941A9681110C941F69E0E6FFE04B
:1094000084918F01882339F00E947DFA0F5F1F4FEE
:10941000F8018491F7CFE98124E0E29FF001112463
:10942000EB58F04F608171818281938141E00E940D
:1094300020FBEDE5FFE084918F01882339F00E9445
:109440007DFA0F5F1F4FF8018491F7CFE981F0E0BB
:10945000EE0FFF1FE05AFA4E60817181072E000C5B
:10946000880B990B0F9434A941E00E9420FBE9E599
:10947000FFE084918F01882339F00E947DFA0F5F0D
:109480001F4FF8018491F7CF609114077091150771
:10949000809116079091170741E00E9420FBE6E5B6
:1094A000FFE084918F01882339F00E947DFA0F5FDD
:1094B0001F4FF8018491F7CF60911E0D70911F0D21
:1094C000072E000C880B990B0F9434A941E00E94E1
:1094D00020FBE3E5FFE084918F01882339F00E94AF
:1094E0007DFA0F5F1F4FF8018491F7CF60E070E0C5
:1094F000CB010E9406FBE1E5FFE084918F01882308
:1095000039F00E947DFA0F5F1F4FF8018491F7CF69
:109510006091750F7091760F8091770F9091780F11
:1095200041E00E9420FBEEE4FFE084918F0188235C
:1095300039F00E947DFA0F5F1F4FF8018491F7CF39
:109540006091601570916115072E000C880B990BC6
:109550000F9434A941E00E9420FBEAE4FFE08491EB
:109560008F01882339F00E947DFA0F5F1F4FF801A9
:109570008491F7CFE981F0E0E75FF04F608170E020
:1095800080E090E00E9406FBE5E4FFE084918F011B
:10959000882339F00E947DFA0F5F1F4FF8018491F4
:1095A000F7CF6091080F70E080E090E00E9406FB2A
:1095B000E1E4FFE084918F01882339F00E947DFA75
:1095C0000F5F1F4FF8018491F7CF6091C31970911D
:1095D000C4198091C5199091C61941E00E9420FBE1
:1095E000EDE3FFE084918F01882339F00E947DFA3A
:1095F0000F5F1F4FF8018491F7CF6091BF197091F1
:10960000C0198091C1199091C21941E00E9420FBBC
:109610008AE00E947DFA81E090E090932802809396
:1096200027020C946E70BE016F5F7F4F8DE690E055
:109630000F941A9681110C941F6988E494E20F9498
:10964000FC2781E090E090932E0D80932D0D80916A
:10965000F00E882329F060E081E090E00F94EC00A8
:1096600083E50F94EB99882379F019810F94E2999F
:10967000111106C00F9479B3709361156093601552
:1096800081E08093040212C082E50F94EB99882355
:1096900069F019810F94E299111106C00F9479B302
:1096A0007093611560936015109204020F944E86BA
:1096B0004B015C01F9800F2D10E0F801EE0FFF1F48
:1096C000E05AFA4E60817181072E000C880B990BCD
:1096D0000F9434A9F801EE0FFF1FEE0FFF1FEB5898
:1096E000F04F11E020813181428153810F9465B4A4
:1096F00018160CF010E01093240D81E090E0909388
:109700002802809327021092D20E4F2DC501B4017A
:109710000E9452938AE394E20F94FC2782E090E047
:10972000909328028093270290932E0D80932D0D05
:109730008091F00E882329F060E082E090E00F94A1
:10974000EC000F944E8660936719709368198093AC
:10975000691990936A190C941F698EE294E20F9430
:10976000FC2783E090E090932E0D80932D0D809147
:10977000F00E882329F060E081E090E00F94EC0087
:1097800083E50F94EB99882361F00F94E2990F948D
:1097900079B370931F0D60931E0D81E080930402D6
:1097A0000FC082E50F94EB99882351F00F94E29952
:1097B0000F9479B370931F0D60931E0D10920402E5
:1097C0000F944E864B015C011092D20E60911E0DDB
:1097D00070911F0D072E000C880B990B0F9434A964
:1097E00011E0209114073091150740911607509110
:1097F00017070F9465B418160CF010E01093240DA1
:1098000081E090E090932802809327020AE31FE012
:10981000B6E3EB2EBFE0FB2E82E3C82E8FE0D82EFE
:109820008091240D60911E0D70911F0D8823B9F059
:109830008091D20E811113C0072E000C880B990B5A
:109840000F9434A920911407309115074091160701
:10985000509117070F9465B41816BCF08BC0072EF3
:10986000000C880B990B0F9434A9209114073091A8
:10987000150740911607509117070F942EA987FFDF
:1098800079C080910402811175C00F944E86DC016D
:10989000CB0188199909AA09BB09893E9340A10502
:1098A000B10508F45EC08091F00E811156C0E091C0
:1098B0001A0D24E0E29FF0011124EB58F04F408094
:1098C000518062807380F8018491AAE3AA2EAFE0F0
:1098D000BA2E882341F00E947DFAFFEFAF1ABF0A2B
:1098E000F5018491F6CF42E0C301B2010E9420FB52
:1098F000F7018491F6E3AF2EFFE0BF2E882341F0FD
:109900000E947DFAFFEFAF1ABF0AF5018491F6CFEE
:1099100060911A0D70E080E090E00E9406FBF60175
:109920008491E2E3AE2EEFE0BE2E882341F00E9448
:109930007DFAFFEFAF1ABF0AF5018491F6CF60916F
:10994000140770911507809116079091170741E051
:109950000E9420FB8AE00E947DFA0F944E864B0104
:109960005C010F94CD7980E00F940C8080E00E9420
:109970005CA556CF85E294E20F94FC2782E090E04C
:10998000909328028093270284E090E090932E0D1C
:1099900080932D0D0F944E8660936719709368190C
:1099A0008093691990936A190C941F6983E50F9449
:1099B000EB99882319F10F94E29920E030E0A90196
:1099C0000F942EA987FD0FC00F94E29920E030E09C
:1099D0004FE753E40F9465B4181644F00F94E299DE
:1099E0000F9479B305C060E070E002C06FEF70E0E3
:1099F0007093B0196093AF190C941F698FEF90E0CA
:109A00009093B0198093AF190C941F691092B019FC
:109A10001092AF190C941F690F94681A0F94AB7FC2
:109A2000149A0F9403801092B0191092AF1968EE37
:109A300073E080E090E00F9436858CE094E00F9422
:109A4000FC2780E00E945CA50C941F691092230EF5
:109A50000C941F6983E50F94EB99882399F00F9478
:109A6000E29920E030E04AE754E40F9426A40F94F2
:109A70007FB360938C0270938D0280938E029093DB
:109A80008F021DC088E50F94EB9981110C94376CFF
:109A900089E50F94EB9981110C94376C8AE50F944A
:109AA000EB9981110C94376C85E40F94EB9981113B
:109AB0000C94376C0F94AB7F149A0F9403808FEF44
:109AC0009FEF9093420280934102909340028093D3
:109AD0003F0280933E0280933D021092240E0C942C
:109AE0001F6983E50F94EB99882311F40C941F6987
:109AF0000F94E29920E030E04AE754E40F9426A462
:109B00000F947FB360936319709364198093651900
:109B1000909366190C941F6983E50F94EB99882341
:109B200011F40C941F690F94E29920E030E04AE7A9
:109B300054E40F9426A40F947FB36093880270932B
:109B4000890280938A0290938B0280E496E10F94BD
:109B5000405E0C941F6926E333E03BAF2AAF03E27B
:109B600010E175E4C72E7DE0D72EF12CAAADBBAD78
:109B70008D91BBAFAAAF0F94EB99882309F463C012
:109B8000B3E0FB1259C00F94E2992B013C0120E095
:109B900030E040EA51E40F942EA987FF45C0A301AD
:109BA0009201F80164817581868197810F9408B3D1
:109BB0004B015C019B01AC016091771070917810B2
:109BC0008091791090917A100F9426A46093771069
:109BD000709378108093791090937A1020904602B9
:109BE00030904702A5019401D1011C966D917D91A1
:109BF0008D919C911F970F9426A4F101648775871E
:109C000086879787D6016D917D918D919C910F9458
:109C100032A9A50194010F9426A40F947FB3F601F5
:109C20006083718382839383D80114964D925D92F1
:109C30006D927C92179707C00F94E299F8016483A4
:109C4000758386839783F3940C5F1F4FF4E0CF0EE8
:109C5000D11C64E0862EF81089CF0C941F698EE425
:109C60000F94EB99882311F40C941F690F94D799E2
:109C700060933F137093401380934113909342136A
:109C80000C941F6983E50F94EB99882379F08091F8
:109C90003D1390913E134AE050E060E070E0019681
:109CA0000F944EA660935A020C941F69E3E3FDE5FE
:109CB00084918F01882339F00E947DFA0F5F1F4F36
:109CC000F8018491F7CFC0905A02D12CE12CF12CED
:109CD000EBE2FFE084918F01882339F00E947DFA46
:109CE0000F5F1F4FF8018491F7CF4AE0C701B6011B
:109CF0000E9495FA8AE00E947DFA0C941F6986E51D
:109D00000F94EB99882379F0E7EAF5E584918F01C8
:109D1000882311F40C94C3450E947DFA0F5F1F4FF6
:109D2000F8018491F5CF85E50F94EB99382E8823BF
:109D3000D9F1E0903D13F0903E13FFEFEF1AFF0AC8
:109D4000F0923E13E0923D13270167014601D601D0
:109D50008D916D0190ED980F9A30C0F38E3211F015
:109D60000C941F695D013501F50181915F0190ED52
:109D7000980F9A30C0F38E3211F00C941F69CF0106
:109D80008C01DC012C90019620ED220D2A30C0F3CD
:109D9000822D0F94D22781110C94566CBDE22B12A8
:109DA0000C941F690C94566CEDE0FFE084918F01D8
:109DB000882339F00E947DFA0F5F1F4FF8018491CC
:109DC000F7CFE7EAF5E584918F01882339F00E9407
:109DD0007DFA0F5F1F4FF8018491F7CFE3EBFEE0B0
:109DE00084918F01882339F00E947DFA0F5F1F4F05
:109DF000F8018491F7CFEFEAFEE084918F01882388
:109E000039F00E947DFA0F5F1F4FF8018491F7CF60
:109E1000E0EAFEE084918F01882339F00E947DFA08
:109E20000F5F1F4FF8018491F7CFE3E9FEE08491C3
:109E30008F01882339F00E947DFA0F5F1F4FF801D0
:109E40008491F7CFE2E8FEE084918F01882339F016
:109E50000E947DFA0F5F1F4FF8018491F7CFE0E871
:109E6000FEE084918F01882339F00E947DFA0F5F14
:109E70001F4FF8018491F7CFE9E7FEE084918F014D
:109E8000882339F00E947DFA0F5F1F4FF8018491FB
:109E9000F7CFE4E5FEE084918F01882311F40C9460
:109EA000C3450E947DFA0F5F1F4FF8018491F5CFE3
:109EB000E7E0FDE084918F01882339F00E947DFA6C
:109EC0000F5F1F4FF8018491F7CF6091DF0F709102
:109ED000E00F8091E10F9091E20F42E00E9420FBA1
:109EE000E3E0FDE084918F01882339F00E947DFA40
:109EF0000F5F1F4FF8018491F7CF6091E30F7091CE
:109F0000E40F8091E50F9091E60F42E00E9420FB64
:109F1000EFEFFCE084918F01882339F00E947DFAF5
:109F20000F5F1F4FF8018491F7CF6091E70F709199
:109F3000E80F8091E90F9091EA0F42E00E9420FB28
:109F4000EBEFFCE084918F01882339F00E947DFAC9
:109F50000F5F1F4FF8018491F7CF6091EB0F709165
:109F6000EC0F8091ED0F9091EE0F42E00E9420FBEC
:109F7000ECE3F5E084918F01882339F00E947DFAAB
:109F80000F5F1F4FF8018491F7CF80E00F948A7F15
:109F90000F9434A920912710309128104091291056
:109FA00050912A100F9408B342E00E9420FBE7EF83
:109FB000FCE084918F01882339F00E947DFA0F5FC5
:109FC0001F4FF8018491F7CF81E00F948A7F0F949F
:109FD00034A920912B1030912C1040912D105091CC
:109FE0002E100F9408B342E00E9420FBE3EFFCE048
:109FF00084918F01882339F00E947DFA0F5F1F4FF3
:10A00000F8018491F7CF82E00F948A7F0F9434A9EE
:10A0100020912F103091301040913110509132101A
:10A020000F9408B342E00E9420FBEFEEFCE0849125
:10A030008F01882339F00E947DFA0F5F1F4FF801CE
:10A040008491F7CF83E00F948A7F0F9434A92091F5
:10A0500033103091341040913510509136100F94D8
:10A0600008B342E00E9420FB8AE00E947DFA0C9433
:10A070001F69109226020C941F6981E080932602CA
:10A080000C941F69882339F00E947DFA0F5F1F4FDF
:10A09000F8018491F7CF8AE00E947DFAE9EEF5E0BD
:10A0A00084918F01882339F00E947DFA0F5F1F4F42
:10A0B000F8018491F7CF1E9B0DC0EDECF2E1849185
:10A0C0008F018823A1F00E947DFA0F5F1F4FF801D6
:10A0D0008491F7CFE8ECF2E184918F01882339F085
:10A0E0000E947DFA0F5F1F4FF8018491F7CF8AE03D
:10A0F0000E947DFAE1EEF5E084918F01882339F02A
:10A100000E947DFA0F5F1F4FF8018491F7CF809175
:10A11000060182FF0DC0EDECF2E184918F018823EE
:10A12000A1F00E947DFA0F5F1F4FF8018491F7CFD5
:10A13000E8ECF2E184918F01882339F00E947DFAE6
:10A140000F5F1F4FF8018491F7CF8AE00E947DFADC
:10A15000E9EDF5E084918F01882339F00E947DFAC2
:10A160000F5F1F4FF8018491F7CF1D9B0DC0EDECE1
:10A17000F2E184918F018823A1F00E947DFA0F5FA4
:10A180001F4FF8018491F7CFE8ECF2E184918F0141
:10A19000882339F00E947DFA0F5F1F4FF8018491E8
:10A1A000F7CF8AE00E947DFAE1EDF5E084918F011E
:10A1B000882339F00E947DFA0F5F1F4FF8018491C8
:10A1C000F7CF8091060187FF0DC0EDECF2E184919D
:10A1D0008F018823A1F00E947DFA0F5F1F4FF801C5
:10A1E0008491F7CFE8ECF2E184918F01882339F074
:10A1F0000E947DFA0F5F1F4FF8018491F7CF8AE02C
:10A200000E947DFAE9ECF5E084918F01882339F012
:10A210000E947DFA0F5F1F4FF8018491F7CF1C9BBE
:10A220000DC0EDECF2E184918F018823A1F00E9432
:10A230007DFA0F5F1F4FF8018491F7CFE8ECF2E150
:10A2400084918F01882339F00E947DFA0F5F1F4FA0
:10A25000F8018491F7CF8AE00E947DFAE1ECF5E005
:10A2600084918F01882339F00E947DFA0F5F1F4F80
:10A27000F8018491F7CF01990FC0EDECF2E18491E0
:10A280008F01882311F40C94C3450E947DFA0F5F5F
:10A290001F4FF8018491F5CFE8ECF2E184918F0132
:10A2A000882311F40C94C3450E947DFA0F5F1F4F61
:10A2B000F8018491F5CF10911A0D84E50F94EB9974
:10A2C000882301F10F94E2990F947FB3162F662330
:10A2D000C9F0E3E3FDE584918F01882339F00E9402
:10A2E0007DFA0F5F1F4FF8018491F7CF01EB12E168
:10A2F000D8018D918D01882311F40C941F690E945F
:10A300007DFAF6CF84E40F94EB99882311F40C9432
:10A310001F690F94E29920E030E0A9010F942EA963
:10A32000811103C01092BA102EC00F94E299B4E0CC
:10A330001B9FF0011124E554FF4E608371838283DB
:10A340009383C090BB10D090BC10E090BD10F090F3
:10A35000BE1020E030E0A901C701B6010F942EA97C
:10A36000811106C0C12CD12C50EEE52E5FE3F52EF5
:10A37000C092BB10D092BC10E092BD10F092BE1003
:10A3800081E08093BA100E94C8940C941F69F70171
:10A3900081917F010F94EB998823A1F10F94E299A9
:10A3A0000F947FB3F1E0FD15ACF0653C29E0720736
:10A3B00081059105A0F4562F472F382F292F613C96
:10A3C000A3E07A078105910590F050EC43E030E07E
:10A3D00020E00DC0562F472F382F292F08C050ECF2
:10A3E00043E030E020E064EC79E080E090E0F801C8
:10A3F00064A375A386A397A3E455FF4F50834183BD
:10A4000032832383D3940C5F1F4FF4E0DF12BFCF5E
:10A410000E9425BA0C941F6926E3A22E23E0B22ED7
:10A4200033E2C32E30E1D32E912CD5018D915D0105
:10A430000F94EB99882309F43EC00F94E2997B01B5
:10A440008C01B1E0B91514F120E030E048E453E4A8
:10A450000F9465B418163CF4512C612C88E4782EC6
:10A4600093E4892E04C05E2C6F2C702E812E20E088
:10A4700030E048EC52E4B701C8010F9465B41816F7
:10A480004CF4E12CF12C08EC12E404C0562E6F2C95
:10A49000782E812E852D962DA72DB82DF601848B33
:10A4A000958BA68BB78BC701D801E456FF4F8083ED
:10A4B0009183A283B3839394F4E0CF0ED11C14E074
:10A4C000812E9810B2CF0C941F6983E50F94EB99FD
:10A4D0008823E9F00F94E299609357107093581015
:10A4E0008093591090935A1084E50F94EB99882328
:10A4F00011F40C941F690F94E29960935B107093B0
:10A500005C1080935D1090935E100C941F6980E541
:10A510000F94EB99882351F00F94E29960935710B0
:10A52000709358108093591090935A1082E50F94AD
:10A53000EB99882351F00F94E29960935B1070932C
:10A540005C1080935D1090935E1084E50F94EB99FE
:10A550000C941F6983E50F94EB99882351F00F94B5
:10A56000E29960935F1070936010809361109093F4
:10A57000621084E50F94EB99882351F00F94E299CF
:10A5800060936310709364108093651090936610CD
:10A5900082E40F94EB99882361F00F94E2990F9471
:10A5A0007FB36093671070936810809369109093E5
:10A5B0006A1088E50F94EB99882391F00F94E29943
:10A5C00060936F107093701080937110909372105D
:10A5D00060936B1070936C1080936D1090936E105D
:10A5E00089E50F94EB99882351F00F94E2996093D9
:10A5F0006F107093701080937110909372108AE5B1
:10A600000F94EB99882351F00F94E29960937310A3
:10A6100070937410809375109093761085E40F9466
:10A62000EB99882351F00F94E2996093771070931F
:10A6300078108093791090937A1020E030E040E217
:10A6400051E460916B1070916C1080916D1090913D
:10A650006E100F9465B4181664F480E090E0A0E2E8
:10A66000B1E480936B1090936C10A0936D10B09335
:10A670006E1020E030E040E251E460916F10709184
:10A68000701080917110909172100F9465B418162B
:10A6900014F00C941F6980E090E0A0E2B1E4809394
:10A6A0006F1090937010A0937110B09372100C946F
:10A6B0001F69A6E3EA2EA3E0FA2E0BE710E1B7E844
:10A6C000CB2EB0E1DB2ED7018D917D010F94EB995C
:10A6D000882339F00F94E299F801608371838283B3
:10A6E00093830C5F1F4FC016D10669F70C941F6946
:10A6F00083E50F94EB99882351F00F94E2996093CE
:10A70000A6107093A7108093A8109093A91086E4C8
:10A710000F94EB99882381F00F94E29920E030E0C8
:10A7200040E752E40F9408B36093AA107093AB1003
:10A730008093AC109093AD108AE50F94EB99882329
:10A7400011F40C941F690F94E2996093AE1070930A
:10A75000AF108093B0109093B1100C941F6983E5F3
:10A760000F94EB99882351F00F94E2996093B21003
:10A770007093B3108093B4109093B51086E40F9447
:10A78000EB99882311F40C941F690F94E29920E04F
:10A7900030E040E752E40F9408B36093B610709332
:10A7A000B7108093B8109093B9100C941F6983E58B
:10A7B0000F94EB99882311F40C941F690F94E2997C
:10A7C0000F9479B36115710551F06130710569F429
:10A7D00081E08093A5101092F10E0C941F691092E5
:10A7E000A5101092F10E0C941F69E3E3FDE584912E
:10A7F0008F01882339F00E947DFA0F5F1F4FF80107
:10A800008491F7CFEEEAF5E084918F01882339F047
:10A810000E947DFA0F5F1F4FF8018491F7CF0091DE
:10A820005E1510915F150C581C4ED8018D918D014D
:10A83000882319F00E947DFAF8CFEFE4FEE08491BE
:10A840008F01882311F40C94C3450E947DFA0F5F99
:10A850001F4FF8018491F5CF83E50F94EB9988237E
:10A8600011F40C941F690F94E2990F9479B37093CB
:10A87000600260935F020C941F6983E50F94EB996B
:10A88000882309F480CD0F94E2990F9479B36B017A
:10A890007C0184E50F94EB99882359F0BE016F5F2A
:10A8A0007F4F8DED90E00F941A9681110C941F69E3
:10A8B0006ACDD0926302C092620265CD80E50F94AA
:10A8C000EB99882311F40C941F690F94E2990F946B
:10A8D00079B3D62E862F972F7C0183E50F94EB99C1
:10A8E000882331F00F94E2990F9479B38B0102C061
:10A8F0000FEF1FEFC8010196039710F00C941F692A
:10A90000E5E9F2E08DEC92E021913191E216F30657
:10A9100011F40C941F698E179F07B1F7F7FE02C060
:10A920000C941F690F94AB7FFD2C60E08D2D0F946C
:10A9300033840F3FFFEF1F0731F00130110571F431
:10A9400001E010E00DC08D2D0F94FAA331E020E05E
:10A95000892B09F030E0032F122F02C000E010E035
:10A960008F2D0F94FAA38017910711F40C941F698F
:10A970000F94CD7980E00F940C8080E00E945CA55C
:10A98000EFCF83E50F94EB99882331F00F94E29990
:10A990000F9479B38B0102C00EE610E080E50F94AE
:10A9A000EB99882329F00F94E2990F9479B302C0B0
:10A9B00068EE73E06B01770FEE08FF0810161106C2
:10A9C00094F480910D0790910E07029718F4C80136
:10A9D0000F94DC46C701B6010F94368584E50F94C9
:10A9E00060230C941F69C701B6010F9436850C943F
:10A9F0001F6980E50F94EB99882351F00F94E29939
:10AA000060938B1070938C1080938D1090938E10A8
:10AA100089E40F94EB99882381F00F94E2992CEA52
:10AA200035EC47E25EE30F9426A460938F10709399
:10AA30009010809391109093921084E40F94EB996E
:10AA4000882381F00F94E2992CEA35EC47E25EE32B
:10AA50000F9408B3609393107093941080939510A3
:10AA60009093961083E40F94EB99882351F00F9400
:10AA7000E299609300027093010280930202909326
:10AA800003020F94627EE5E8F7E184918F01882349
:10AA900039F00E947DFA0F5F1F4FF8018491F7CFC4
:10AAA00009E114E0D8018D918D01882319F00E94ED
:10AAB0007DFAF8CF60918B1070918C1080918D1081
:10AAC00090918E1042E00E9420FB0DE114E0F8010D
:10AAD00081918F01882319F00E947DFAF8CF2CEA2A
:10AAE00035EC47E25EE360918F1070919010809199
:10AAF0009110909192100F9408B342E00E9420FBB5
:10AB000001E214E0D8018D918D01882319F00E9493
:10AB10007DFAF8CF2CEA35EC47E25EE360919310C2
:10AB20007091941080919510909196100F9426A496
:10AB300042E00E9420FB05E214E0F80181918F01C0
:10AB4000882319F00E947DFAF8CF6091000270917D
:10AB50000102809102029091030242E00E9420FBD8
:10AB60008AE00E947DFA0C941F6980E50F94EB99AE
:10AB7000882351F00F94E299609397107093981086
:10AB80008093991090939A1089E40F94EB998823FD
:10AB900081F00F94E2992CEA35EC47E25EE30F94E2
:10ABA00026A460939B1070939C1080939D109093AB
:10ABB0009E1084E40F94EB99882381F00F94E2991E
:10ABC0002CEA35EC47E25EE30F9408B360939F10E4
:10ABD0007093A0108093A1109093A2100F94627EA6
:10ABE000E5E8F7E184918F01882339F00E947DFA2E
:10ABF0000F5F1F4FF8018491F7CF09E114E0D801EE
:10AC00008D918D01882319F00E947DFAF8CF609113
:10AC10009710709198108091991090919A1042E03D
:10AC20000E9420FB0DE114E0F80181918F0188233F
:10AC300019F00E947DFAF8CF2CEA35EC47E25EE38A
:10AC400060919B1070919C1080919D1090919E102E
:10AC50000F9408B342E00E9420FB01E214E0D80107
:10AC60008D918D01882319F00E947DFAF8CF2CEA8E
:10AC700035EC47E25EE360919F107091A0108091E7
:10AC8000A1109091A2100F9426A442E00E9420FBF4
:10AC90008AE00E947DFA0C941F6983E50F94EB997A
:10ACA000882319F00F94E29903C060E070E0CB01B3
:10ACB0006093690270936A0280936B0290936C02B6
:10ACC0000C941F6985E40F94EB99882359F00F9435
:10ACD000E2990F9479B324967FAF6EAF249777FFF4
:10ACE00005C013C024961FAE1EAE249763961FAEF8
:10ACF000639764961FAE649726E166962FAF6697BA
:10AD000033E468963FAF68970EC063961FAE6397B3
:10AD100064961FAE64974CE866964FAF669752E410
:10AD200068965FAF689783E50F94EB99882371F07D
:10AD30000F94E29963966FAF639764967FAF6497C1
:10AD400066968FAF669768969FAF689783E40F9477
:10AD5000EB99882349F00F94E2990F9479B3A79661
:10AD60007FAF6EAFA79706C085E090E0A7969FAF34
:10AD70008EAFA797A7968EAC9FACA79790922A0DFF
:10AD80008092290D10925E0E10922C0D10922B0DB8
:10AD90000F944E8662966CAF7DAF8EAF9FAF629779
:10ADA0002496AEACBFAC2497B7FC05C02AE0A896A9
:10ADB0002FAFA89704C03DE2A8963FAFA8970F9485
:10ADC0004E86E4966CAF7DAF8EAF9FAFE49724962E
:10ADD0008EAC9FAC249718141904B4F409E214E063
:10ADE000D8018D918D01882319F00E947DFAF8CF4A
:10ADF0008AE00E947DFA81E080935E0E10922C0D15
:10AE000010922B0D0C941F6903E514E0F801819159
:10AE10008F01882319F00E947DFAF8CF8AE00E9402
:10AE20007DFA0F94681A24968EAC9FAC24978FE716
:10AE3000892809F451C08093080F62968CAC9DACB0
:10AE4000AEACBFAC62976D968CAE9DAEAEAEBFAEF3
:10AE50006D97E0968CAE9DAEAEAEBFAEE0972B96F2
:10AE60001FAE2B976E961FAE6E9720E46F962FAF96
:10AE70006F973CE1A0963FAFA09746E4A1964FAFF5
:10AE8000A197A2961FAEA297A3961FAEA397A496D2
:10AE90001FAEA497A5961FAEA597EFE78E2E912C17
:10AEA000A12CB12C2A968CAE9DAEAEAEBFAE2A9729
:10AEB000FFE74F2E512C612C712CAC961CAE1DAEB1
:10AEC0001EAE1FAEAC9721E0E9962FAFE9971AAE00
:10AED0001EAE212C312C06C08093090FAECF80E02E
:10AEE0000E945CA5A89580910A0F882309F474C17B
:10AEF0000F94842124968EAC9FAC2497892859F412
:10AF00009090750F9AAEA090760FAEAE2090770F0E
:10AF10003090780F0AC0B0901407BAAE8090150731
:10AF20008EAE20901607309017072AAD3EADA101D6
:10AF3000A2966FADA297A3967FADA397A4968FAD6F
:10AF4000A497A5969FADA5970F9465B4181674F0B5
:10AF50009AACA2969FAEA297AEACA396AFAEA397C3
:10AF6000A4962FAEA497A5963FAEA5976E962FAD4B
:10AF70006E976F963FAD6F97A0964FADA097A19635
:10AF80005FADA1976AAD7EADC1010F9465B418168F
:10AF900074F0BAAC6E96BFAE6E978EAC6F968FAEF5
:10AFA0006F97A0962FAEA097A1963FAEA1970F9452
:10AFB0004E86DC01CB01E4968CAC9DACAEACBFAC54
:10AFC000E49788199909AA09BB09853C9940A1050C
:10AFD000B10550F00F94AB790F944E86E4966CAFA8
:10AFE0007DAF8EAF9FAFE497E9968FACE99788204D
:10AFF00009F474C02AAD3EADA10163966FAD6397AD
:10B0000064967FAD649766968FAD669768969FADA0
:10B0100068970F942EA987FFDFC00F944E86DC013E
:10B02000CB0162968CAC9DACAEACBFAC629788197C
:10B030009909AA09BB0989389341A105B10508F40A
:10B04000CBC0D301C2012A968CAC9DACAEACBFACD8
:10B050002A9788199909AA09BB092496AEACBFACF6
:10B060002497B595A79597958795AB2819F0809368
:10B07000080F02C08093090F0F944E866D966CAF37
:10B080007DAF8EAF9FAF6D974B015C0162962CAD8B
:10B090003DAD4EAD5FAD6297821A930AA40AB50A20
:10B0A000AC968CAE9DAEAEAEBFAEAC9763968FAC99
:10B0B0006397A2968FAEA29764969FAC6497A3966F
:10B0C0009FAEA3976696AFAC6697A496AFAEA497D3
:10B0D0006896BFAC6897A596BFAEA5972AAD3EAD62
:10B0E000A10163966FAD639764967FAD6497669692
:10B0F0008FAD669768969FAD68970F9465B41816E4
:10B1000014F00C94546F0F944E86DC01CB016D96B5
:10B110008CAC9DACAEACBFAC6D9788199909AA09EF
:10B12000BB0989389341A105B10510F40C94546F03
:10B130000F944E8662966CAF7DAF8EAF9FAF6297D5
:10B14000DC01CB0188199909AA09BB0920912B0DB3
:10B1500030912C0D1216130614F40C947F6D2A9660
:10B160008CAD9DADAEADBFAD2A97840D951DA61DCE
:10B17000B71D24968EAC9FAC2497B595A79597954F
:10B180008795892811F40C94506F8093080F809153
:10B190002B0D90912C0D019690932C0D80932B0DDF
:10B1A00063969FAC63976E969FAE6E976496AFACB6
:10B1B00064976F96AFAE6F976696BFAC6697A09692
:10B1C000BFAEA09768968FAC6897A1968FAEA197F7
:10B1D00021E0E9962FAFE99720E030E040EA51E422
:10B1E00063966FAD639764967FAD649766968FADF7
:10B1F000669768969FAD68970F941AB22AAD3EADD8
:10B20000A1010F942EA987FF0EC0EEE7FCE0849108
:10B210008F01882309F4ECCD0E947DFA0F5F1F4F48
:10B22000F8018491F6CF0F944E86DC01CB01E096B5
:10B230008CAC9DACAEACBFACE09788199909AA095B
:10B24000BB09813D9740A105B10508F4B4C024961F
:10B250008EAC9FAC2497892881F0E090080FF12CE8
:10B26000EBE7FCE084918F018823B9F00E947DFA1E
:10B270000F5F1F4FF8018491F7CFE090090FF12C79
:10B28000E8E7FCE084918F01882339F00E947DFA81
:10B290000F5F1F4FF8018491F7CF42E06AAD7EAD9A
:10B2A000C1010E9420FBE4E7FCE084918F01882328
:10B2B00039F00E947DFA0F5F1F4FF8018491F7CF9C
:10B2C000B701FF0C880B990B0E9406FB8AE00E94D5
:10B2D0007DFA2B968FAC2B97882009F452C0A89644
:10B2E0009FACA897891418F4282D2F5F59C02B966E
:10B2F0008FAC2B97A8969FACA897891054C0282D87
:10B300002F5F2B962FAF2B97E5962FADE597E696FF
:10B310003FADE697E7964FADE797E8965FADE897C4
:10B320006AAD7EADC1010F9419B26B017C0120E0C2
:10B3300030E0A9010F9465B418165CF420E030E009
:10B3400040EA50E4C701B6010F942EA987FF2BC035
:10B350000AC020E030E040EA50ECC701B6010F948B
:10B3600065B4181604F524966FAD2497661F6627FA
:10B37000661F80E00F94931D81E080935E0E0C9415
:10B380001F698AACE5968FAEE5979EACE6969FAEB8
:10B39000E697E7962FAEE797E8963FAEE89721E06D
:10B3A0002B962FAF2B970F944E86E0966CAF7DAF08
:10B3B0008EAF9FAFE0970F944E866B017C010F9488
:10B3C0004E866D960CAD1DAD2EAD3FAD6D97629660
:10B3D0008CAC9DACAEACBFAC6297080D191D2A1D9C
:10B3E0003B1DC01AD10AE20AF30ADC01CB018C0D25
:10B3F0009D1DAE1DBF1D81389F44A241B10570F057
:10B40000E7E5FCE084918F01882309F4F1CC0E94E8
:10B410007DFA0F5F1F4FF8018491F6CF80912B0DBD
:10B4200090912C0DA7968EAC9FACA7978816990685
:10B430000CF055CDEBEFFBE084918F01882309F4EC
:10B44000D7CC0E947DFA0F5F1F4FF8018491F6CF91
:10B450000F94AB7F0C941F6980915213882311F4D1
:10B460000C941F6985E40F94EB99882331F00F94B5
:10B47000E2990F947FB3162F01C01FEF86E40F945B
:10B48000EB99882331F00F94E2990F947FB3062F44
:10B4900001C00FEF1F920F931F921F938AEE9BE044
:10B4A0009F938F930F949AA81F920F931F921F93AD
:10B4B00082EE9BE09F938F930E9471D90FB6F89410
:10B4C000DEBF0FBECDBF1AE00E9465D9181614F476
:10B4D0000C941F69115011F00C94596F0C941F6952
:10B4E0000E94A0FD0C941F690E942FFC0C941F6900
:10B4F000809186108F93809185108F938091841016
:10B500008F93809183108F93809182108F9380917D
:10B5100081108F93809180108F9380917F108F93F3
:10B5200080917E108F9380917D108F9380917C10FD
:10B530008F9380917B108F9303E31DE51F930F93EF
:10B540001F930F9380917A108F93809179108F932E
:10B55000809178108F93809177108F9380917610DF
:10B560008F93809175108F93809174108F93809139
:10B5700073108F93809172108F93809171108F93BD
:10B58000809170108F9380916F108F9380916E10C7
:10B590008F9380916D108F9380916C108F93809119
:10B5A0006B108F9380916A108F93809169108F93A5
:10B5B000809168108F93809167108F9380916610AF
:10B5C0008F93809165108F93809164108F938091F9
:10B5D00063108F93809162108F93809161108F938D
:10B5E000809160108F9380915F108F931F930F93C2
:10B5F0001F930F9380915E108F9380915D108F93B6
:10B6000080915C108F9380915B108F9380915A1082
:10B610008F93809159108F93809158108F938091C0
:10B6200057108F931F930F931F930F938091DE10EA
:10B630008F938091DD108F938091DC108F93809198
:10B64000DB108F938091DA108F938091D9108F93B4
:10B650008091D8108F938091D7108F938091D610BE
:10B660008F938091D5108F938091D4108F93809178
:10B67000D3108F938091D2108F938091D1108F939C
:10B680008091D0108F938091CF108F931F930F9341
:10B690001F930F93809156108F93809155108F9325
:10B6A000809154108F93809153108F9380915210FA
:10B6B0008F93809151108F93809150108F93809130
:10B6C0004F108F9380914E108F9380914D108F93D8
:10B6D00080914C108F9380914B108F9380914A10E2
:10B6E0008F93809149108F93809148108F93809110
:10B6F00047108F931F930F931F930F938091CE103A
:10B700008F938091CD108F938091CC108F938091E7
:10B71000CB108F938091CA108F938091C9108F9313
:10B720008091C8108F938091C7108F938091C6101D
:10B730008F938091C5108F938091C4108F938091C7
:10B74000C3108F938091C2108F938091C1108F93FB
:10B750008091C0108F938091BF108F931F930F9390
:10B760001F930F93809146108F93809145108F9374
:10B77000809144108F93809143108F938091421059
:10B780008F93809141108F93809140108F9380917F
:10B790003F108F9380913E108F9380913D108F9337
:10B7A00080913C108F9380913B108F9380913A1041
:10B7B0008F93809139108F93809138108F9380915F
:10B7C00037108F931F930F931F930F938091361011
:10B7D0008F93809135108F93809134108F93809147
:10B7E00033108F93809132108F93809131108F930B
:10B7F000809130108F9380912F108F9380912E1015
:10B800008F9380912D108F9380912C108F93809126
:10B810002B108F9380912A108F93809129108F93F2
:10B82000809128108F93809127108F931F930F93EF
:10B830001F930F9382E399E09F938F930F949AA89D
:10B840000FB6F894DEBF0FBECDBF2CEA35EC47E251
:10B850005EE3609193107091941080919510909197
:10B8600096100F9426A49F938F937F936F932CEA47
:10B8700035EC47E25EE360918F10709190108091FB
:10B880009110909192100F9408B39F938F937F9390
:10B890006F9380918E108F9380918D108F938091F4
:10B8A0008C108F9380918B108F931F930F931F9306
:10B8B0000F9385E099E09F938F930F949AA82CEAB9
:10B8C00035EC47E25EE360919F107091A01080918B
:10B8D000A1109091A2100F9426A49F938F937F9311
:10B8E0006F932CEA35EC47E25EE360919B10709118
:10B8F0009C1080919D1090919E100F9408B39F937F
:10B900008F937F936F9380919A108F93809199106A
:10B910008F93809198108F93809197108F931F939E
:10B920000F931F930F9380ED98E09F938F930F9445
:10B930009AA80FB6F894DEBF0FBECDBF8091A510B8
:10B940001F928F931F930F931F930F9320E030E06C
:10B9500040E752E46091B6107091B7108091B81032
:10B960009091B9100F9426A49F938F937F936F9318
:10B970008091B5108F938091B4108F938091B31004
:10B980008F938091B2108F931F930F931F930F93F8
:10B990008091B1108F938091B0108F938091AF10F0
:10B9A0008F938091AE108F9320E030E040E752E417
:10B9B0006091AA107091AB108091AC109091AD1075
:10B9C0000F9426A49F938F937F936F938091A910D8
:10B9D0008F938091A8108F938091A7108F9380915F
:10B9E000A6108F931F930F931F930F938FEC97E0E5
:10B9F0009F938F930F949AA80FB6F894DEBF0FBE53
:10BA0000CDBF8091BA108823E9F08091BE108F934A
:10BA10008091BD108F938091BC108F938091BB104B
:10BA20008F931F930F931F930F9389EA97E09F9330
:10BA30008F930F949AA80FB6F894DEBF0FBECDBFB8
:10BA40000C941F691F930F938AE897E09F938F933D
:10BA50000F949AA80F900F900F900F900C941F695D
:10BA6000882339F00E947DFA0F5F1F4FF8018491FF
:10BA7000F7CFEFE3FEE084918F01882311F40C945B
:10BA80001F690E947DFA0F5F1F4FF8018491F5CF67
:10BA90008AE50F94EB99882309F489C00F94E29901
:10BAA0006B017C0120E030E040E751EC0F9465B47D
:10BAB00087FD38C020E030E040EA50ECC701B60115
:10BAC0000F942EA9181674F1F7FAF094F7F8F09481
:10BAD000C0928710D0928810E0928910F0928A105C
:10BAE000E3E3FDE584918F01882339F00E947DFA1C
:10BAF0000F5F1F4FF8018491F7CFE5EAF5E08491DD
:10BB00008F01882339F00E947DFA0F5F1F4FF801E3
:10BB10008491F7CF8AE00E947DFA8AE00E947DFA44
:10BB20000C941F69E3E3FDE584918F01882339F0CC
:10BB30000E947DFA0F5F1F4FF8018491F7CFE5EA6D
:10BB4000F5E084918F01882339F00E947DFA0F5F20
:10BB50001F4FF8018491F7CFE9ECF5E084918F0154
:10BB6000882339F00E947DFA0F5F1F4FF8018491FE
:10BB7000F7CF61EF7FEF8FEF9FEF0E9406FBE1ECC5
:10BB8000F5E084918F01882339F00E947DFA0F5FE0
:10BB90001F4FF8018491F7CF6BEF7FEF8FEF9FEF8F
:10BBA0000E9406FB8AE00E947DFA0C941F69E3E381
:10BBB000FDE584918F01882339F00E947DFA0F5FA3
:10BBC0001F4FF8018491F7CFE5EAF5E084918F01EA
:10BBD000882339F00E947DFA0F5F1F4FF80184918E
:10BBE000F7CF8AE00E947DFA8091871090918810AB
:10BBF000A0918910B0918A10BC01CD01905842E00B
:10BC00000E9420FB8AE00E947DFA0C941F690F9429
:10BC1000AB7F85E40F94EB99882329F00F94E29988
:10BC20006B017C0105C0C12CD12CE12C80ECF82EDD
:10BC30008CE40F94EB9981110F94E2998AE50F94AB
:10BC4000EB99882329F00F94E2992B013C011CC049
:10BC500020E030E048EC51E46091E70F7091E80F8C
:10BC60008091E90F9091EA0F0F942EA987FF07C0EA
:10BC7000412C512C08ED602E01E4702E05C0412CA2
:10BC8000512C612C10E4712E88E50F94EB998823D8
:10BC900049F00F94E29922966CAF7DAF8EAF9FAFC3
:10BCA00022970CC0812C912CB3E5AB2EB3E4BB2EB4
:10BCB00022968CAE9DAEAEAEBFAE229789E50F94B4
:10BCC000EB99882349F00F94E29926966CAF7DAFEB
:10BCD0008EAF9FAF269706C026961CAE1DAE1EAE39
:10BCE0001FAE269780915213882311F40C945F6F36
:10BCF00086E694E00E94B3F4882311F40C945F6FFD
:10BD000021E02AAF0F94AB7F8091F00E882329F0B9
:10BD100060E086E190E00F94EC0030915F02639662
:10BD20003FAF63974091600264964FAF6497E09194
:10BD30001A0DF0E0EE0FFF1FE05AFA4E808191815C
:10BD400067969FAF8EAF6797A091AF19B091B0196A
:10BD50006996BFAFAEAF69978090DF0F9090E00F0C
:10BD6000A090E10FB090E20F2A968CAE9DAEAEAEE1
:10BD7000BFAE2A9789829A82AB82BC822091E30F60
:10BD80003091E40F4091E50F5091E60F2E962CAFC5
:10BD90003DAF4EAF5FAF2E972D833E834F835887C5
:10BDA0008091E70F9091E80FA091E90FB091EA0F11
:10BDB00062968CAF9DAFAEAFBFAF629789879A870F
:10BDC000AB87BC872091EB0F3091EC0F4091ED0FCA
:10BDD0005091EE0F2D873E874F87588BC701B601D4
:10BDE0000F941AB26093EB0F7093EC0F8093ED0FEA
:10BDF0009093EE0F6AE1262E6DE0362E3F922F9241
:10BE0000812C912C78EEA72E72E4B72EEBEECE2E7D
:10BE1000EFE0DE2E6296ECACFDAC0EAD1FAD62978E
:10BE20002E962CAD3DAD4EAD5FAD2E972A966CADE6
:10BE30007DAD8EAD9FAD2A970F94C52E0F94AB7F2D
:10BE40002091E70F3091E80F4091E90F5091EA0FF0
:10BE5000C301B2010F941AB27B018C016093E70F0A
:10BE60007093E80F8093E90F9093EA0F2091E30F0E
:10BE70003091E40F4091E50F5091E60F6091DF0F94
:10BE80007091E00F8091E10F9091E20F3F922F921D
:10BE9000812C912CF0E7AF2EF1E4BF2E0F94C52E2C
:10BEA0000F94AB7F22968CAC9DACAEACBFAC22970E
:10BEB0008092DF0F9092E00FA092E10FB092E20F1C
:10BEC00026962CAD3DAD4EAD5FAD26972093E30F8A
:10BED0003093E40F4093E50F5093E60FE090E70FA7
:10BEE000F090E80F0091E90F1091EA0F3F922F9226
:10BEF000812C912CA8E4AA2EA2E4BA2E26962CAD71
:10BF00003DAD4EAD5FAD269722966CAD7DAD8EAD4D
:10BF10009FAD22970F94C52E0F94AB7F0F900F907B
:10BF20000F900F900F900F9080915213811124C0A9
:10BF300084E090E090932802809327020F944E862D
:10BF40004B015C0185EA90E10F948F04CC24C394EB
:10BF5000D12CE12CF12CD1100C94A36F0E9434A6AB
:10BF6000882311F40C94A36F9FB7F8948091020179
:10BF70008B7F809302019FBF1092B4068091521371
:10BF8000882319F00E9472D802C00E944FCE0F94ED
:10BF9000AB7F80915213811117C084E090E09093A1
:10BFA00028028093270241E060E088EE91E10F943F
:10BFB0009C048093B406811104C088EB91E10F9436
:10BFC000790581E00E9463AD80915213882309F4C2
:10BFD0007AC0AAADA11173C08091B70E882329F051
:10BFE00060E08091270D0E948AD784E090E09093D2
:10BFF0002802809327028EEC90E10F948F04FF2497
:10C00000F39400E010E00E9434A6811139C00F942F
:10C01000CD7981E00F940C80043FB1E01B0711F44F
:10C0200000E010E08091010184608093010101151E
:10C030001105A1F480910D0790910E07009721F052
:10C040000197B9F4FF20A9F09FB7F89480910201FD
:10C050008460809302019FBFF12C0BC00431110555
:10C0600041F49FB7F894809102018B7F8093020185
:10C070009FBF0F5F1F4F84E090E00E94A594C3CF45
:10C080009FB7F894809102018B7F809302019FBF3C
:10C090008091B70E882399F00E9459AD62E080E04C
:10C0A0000E94AAA885E692E40E94D1A780E6809328
:10C0B000260E1092250E60E080E00E943ED58AADEB
:10C0C0000F941D986FC00E9459AD61E080E00E94FE
:10C0D000AAA887E291E10E94D1A762E080E00E94D5
:10C0E000AAA884E191E10E94D1A784E090E0909316
:10C0F0002802809327020F9498530E9434A681113E
:10C100001AC00F94CD7981E00F940C800F94DF5307
:10C11000882399F380910D0790910E07029720F4E0
:10C1200088EE93E00F94DC4682E390E00E94A594B1
:10C1300084E50F9460230F94455282E090E0909341
:10C1400028028093270286E40F9406520F94DF980A
:10C1500080910D0790910E07029720F484EF91E0F3
:10C160000F94DC4682E390E00E94A59484E50F944E
:10C1700060230F9494510F943550811110C041E009
:10C1800060E087E391E10F949C04182F81E00E9406
:10C1900063AD82E00E945CA511110F945F5280E0B4
:10C1A0000E9463ADEAADE1114AC11092B406F4E019
:10C1B0002F2E312CA2E04A2E512CBAE16B2EBDE07D
:10C1C0007B2E8091B406813009F439C11092B406F7
:10C1D00030922802209227020E9459AD60E080E050
:10C1E0000E94AAA887E891E10E94D1A761E081E0BE
:10C1F0000E94AAA888EF9CE40E94D1A762E081E097
:10C200000E94AAA883E791E10E94D1A763E081E0A0
:10C210000E94AAA881E691E10E94D1A761E080E096
:10C220000E94AAA88BE694E00E944CA7E090B11966
:10C230000E2C000CFF0801E010E08091B406811183
:10C2400068C00F94CD7981E00F940C808091B11972
:10C25000082E000C990B9701281B390B37FF03C0E0
:10C26000319521953109253031050CF444C08E15E6
:10C270009F0514F401501109E816F90634F40F5F14
:10C280001F4F0430110564F009C00430110534F467
:10C290000115110529F401E010E002C003E010E0EF
:10C2A00061E080E00E94AAA889E695E00E944CA780
:10C2B00062E080E00E94AAA889E695E00E944CA76F
:10C2C00063E080E00E94AAA889E695E00E944CA75E
:10C2D000602F80E00E94AAA88BE694E00E944CA701
:10C2E000E090B1190E2C000CFF0864E670E080E0CD
:10C2F00090E00F9436850E9434A6882309F49DCFE0
:10C300000093B40664EF71E080E090E00F9436850E
:10C3100094CF0E9459AD0F94B38850922802409256
:10C3200027028091B406823009F454C0833009F0AA
:10C330007BC020E030E048E452E46091EB0F709164
:10C34000EC0F8091ED0F9091EE0F0F941AB2609365
:10C35000EB0F7093EC0F8093ED0F9093EE0FE09046
:10C36000E70FF090E80F0091E90F1091EA0F20918C
:10C37000E30F3091E40F4091E50F5091E60F60918B
:10C38000DF0F7091E00F8091E10F9091E20F7F92AB
:10C390006F92812C912CA12CB0E4BB2EEBEECE2E13
:10C3A000EFE0DE2E0F94C52E0E9459AD60E080E0D4
:10C3B0000E94AAA88AE991E10E94D1A762E080E0E8
:10C3C0000E94AAA885E692E40E94D1A70F900F9040
:10C3D00010E01EC080915213882321F080E00F945A
:10C3E0001D98EFCE0F94DF98ECCE0F94CD7981E0BD
:10C3F0000F940C8065E570E080E090E00F94368546
:10C40000F1E0EF1AF10889F71F5F143109F4D9CE72
:10C4100063E0812F0E94AAA88AE195E00E944CA7C0
:10C42000AAE0EA2EF12CE1CF0E9459AD62E080E053
:10C430000E94AAA888EA91E10E94D1A7C2CE81E019
:10C440000E9463AD69968EAC9FAC69979092B019CB
:10C450008092AF199AAC91103FC020E030E040EAE2
:10C4600050E46091EB0F7091EC0F8091ED0F909183
:10C47000EE0F0F941AB26093EB0F7093EC0F809352
:10C48000ED0F9093EE0FE090E70FF090E80F009122
:10C49000E90F1091EA0F2091E30F3091E40F4091E2
:10C4A000E50F5091E60F6091DF0F7091E00F8091E2
:10C4B000E10F9091E20FEAE1FDE0FF93EF93812C11
:10C4C000912CA12CE0E4BE2EFBEECF2EFFE0DF2E60
:10C4D0000F94C52E0F900F90E090E70FF090E80FAB
:10C4E0000091E90F1091EA0F2D813E814F8158850F
:10C4F00069817A818B819C81EAE16E2EEDE07E2E4E
:10C500007F926F92812C912CF8E4AF2EF2E4BF2E33
:10C51000ABEECA2EAFE0DA2E0F94C52E0F94AB7F90
:10C52000E984FA840B851C852D813E814F815885D5
:10C5300069817A818B819C817F926F92812C912C71
:10C54000B0E7AB2EB1E4BB2E0F94C52E0F94AB7F9A
:10C55000CE010D960E9483BA80E1FE013196AFEDC7
:10C56000BFE001900D928A95E1F780E1EFEDFFE0E9
:10C57000A8E0BDE001900D928A95E1F76396AFAC1B
:10C580006397A0925F026496BFAC6497B09260021A
:10C59000BF92AF9281E897E09F938F938E01015EE7
:10C5A0001F4F1F930F930F94F2A860E0C8010F94E0
:10C5B000685C87EE94E10F94FC271092B90E1092FC
:10C5C000B80E0FB6F894DEBF0FBECDBF38C60F94BD
:10C5D000AF8935C683E50F94EB99882309F42FC6FC
:10C5E0000F94E2990F9479B36B017C012B0185E6DE
:10C5F00092E40F94FC27ECE1FEE084918F01882304
:10C6000039F00E947DFA0F5F1F4FF8018491F7CF38
:10C610000D2C000CEE08FF08C701B6010E9406FBB6
:10C620008AE00E947DFA0F944E864B015C011092C5
:10C63000D20E60911E0D70911F0D072E000C880BFD
:10C64000990B0F9434A920E030E0A9010F942EA992
:10C65000811111C06091601570916115072E000C59
:10C66000880B990B0F9434A911E020E030E0A90168
:10C670000F942EA9811110E0052C000C6608770894
:10C6800087E1282E8EE0382E111115C08091D20E30
:10C6900081116CC0C301B2010F9434A92091C31958
:10C6A0003091C4194091C5195091C6190F9465B4C1
:10C6B00018168CF05BC0C301B2010F9434A920910D
:10C6C000C3193091C4194091C5195091C6190F94DE
:10C6D0002EA987FF4BC00F944E86DC01CB01881931
:10C6E0009909AA09BB09893E9340A105B10508F43F
:10C6F00034C0E9E1FEE084915F01882341F00E94AB
:10C700007DFAFFEFAF1ABF0AF5018491F6CF609171
:10C71000C3197091C4198091C5199091C61941E04F
:10C720000E9420FBF101849107E1A02E0EE0B02EC3
:10C73000882341F00E947DFAFFEFAF1ABF0AF5018E
:10C740008491F6CFC701B6010E9406FB8AE00E94E1
:10C750007DFA0F944E864B015C010F94CD7980E0F9
:10C760000F940C8080E00E945CA58ECF85E897E155
:10C770000F94FC2764C58FE30F94EB99882309F489
:10C78000BCC00E949AF61A821982882381F00DE6B5
:10C7900014E0D8018D918D01882319F00E947DFA53
:10C7A000F8CF8AE00E947DFA01E814E00AC008E9A7
:10C7B00014E0F80181918F01882399F30E947DFA9A
:10C7C000F8CFD8018D918D01882319F00E947DFA50
:10C7D000F8CF8AE00E947DFA44244A94542C320116
:10C7E000A3E28A2E912CA12CB12CB0EB2B2EBFE012
:10C7F0003B2E1AAE69817A81072E000C880B990BAB
:10C800000F9434A920912F103091301040913110A5
:10C81000509132100F9408B36B017C012AAD2111A5
:10C820000DC0E3E1FEE084918F01882359F00E945E
:10C830007DFA0F5F1F4FF8018491F7CFC301B2015A
:10C840000E9406FBE0E1FEE084918F01882339F02D
:10C850000E947DFA0F5F1F4FF8018491F7CFC50149
:10C86000B4010E9406FBEDE0FEE084918F01882375
:10C8700039F00E947DFA0F5F1F4FF8018491F7CFC6
:10C8800069817A81072E000C880B990B0E9406FBA8
:10C89000EAE0FEE084918F01882339F00E947DFA5E
:10C8A0000F5F1F4FF8018491F7CF20E030E04AE797
:10C8B00054E4C701B6010F9426A442E00E9420FB75
:10C8C0008AE00E947DFAFAADFF5FFAAFF63009F414
:10C8D000B6C4BE016F5F7F4FC1010E9435C6B2E092
:10C8E0002B0E311CE5E08E0E911CA11CB11CFFEF3C
:10C8F0004F1A5F0A6F0A7F0A7DCF81E20F94EB998E
:10C90000882309F44AC061E086EA9FE00F94BEB133
:10C9100088E090E09A838983BE016F5F7F4F80EB50
:10C920009FE00E944FC688E190E09A838983BE0110
:10C930006F5F7F4F82EB9FE00E944FC680E390E0E5
:10C940009A838983BE016F5F7F4F84EB9FE00E94D3
:10C950004FC680E590E09A838983BE016F5F7F4F69
:10C9600086EB9FE00E944FC688E790E09A83898318
:10C97000BE016F5F7F4F88EB9FE00E944FC60CEABD
:10C9800014E0D8018D918D01882319F00E947DFA61
:10C99000F8CF8AE00E947DFA52C48AE50F94EB99A1
:10C9A000882319F161E086EA9FE00F94BEB11A82F4
:10C9B000198200EB1FE0BE016F5F7F4FC8010E942C
:10C9C0004FC60E5F1F4F0A3BBFE01B07A1F70DEBE1
:10C9D00014E0F80181918F01882319F00E947DFAFB
:10C9E000F8CF8AE00E947DFA2AC483E50F94EB9980
:10C9F000882309F4CEC00F94E2990F9479B37A8317
:10CA0000698389E40F94EB99882309F418C40F947F
:10CA1000E2990F947FB3653008F011C4862F90E03F
:10CA20008852984FBE016F5F7F4F880F991F0E94F9
:10CA30004FC607EC14E0D8018D918D01882319F0C1
:10CA40000E947DFAF8CF8AE00E947DFA01E814E0A6
:10CA5000F80181918F01882319F00E947DFAF8CFA7
:10CA60008AE00E947DFA5EEA252E5FE0352E44249E
:10CA70004A94542C320173E2872E912CA12CB12CB4
:10CA80001AAE1A821982FAADFF2331F0BE016F5F30
:10CA90007F4FC1010E9435C669817A81072E000C43
:10CAA000880B990B0F9434A920912F1030913010DE
:10CAB00040913110509132100F9408B36B017C01FA
:10CAC0002AAD21110DC0E6E0FEE084918F0188239C
:10CAD00059F00E947DFA0F5F1F4FF8018491F7CF44
:10CAE000C301B2010E9406FBE3E0FEE084918F01E6
:10CAF000882339F00E947DFA0F5F1F4FF80184915F
:10CB0000F7CFC501B4010E9406FBE0E0FEE084918E
:10CB10008F01882339F00E947DFA0F5F1F4FF801C3
:10CB20008491F7CF69817A81072E000C880B990BCD
:10CB30000E9406FBEDEFFDE084918F01882339F020
:10CB40000E947DFA0F5F1F4FF8018491F7CF20E01C
:10CB500030E04AE754E4C701B6010F9426A442E04E
:10CB60000E9420FB8AE00E947DFAFAADFF5FFAAFD7
:10CB700025E0820E911CA11CB11C3FEF431A530A01
:10CB8000630A730A42E0240E311CF63009F079CFB3
:10CB900056C3ECEEFDE084918F01882309F44FC366
:10CBA0000E947DFA0F5F1F4FF8018491F6CF0F941A
:10CBB000AB7F8BE40F94EB99882399F00F94AC9999
:10CBC0006B017C0120E030E0A9010F9465B487FD82
:10CBD00008C0C092BB0FD092BC0FE092BD0FF09284
:10CBE000BE0F82E50F94EB99882361F00F94AC9906
:10CBF0006B017C0120E030E0A9010F942EA987FF92
:10CC000089C006C0C12CD12C40E8E42E4FEBF42E95
:10CC100084E40F94EB99882329F00F94AC994B018D
:10CC20005C0106C0812C912C30E8A32E3FEBB32E83
:10CC300087E50F94EB99882329F00F94AC992B0189
:10CC40003C0106C0412C512C20E8622E2FEB722EA5
:10CC500088E40F94EB99882339F00F94AC996AAF6C
:10CC60007BAF8CAF9DAF08C020E030E040E85FEBC9
:10CC70002AAF3BAF4CAF5DAF20E030E0A901C5016A
:10CC8000B4010F9465B487FD45C020E030E0A901F0
:10CC9000C301B2010F9465B487FD3CC020E030E0D1
:10CCA000A9016AAD7BAD8CAD9DAD0F9465B487FDD8
:10CCB00031C020E030E0A901C501B4010F942EA9D4
:10CCC000882391F120E030E040E05FE3C501B4014A
:10CCD0000F9426A46B017C012AAD3BAD4CAD5DAD3C
:10CCE000C301B2010F9426A44B015C01A701960178
:10CCF000C701B6010F9426A42BED3FE049E450E4B0
:10CD00000F9426A49B01AC01C501B4010F9408B394
:10CD10006B017C0120E030E0A901C701B6010F944E
:10CD200065B487FF04C00BC0C12CD12C7601C09222
:10CD3000B70FD092B80FE092B90FF092BA0FE3E3B9
:10CD4000FDE584918F01882339F00E947DFA0F5F01
:10CD50001F4FF8018491F7CFE6E7F7E084918F0148
:10CD6000882339F00E947DFA0F5F1F4FF8018491EC
:10CD7000F7CF6091BB0F7091BC0F8091BD0F909168
:10CD8000BE0F42E00E9420FB8AE00E947DFAE0E7AD
:10CD9000F7E084918F01882339F00E947DFA0F5FBC
:10CDA0001F4FF8018491F7CFC090B70FD090B80F04
:10CDB000E090B90FF090BA0F20E030E0A901C70170
:10CDC000B6010F942EA9882349F042E0C701B601AD
:10CDD0000E9420FB8AE00E947DFA31C2EBE6F7E078
:10CDE00084918F01882311F40C94C3450E947DFA2D
:10CDF0000F5F1F4FF8018491F5CF0F945D181FC28C
:10CE000088E50F94EB99882339F00F94E2990F94F9
:10CE10007FB380E00F94E89689E50F94EB9988231F
:10CE200039F00F94E2990F947FB381E00F94E89664
:10CE30008AE50F94EB99882339F00F94E2990F94C7
:10CE40007FB382E00F94E89685E40F94EB998823F2
:10CE500009F4F5C10F94E2990F947FB383E00F9426
:10CE6000E896EDC188E50F94EB99882339F00F948B
:10CE7000E2990F947FB380E00F94D79689E50F94E1
:10CE8000EB99882339F00F94E2990F947FB381E0F6
:10CE90000F94D7968AE50F94EB99882339F00F9475
:10CEA000E2990F947FB382E00F94D79685E40F94B4
:10CEB000EB99882309F4C3C10F94E2990F947FB3CF
:10CEC00083E00F94D796BBC181E0809324070E9432
:10CED00067BA0F945D18B3C188E50F94EB99882366
:10CEE00031F00F94E2990F947FB36093650289E566
:10CEF0000F94EB99882331F00F94E2990F947FB34C
:10CF0000609366028AE50F94EB99882331F00F94C1
:10CF1000E2990F947FB36093670285E40F94EB99D5
:10CF2000882331F00F94E2990F947FB360936802E5
:10CF300015E6C12E12E0D12E0AE313E08EE3A82EEF
:10CF400083E0B82E9EE8E92E95E0F92ED6019D915A
:10CF50006D01F80181918F011F929F93282F082E58
:10CF6000000C330B3F938F93FF92EF920F949AA88C
:10CF70000F900F900F900F900F900F90A016B1068A
:10CF800029F75DC188E50F94EB99882339F00F9458
:10CF9000E2990F947FB380E00F94B69689E50F94E1
:10CFA000EB99882339F00F94E2990F947FB381E0D5
:10CFB0000F94B6968AE50F94EB99882331F00F947D
:10CFC000E2990F947FB36093370285E40F94EB9955
:10CFD000882309F434C10F94E2990F947FB36093CE
:10CFE00038022DC188E50F94EB99882339F00F940E
:10CFF000E2990F947FB380E00F94949689E50F94A3
:10D00000EB99882339F00F94E2990F947FB381E074
:10D010000F9494968AE50F94EB99882331F00F943E
:10D02000E2990F947FB360933B0285E40F94EB99F0
:10D03000882309F404C10F94E2990F947FB360939D
:10D040003C02FDC085E40F94EB99882309F4F7C0F6
:10D050000F94E2990F947FB36B017C018B016830D0
:10D06000710569F06031710551F06032710539F078
:10D070006034710521F06038710509F0E0C00F944B
:10D08000AB7F80E091E05C0100901F0702C0B69486
:10D09000A7940A94E2F7C6010E94E69E80931F07B8
:10D0A00020911D0240912102682F83E00E94099F78
:10D0B00040901F105090201060902110709022100E
:10D0C000A016B10670F5C801B5010F94C5B66B0185
:10D0D000E12CF12CC701B6010F9432A99B01AC01E0
:10D0E000609133107091341080913510909136100A
:10D0F0000F9426A4609333107093341080933510EE
:10D1000090933610A3019201C701B6010F94CFB1DD
:10D1100060931F1070932010809321109093221021
:10D120008EC0C501B8010F94C5B66B01E12CF12C7E
:10D13000C701B6010F9432A99B01AC016091331075
:10D140007091341080913510909136100F9408B37F
:10D150006093331070933410809335109093361091
:10D16000C301B201A70196010F94ECB620931F10E2
:10D1700030932010409321105093221060C0809172
:10D180005213882329F085E40F94EB99811184C709
:10D190000F94DB6054C0809152138823D9F185E548
:10D1A0000F94EB99882359F120E030E04FE253E4EB
:10D1B0006091750F7091760F8091770F9091780F35
:10D1C0000F9465B41816C4F400E010E08091240EAA
:10D1D000082E000C990B002E02C0959587950A9495
:10D1E000E2F780FD0E9472D80F5F1F4F04301105D7
:10D1F00069F71092240E23C00E9422D520C083E438
:10D200000F94EB99882319F00E9472D818C00E94DD
:10D2100042D915C00E944FCE12C080915E159091E8
:10D220005F158C589C4E9F938F9387ED9DE09F9345
:10D230008F930F949AA80F900F900F900F901092C9
:10D240001E0E10921D0E57C284E50F94EB99882391
:10D2500009F4E2C00F94AB7F20913D1330913E134F
:10D26000F90131968F01021B130B81918032D1F3AA
:10D270008930C1F390ED980F953020F18F3371F024
:10D28000E7ECFDE084918F01882309F4C1C00E947E
:10D290007DFA0F5F1F4FF8018491F6CF80915213F2
:10D2A00040E050E0882329F06FEC7AE480EA92E1D4
:10D2B00004C066E872E18FE892E10E945DCF80933E
:10D2C000260D06C00F94E2990F947FB36093260D4C
:10D2D0008091260D21E030E0082E01C0220F0A9433
:10D2E000EAF79091240E292B2093240E909152134B
:10D2F000992301F1805F8093260E1092250E61E044
:10D3000081E00E943ED580E38093260E1092250E88
:10D310008091260D8093270D80913D1390913E13AF
:10D32000FC01E00FF11F80818F3309F0E4C10F94FD
:10D33000F996E1C1882309F432C0E3E3FDE5849165
:10D340008F01882339F00E947DFA0F5F1F4FF8018B
:10D350008491F7CFE5ECFDE084918F01882339F0CB
:10D360000E947DFA0F5F1F4FF8018491F7CF609103
:10D37000260D70E080E090E00E9406FB8AE00E94AB
:10D380007DFAEDE7F5E084918F01882309F440C030
:10D390000E947DFA0F5F1F4FF8018491F6CF86E45B
:10D3A0000F94EB99882399F00F94E2996B017C011B
:10D3B00020E030E0A9010F9465B4181644F4C0923F
:10D3C0002202D0922302E0922402F0922502E3E3AB
:10D3D000FDE584918F01882339F00E947DFA0F5F6B
:10D3E0001F4FF8018491F7CFEBE6F5E084918F01B0
:10D3F000882339F00E947DFA0F5F1F4FF801849156
:10D40000F7CF60911A0D70E080E090E00E9406FB7B
:10D410008AE00E947DFA6FC184E40F94EB9988231F
:10D4200009F408C10F94E2990F9479B36330710540
:10D4300009F061C184E295E09F938F930F949AA8BD
:10D4400081E40F94EB990F900F908823B9F08091AD
:10D450003D1390913E13DC0111962C91283741F435
:10D4600040E150E060E070E002960F944EA604C0E8
:10D470000F94E2990F9479B38B0102C000E010E0A1
:10D4800083E40F94EB99882339F00F94E2990F9479
:10D4900079B3262F872F02C020E080E11F71A22ED2
:10D4A000B82EB1E0AB16B0E1BB0618F0A12CB0E18C
:10D4B000BB2EC501800F911F8130904128F080E084
:10D4C00090E15C01A01AB10A88E50F94EB998823DA
:10D4D00009F475C020913D1330913E13A9014F5FAF
:10D4E0005F4F9E012F5F3F4F6901F901E12CF12C45
:10D4F0009A01D9018C912F5F3F4F8823A1F140E120
:10D50000E416F10469F18032A1F38A3061F190ED03
:10D51000980F9A3018F48295807F07C09FE9980F82
:10D520009630A8F48295807F8057AD014E5F5F4FA3
:10D5300011969C9120ED290F2A3010F4822B0BC0FC
:10D540002FE9290F263018F49755892B04C0F19440
:10D55000E194F10808C081936FEFE61AF60AC8CF8C
:10D56000A0E1EA2EF12C5701E114F10441F1812CE4
:10D57000912CD6016D916D01C801880D991D0F94F4
:10D58000BEB1BFEF8B1A9B0AE814F90491F71F9301
:10D590000F93FF92EF9287EF94E09F938F930F94F6
:10D5A0009AA86091CD197091CE198AE090E00F94FD
:10D5B000CBB00F900F900F900F900F900F906801CD
:10D5C000E12CF12CA114B10409F495C08D2D0F9418
:10D5D000009A8C2D0F94009A6091CD197091CE19FC
:10D5E00080E290E00F94CBB010E1EFEFCE1ADE0AAC
:10D5F000EE0AFE0AC60101970F948EB1082F6091C2
:10D60000CD197091CE1980E290E00F94CBB0802FAD
:10D610000F94009A1150F1E0AF1AB10811F01111F6
:10D62000E4CF6091CD197091CE198AE090E00F940B
:10D63000CBB0C8CFE3E3FDE584918F01882339F0B7
:10D640000E947DFA0F5F1F4FF8018491F7CFEEEA39
:10D65000F5E084918F01882339F00E947DFA0F5FF5
:10D660001F4FF8018491F7CF00915E1510915F155F
:10D670000C581C4ED8018D918D01882319F00E9401
:10D680007DFAF8CFE0ECFDE084918F01882309F466
:10D69000BFCE0E947DFA0F5F1F4FF8018491F6CF35
:10D6A000C090140DD090150DE090160DF090170D50
:10D6B0002091EB0F3091EC0F4091ED0F5091EE0F58
:10D6C000C701B6010F9419B24B015C012DEC3CEC83
:10D6D0004CEC5DEB0F942EA987FD3AC02DEC3CEC91
:10D6E0004CEC5DE3C501B4010F9465B418160CF45D
:10D6F00038C00F94AFA081E090E09093280280930F
:10D7000027020F944E86609367197093681980936F
:10D71000691990936A19E0915E15F0915F15EF58C1
:10D72000FC4E8081813019F0863009F0D7C4E5E8DD
:10D73000F7E184918F01882339F00E947DFA0F5F11
:10D740001F4FF8018491F7CF8AE00E947DFAC6C48A
:10D75000E0911A0DF0E0EF50F14F80818111A3C4E8
:10D7600009C0E0911A0DF0E0EF50F14F808188235D
:10D7700009F4BFCFC092EB0FD092EC0FE092ED0F07
:10D78000F092EE0F8BEE9FE00E9483BAE0911A0DAB
:10D79000F0E0EF50F14F908181E089270F94609A7B
:10D7A0009DC420E030E040E85FE36091EB0F7091B2
:10D7B000EC0F8091ED0F9091EE0F0F941AB26093E1
:10D7C000EB0F7093EC0F8093ED0F9093EE0FE090C2
:10D7D000E70FF090E80F0091E90F1091EA0F209108
:10D7E000E30F3091E40F4091E50F5091E60F609107
:10D7F000DF0F7091E00F8091E10F9091E20FEAE16D
:10D80000FDE0FF93EF93812C912CE8ECAE2EE3E446
:10D81000BE2EFBEECF2EFFE0DF2E0F94C52E0F9015
:10D820000F900C94914082E090E0909328028093B6
:10D8300027021092BF0E1092BE0E0C946E450F94EC
:10D84000D799AB01BC0140933219509333196093BF
:10D850003419709335198DE798E10E9410DCEFCCF4
:10D860000F94E2990F9479B38B010C94EB480F94C9
:10D87000AB7F88E50F94EB99882319F0179A1092E3
:10D880001B0D89E50F94EB99882319F0169A1092D5
:10D890001C0D8AE50F94EB9985E40F94EB9988238E
:10D8A00011F40C945F4D149A0C945F4D1A821982F6
:10D8B0004AE050E0BE016F5F7F4FC7010F944EA654
:10D8C00078A36F8F89819A818816990609F0B7CC61
:10D8D0004AE050E0BE016F5F7F4FC6010F944EA635
:10D8E0007AA369A389819A816816790609F0A7CC81
:10D8F0004AE050E0BE016F5F7F4FC5010F944EA616
:10D900007CA36BA389819A810817190709F097CC2A
:10D910008FE790E09EA38DA35801EFEFAE1ABE0AE9
:10D92000D8018C918D3211F575016701BFEFCB1ACB
:10D93000DB0AF70180810F94D227382E811102C0B3
:10D940007601F3CFEA18FB08DE2CC7019927833054
:10D95000910569F543E050E06BEB75E5C5010F9467
:10D96000C0A7892B09F042C01EA21DA2332009F4D2
:10D9700066CCCE0101960F94D54C882309F45FCC78
:10D98000FE017F96DE011196AE01495D5F4F219148
:10D9900031918D919D918217930708F44CC02817FF
:10D9A000390708F44CCC4E175F0789F748CC85300F
:10D9B000910571F445E050E065EB75E5C5010F9404
:10D9C000C0A7892B99F481E090E09EA38DA3CECFD0
:10D9D000049761F444E050E060EB75E5C5010F94F5
:10D9E000C0A7892B19F482E090E0EFCF8EEF8E0D67
:10D9F000823008F024CCD80111968C9111978F7D3C
:10DA0000823509F01CCC12968C918F7D833409F0FD
:10DA100016CCB2E0DB1203C083E090E0D6CFF80171
:10DA2000838190ED980F9A3008F009CC082E000CF5
:10DA3000990B8E97CACF88E192E10F948F044AE048
:10DA40005DE062E080E00E944EADD2011D912D01AB
:10DA5000812F0F94D227811108C063ED76E0812FCA
:10DA6000110F990B0F94CBB0F0CF48E052E163E077
:10DA700080E00E944EAD80910D0790910E070297B5
:10DA800020F488EE93E00F94DC4682E390E00E945D
:10DA9000A59484E50F94602384EF91E00E94A594FF
:10DAA00080910D0790910E07029720F488EE93E085
:10DAB0000F94DC4682E390E00E94A59484E50F94E5
:10DAC000602384E090E090932802809327020F94D3
:10DAD000CD7981E00F940C800E9434A68823B9F39D
:10DAE00082E090E0909328028093270281E00E94D8
:10DAF00063AD0E9459AD80E00E945CA5A0CBAC96BE
:10DB0000CCACDDACEEACFFACAC97C80ED91EEA1EB7
:10DB1000FB1EAC962CAD3DAD4EAD5FADAC97281B5A
:10DB2000390B4A0B5B0B2A966CAD7DAD8EAD9FAD6C
:10DB30002A970F94CFB1A70196010F94ECB6DA01A2
:10DB4000C901840D951DA61DB71D84319105A10540
:10DB5000B105E4F02C013D018C3E9105A105B10514
:10DB60002CF06BEE462E512C612C712C40E84416A3
:10DB7000510461047104DCF05EEF852E912CA12C20
:10DB8000B12C84189508A608B7080AC034E1432EC2
:10DB9000512C612C712C44E1842E912CA12CB12CA0
:10DBA0002A968CAE9DAEAEAEBFAE2A9706C02A9620
:10DBB0004CAE5DAE6EAE7FAE2A97E7EEFCE0849190
:10DBC0008F01882339F00E947DFA0F5F1F4FF80103
:10DBD0008491F7CFC301B2010E9406FBE2EEFCE0A4
:10DBE00084918F01882339F00E947DFA0F5F1F4FC7
:10DBF000F8018491F7CF2A966CAD7DAD8EAD9FADC7
:10DC00002A970E9406FBEBEDFCE084918F018823AC
:10DC100039F00E947DFA0F5F1F4FF8018491F7CF12
:10DC200042E06E966FAD6E976F967FAD6F97A09640
:10DC30008FADA097A1969FADA1970E9420FBE4ED28
:10DC4000FCE084918F01882339F00E947DFA0F5FF8
:10DC50001F4FF8018491F7CF42E0A2966FADA297D3
:10DC6000A3967FADA397A4968FADA497A5969FADDD
:10DC7000A5970E9420FB8AE00E947DFA80912B0DDF
:10DC800090912C0D039714F40C94AF582A966CAD18
:10DC90007DAD8EAD9FAD2A970F9434A920E030E082
:10DCA00040E850E40F9426A44B015C016E962FAD22
:10DCB0006E976F963FAD6F97A0964FADA097A196C8
:10DCC0005FADA197A2966FADA297A3967FADA397E4
:10DCD000A4968FADA497A5969FADA5970F9419B262
:10DCE00020ED3FE049E450E40F9426A420E030E02A
:10DCF00040E05FE30F9426A49B01AC01C501B40191
:10DD00000F9408B34B015C01C701B6010F9434A90D
:10DD100020E030E04AE754E40F9408B36B017C0143
:10DD2000EEECFCE084918F01882339F00E947DFAAB
:10DD30000F5F1F4FF8018491F7CF42E0C501B40196
:10DD40000E9420FBE8ECFCE084918F01882339F0ED
:10DD50000E947DFA0F5F1F4FF8018491F7CF42E0D8
:10DD6000C701B6010E9420FB8AE00E947DFA2AE9E1
:10DD700039E949E15FE3C501B4010F9426A44B01E1
:10DD80005C0160935A0E70935B0E80935C0E9093CF
:10DD90005D0E9B01AC010F941AB2A70196010F947E
:10DDA00008B36093560E7093570E8093580E90935D
:10DDB000590EA5019401C701B6010F9426A420E0D5
:10DDC00030E040E05EE30F9426A46093520E70931F
:10DDD000530E8093540E9093550EEAEBFCE0849121
:10DDE0008F01882339F00E947DFA0F5F1F4FF801E1
:10DDF0008491F7CF8AE00E947DFAE4EBFCE0849105
:10DE00008F01882339F00E947DFA0F5F1F4FF801C0
:10DE10008491F7CF60915A0E70915B0E80915C0EE9
:10DE200090915D0E42E00E9420FB8AE00E947DFA04
:10DE3000EEEAFCE084918F01882339F00E947DFA9C
:10DE40000F5F1F4FF8018491F7CF6091560E7091CC
:10DE5000570E8091580E9091590E42E00E9420FB7F
:10DE60008AE00E947DFAE8EAFCE084918F01882331
:10DE700039F00E947DFA0F5F1F4FF8018491F7CFB0
:10DE80006091520E7091530E8091540E9091550EE8
:10DE900042E00E9420FB8AE00E947DFA0C94AF5879
:10DEA0008093090F0C94C758E9961FAEE9970C941C
:10DEB000EC5884E690E00E94A5940C94645A1AAE43
:10DEC0000C94825EE12CF12C80910101846080939E
:10DED0000101E114F10409F04EC080910D07909109
:10DEE0000E070097F1F10197D1F14FEFE41AF40A10
:10DEF00051E0D51609F452C0D51608F04AC084E0A6
:10DF000090E00E94A5940F944E86950184010054E0
:10DF1000184D264F3F4F061717072807390710F0EF
:10DF20000C94AB5F8AE790E10F948F041F8E18A2C8
:10DF300019A21AA2CE014F960F94BD720F94AB7F17
:10DF4000149ADD24D3940F94CD7981E00F940C8042
:10DF5000F4EFEF16F1E0FF0609F0B6CFB3CFCC2017
:10DF600021F29FB7F89480910201846080930201AE
:10DF70009FBFC12CBACF34E1E316F10409F0B5CF4D
:10DF80009FB7F894809102018B7F809302019FBF1D
:10DF9000ACCF62E0D616E1F00C94AB5F84E090E089
:10DFA0000E94A5940E9434A6882369F2E0911A0D7C
:10DFB000F0E0EE0FFF1FE05AFA4E67968EAD9FAD70
:10DFC0006797918380830E94E4C542E0D42EBBCF43
:10DFD00000911A0D10E0F801EE0FFF1FE05AFA4E03
:10DFE00060817181072E000C880B990B0F9434A966
:10DFF000000F111F000F111FF801EB58F04F208187
:10E000003181428153810F9419B22B013C0120E0F0
:10E0100030E0A9010F9465B418165CF420E030E0FC
:10E0200040E85FE3C301B2010F942EA987FF16C039
:10E030000AC020E030E040E85FEBC301B2010F947A
:10E0400065B418165CF485EA90E10F948F040F9480
:10E050004E864B015C01D12C0C94AE5F64E081E0F4
:10E060000E94AAA8E0911A0D94E0E99FF001112402
:10E07000EB58F04F80819181A281B3818F8F98A35B
:10E08000A9A3BAA3CE014F960F94F5560E944CA7B0
:10E0900014E1E12EF12C57CF0F94E2990F947FB346
:10E0A0006093260D75C82DEC3CEC4CEC5DE3C5018E
:10E0B000B4010F9465B418160CF45CCB1ACBA5010F
:10E0C0009401F101662D772D8F2F922D0F942EA99B
:10E0D000181614F40C94403A0C94503AC858DF4F78
:10E0E0000FB6F894DEBF0FBECDBFDF91CF911F9169
:10E0F0000F91FF90EF90DF90CF90BF90AF909F90E7
:10E100008F907F906F905F904F903F902F900895E9
:10E110002F923F924F925F926F927F928F929F9237
:10E12000AF92BF92CF92DF92EF92FF920F931F9325
:10E13000CF93DF93CDB7DEB7C95CD1090FB6F894A2
:10E14000DEBF0FBECDBF6B968FAF6B9781E00F9494
:10E15000DA626B962FAD6B97211125C010921F0DBF
:10E1600010921E0D19821A821B821C82CE0101960A
:10E170000F94BD7261E080EC9FE00F94A0B160E06D
:10E180008FEB9FE00F94A0B160E08EEB9FE00F94C7
:10E19000A0B160E08DEB9FE00F94A0B160E08CEB4C
:10E1A0009FE00F94A0B180E00E9463AD0F94B94945
:10E1B0000E94C4A21092190D1092180D83E0EBE199
:10E1C000FDE0DF011D928A95E9F781E00E941AF4D3
:10E1D000C855DF4F99838883C85AD04083E69CE1B5
:10E1E0000F948F040E9449F440E050E061E080E029
:10E1F00090E00F941B6340E050E061E081E090E02C
:10E200000F941B63E090E70FF090E80F0091E90F87
:10E210001091EA0F2091E30F3091E40F4091E50F48
:10E220005091E60F6091DF0F7091E00F8091E10F48
:10E230009091E20F0F944A420E94A6B910922602D2
:10E2400020E030E040EA50E46091DF0F7091E00F91
:10E250008091E10F9091E20F0F941AB21B012C01F3
:10E260006093DF0F7093E00F8093E10F9093E20FC4
:10E2700020E030E040EA50E46091E30F7091E40F59
:10E280008091E50F9091E60F0F941AB29B01AC01BB
:10E290006093E30F7093E40F8093E50F9093E60F84
:10E2A000E090E70FF090E80F0091E90F1091EA0F6E
:10E2B000AAE16A2EADE07A2E7F926F92812C912C8A
:10E2C000B0EAAB2EB1E4BB2E8BEEC82E8FE0D82E79
:10E2D000C201B1010F94C52E0F94AB7F0E9459ADBE
:10E2E0004FE75AE161E080E00E944EAD3090260297
:10E2F00081E080932602E4E2FFE1449055244194BA
:10E300000CF4509484E00F94D1171092E70F109200
:10E31000E80F1092E90F1092EA0F2091E30F30916D
:10E32000E40F4091E50F5091E60F6091DF0F70917F
:10E33000E00F8091E10F9091E20FE12CF12C870129
:10E340000F944A420E9449F4EEE1FFE16591759114
:10E35000859194912DEC3CEC4CE85FE30F9426A45E
:10E360006B017C01B201052C000C880B990B0F94FA
:10E3700034A99B01AC01C701B6010F9426A42091DA
:10E38000100D3091110D4091120D5091130D0F94FD
:10E390001AB27B018C016093100D7093110D809364
:10E3A000120D9093130D80E090E0A8E4B4E4809304
:10E3B000220290932302A0932402B093250220917D
:10E3C0000C0D30910D0D40910E0D50910F0D60917F
:10E3D000080D7091090D80910A0D90910B0D7F929F
:10E3E0006F92E5E58E2E982CA82CE1E4BE2EF4E188
:10E3F000CF2EFDE0DF2E0F94C52E0F94AB7F0F9430
:10E400003617109226021092E70F1092E80F109222
:10E41000E90F1092EA0F2091E30F3091E40F409141
:10E42000E50F5091E60F6091DF0F7091E00F809142
:10E43000E10F9091E20FE12CF12C87010F944A42F9
:10E440000E9449F48AE0849DB001859D700D1124DD
:10E45000072E000C880B990B0F9434A92091100DF6
:10E460003091110D4091120D5091130D0F941AB26D
:10E470007B018C016093100D7093110D8093120D30
:10E480009093130D80E090E0A8ECB3E48093220217
:10E4900090932302A0932402B093250220910C0DA7
:10E4A00030910D0D40910E0D50910F0D6091080DA2
:10E4B0007091090D80910A0D90910B0D7F926F92D2
:10E4C000A5E58A2E982CA5EDAA2EA0E4BA2E0F94CD
:10E4D000C52E0F94AB7F3092260280E090E0A4E539
:10E4E000B3E48093E70F9093E80FA093E90FB09304
:10E4F000EA0F2091E30F3091E40F4091E50F509126
:10E50000E60F6091DF0F7091E00F8091E10F909125
:10E51000E20FE12CF12C04E513E40F944A420F942E
:10E5200010630F900F900F900F900F900F906B96BD
:10E53000BFAD6B97B11132C084E090E09093280298
:10E540008093270240E060E088E49CE10F949C0403
:10E55000882321F080E29CE10F94790586EE9BE10F
:10E560000F94790580E59BE10F94790582E090E0B6
:10E57000909328028093270280E39BE10F948F04FD
:10E5800062E080E00E94AAA861E070E080E090E094
:10E590000E94BEA68AE29BE10E94D1A780E090E0A3
:10E5A000A0EAB0E48093E70F9093E80FA093E90FFF
:10E5B000B093EA0F7090260281E08093260284E0F7
:10E5C0000F94D117E090E70FF090E80F0091E90F5A
:10E5D0001091EA0F2091E30F3091E40F4091E50F85
:10E5E0005091E60F6091DF0F7091E00F8091E10F85
:10E5F0009091E20FEAE1FDE0FF93EF93812C912CE3
:10E60000E0EAAE2EE1E4BE2EFBEECF2EFFE0DF2EE1
:10E610000F94C52E0F94AB7F0F943617709226027D
:10E6200082E00F94987F0F900F9020E030E040EA56
:10E6300050E40F942EA981110C946C856B96EFAD6C
:10E640006B97EE23E9F0C855DF4F88819981C85A4E
:10E65000D0400E94F9F30E94B3A40E94C6A00E9479
:10E66000D8A8882311F40C941C850E94D5F9803F0A
:10E6700011F00C94688581E00E94A4F60C946885E2
:10E680008AEF0E94A4F660E070E088EF9FE00F94AC
:10E69000BAB10F94106384ECE4E6F5E1DF011D925A
:10E6A0008A95E9F7EAE0FFE184918F01882339F048
:10E6B0000E947DFA0F5F1F4FF8018491F7CF61E050
:10E6C00070E080E090E00E9406FB0E94B2FBBE0179
:10E6D0006F5A7F4F80E39BE10F947C0462968FAD6D
:10E6E0006297843020F083E062968FAF629780E07B
:10E6F00090E0A0EAB0E48093E70F9093E80FA09336
:10E70000E90FB093EA0F2AEE3EE1C657DF4F398397
:10E710002883CA58D04083E695E1CE57DF4F9983CE
:10E720008883C258D0406C969FAF8EAF6C97A896E6
:10E730003FAF2EAFA89781E090E0A0E0B0E0AE96AA
:10E740008CAF9DAFAEAFBFAFAE970F941063629624
:10E750006FAD629780E00E94AAA8AE966CAD7DADC9
:10E760008EAD9FADAE970E94BEA68AE29BE10E944D
:10E77000D1A765E575E585E591E40E9458A0A896C6
:10E78000EEADFFADA89785919591A591B491809339
:10E79000DF0F9093E00FA093E10FB093E20FA896E4
:10E7A000EEADFFADA897349685919591A591B49162
:10E7B0008093E30F9093E40FA093E50FB093E60FDF
:10E7C00060E070E088E492E40E9458A00091D70FC6
:10E7D0001091D80F2091D90F3091DA0F4091D30FBB
:10E7E0005091D40F6091D50F7091D60F8091CF0FBB
:10E7F0009091D00FA091D10FB091D20F3F932F9352
:10E800001F930F937F936F935F934F93BF93AF9338
:10E810009F938F9386E79EE19F938F930F949AA87F
:10E820000F94AB7F4091CF0F5091D00F6091D10FDB
:10E830007091D20F8091D30F9091D40FA091D50FEA
:10E84000B091D60FC090D70FD090D80FE090D90FCD
:10E85000F090DA0F21E00FB6F894DEBF0FBECDBF07
:10E86000413157420CF420E08131974214F00C946E
:10E870007285822F90E0880F991FFC01E259F14EBA
:10E88000A590B490FC01EA59F14E85909490DF92E6
:10E89000CF929F928F92BF92AF921F922F938DE44F
:10E8A0009EE19F938F930F949AA88DE69CE19F938E
:10E8B0008F930F949AA80F94681A80916E008B7FA3
:10E8C00080936E00EF9880916F008D7F80936F0032
:10E8D0000FB6F894A89580916000886180936000DD
:10E8E000109260000FBE1092070D1092060D89E67F
:10E8F00091E09093050D8093040D81E991E0909350
:10E90000030D8093020D00E028EC30E0A601B40175
:10E91000C5010F9403240091D70F1091D80F2091B7
:10E92000D90F3091DA0F4091D30F5091D40F6091ED
:10E93000D50F7091D60F8091CF0F9091D00FA091ED
:10E94000D10FB091D20F3F932F931F930F937F93CB
:10E950006F935F934F93BF93AF939F938F938DE08C
:10E960009DE19F938F930F949AA88091CF0F9091E0
:10E97000D00FA091D10FB091D20F782E692E809137
:10E98000D30F9091D40FA091D50FB091D60F582EE0
:10E99000492EC090D70FD090D80FE090D90FF090AB
:10E9A000DA0F0FB6F894DEBF0FBECDBF44E8242EB9
:10E9B0004CE1342E95E0C91697EFD9060CF46EC0E1
:10E9C0001A8219821F921F92A3E0AF93B4E8BF93FB
:10E9D0001F92E4E6EF93DF92CF924F925F926F9295
:10E9E0007F923F922F920F949AA80FB6F894DEBFB1
:10E9F0000FBECDBF89819A81803D924030F08981E0
:10EA00009A81803A954050F512C0CE0101967C0162
:10EA100000E010E024E833E0A601652D742D872D79
:10EA2000962D0F94854B81110C946386E8CFDE01FF
:10EA300011967D0100E010E02CE73CEFA601445662
:10EA40005109652D742D872D962D0F94854B8823A4
:10EA500029F089819A8180539D4F1CC089819A81B8
:10EA60008037984008F04AC0FE0131967F0104EBE0
:10EA700010E024E833E0A601485C5109652D742DAF
:10EA8000872D962D0F94854B8823C1F189819A811A
:10EA900080569A4F9A8389830C9463860091D70F8E
:10EAA0001091D80F2091D90F3091DA0F4091D30FE8
:10EAB0005091D40F6091D50F7091D60F8091CF0FE8
:10EAC0009091D00FA091D10FB091D20F3F932F937F
:10EAD0001F930F937F936F935F934F93BF93AF9366
:10EAE0009F938F938CEB9CE19F938F930F949AA8A5
:10EAF0000FB6F894DEBF0FBECDBFD9C389819A810E
:10EB000080349B40A0F49E012F5F3F4F790104EBBE
:10EB100010E02CE73CEFA6014C525140652D742DBE
:10EB2000872D962D0F94854B81110C94778580E06D
:10EB3000E981FA81882311F40C947F858091CF0FAD
:10EB40009091D00FA091D10FB091D20F4091D30FDF
:10EB50005091D40F6091D50F7091D60F0091D70FBF
:10EB60001091D80F2091D90F3091DA0FFF93EF93C6
:10EB70001F930F935F934F939F938F9389EE9CE125
:10EB80009F938F930F949AA84091D70F5091D80FCD
:10EB90006091D90F7091DA0F00E028EC30E0B401F9
:10EBA000C5010F94032485E08F9380E78F938DE157
:10EBB0009EE19F938F930F949AA884E08F9388E3AC
:10EBC0008F938BE09EE19F938F930F949AA88091EF
:10EBD000CF0F9091D00FA091D10FB091D20F6A9624
:10EBE0008CAF9DAFAEAFBFAF6A976896CEACDFACCF
:10EBF00068978091D30F9091D40FA091D50FB091C9
:10EC0000D60FE2968CAF9DAFAEAFBFAFE2978091CB
:10EC1000D70F9091D80FA091D90FB091DA0FA2968B
:10EC20008CAF9DAFAEAFBFAFA2971C0198E4291A7D
:10EC3000310889E08F9380E68F933F922F92E09680
:10EC4000AFADE097AF93AF96BFADAF97BF93689668
:10EC5000EFAD6897EF936796FFAD6797FF9386E3F5
:10EC60009DE19F938F930F949AA84091D70F509155
:10EC7000D80F6091D90F7091DA0F7A0120E931E055
:10EC8000E0966EAD7FADE09768968EAD9FAD6897CC
:10EC90000F940324E0962EAD3FADE0973450EC96F0
:10ECA0003FAF2EAFEC970FB6F894DEBF0FBECDBFCF
:10ECB000812C912CD601B450E896BFAFAEAFE89747
:10ECC000F601FC5FC258DF4FF983E883CE57D0408E
:10ECD000382D3170A3963FAFA39780FC02C00C94EF
:10ECE0008585EF968FADEF97C158DF4F9881CF574D
:10ECF000D04000E020E931E0A701EC966EAD7FAD99
:10ED0000EC970F940324C090D30FD090D40FE090D1
:10ED1000D50FF090D60F8091CF0F9091D00FA0918A
:10ED2000D10FB091D20F01E028EC30E0A101B60183
:10ED30000F940324C090D30FD090D40FE090D50F40
:10ED4000F090D60F8091CF0F9091D00FA091D10F5E
:10ED5000B091D20F0FEF28EC30E040E659E0B60159
:10ED60000F9403248091D70F9091D80FA091D90FC1
:10ED7000B091DA0F7C01A3966FADA39780910B0140
:10ED8000662311F40C948D85816080930B01000043
:10ED9000840125E0000F111F2A95E1F7A3968FAD9E
:10EDA000A397882311F40C94908590EC492E552458
:10EDB0005A94652C752CC12CD12C90E4E3969FAF0E
:10EDC000E397A12CB12C93B1A70142195309292F24
:10EDD000207194FF02C00C94978588EE9FEF840FFA
:10EDE000951F97FD02C00C949B8580E090E0A80ED3
:10EDF000B91E80910B0121110C94A585846080932C
:10EE00000B01000021110C94A8852E143F0434F44A
:10EE100084E00E94ECB9A1E0EA1AF10881E00E94C6
:10EE2000ECB98BE599E00197F1F7E396FFADE39735
:10EE3000F150E396FFAFE397F111C5CFB6E0B6947A
:10EE4000A794BA95E1F7A3962FADA397222311F4C7
:10EE50000C94B7858FE190E08C199D09800F911F6C
:10EE6000FC01EE56F84FA0828091CF0F9091D00F09
:10EE7000A091D10FB091D20F840D951DA61DB71D85
:10EE80008093CF0F9093D00FA093D10FB093D20F58
:10EE9000C7010F2C000CAA0BBB0B8093D70F9093CC
:10EEA000D80FA093D90FB093DA0F3FEFC31AD30A4C
:10EEB00060E2C616D10409F080CF0E56184FF0E27A
:10EEC000BF2EA1E3CA2EADE1DA2ED8018D918D01BE
:10EED0001F928F93DF92CF920F949AA8BA940F90BB
:10EEE0000F900F900F90B110F0CF8FE29DE19F93A4
:10EEF0008F930F949AA8BFEF8B1A9B0AEC96EEADF6
:10EF0000FFADEC97E05CFF4FEC96FFAFEEAFEC97F8
:10EF10000F900F90F0E28F16910409F0D9CEE2E93C
:10EF2000AE2EEBE0BE2E82EB9BE0F501119211922A
:10EF30008E179F07D9F780E090E0DC0175E0AA0FFB
:10EF4000BB1F7A95E1F7AE56B84F40E0ED91F0E087
:10EF500054E0F595E7955A95E1F7EE0FFF1FEE5651
:10EF6000F44F208131812F5F3F4F318320834F5FEA
:10EF7000403261F7019680329105F9F622E9C22EFE
:10EF80002BE0D22E00E010E03EE6E32E3DE1F32E32
:10EF9000D6018C9111969C91B2E0CB0ED11C9F931F
:10EFA0008F931F930F93FF92EF920F949AA80F5F86
:10EFB0001F4F0F900F900F900F900F900F900031F8
:10EFC000110531F78091940B9091950BE4E9FBE0EA
:10EFD00031E021E0419151918417950710F4322FCF
:10EFE000CA012F5F2031B1F7032F1F923F939F93E8
:10EFF0008F9385E99DE19F938F930F949AA8E0EBFF
:10F00000FBE00F900F900F900F900F900F908EE0FD
:10F01000329122912A30310510F40C94BA858295F0
:10F02000807F2091920B3091930B2037334010F06A
:10F030000C94C185000F000F000F182F101B1F929A
:10F040001F931F928F931F920F938EE79DE19F93C3
:10F050008F930F949AA892E9492E97E0592E0FB6F4
:10F06000F894DEBF0FBECDBFF201202F30E0012F9C
:10F0700010E0808190E02817390710F00C94C485C7
:10F08000821B930B982F80E0B8010F94C5B66F3F99
:10F09000710519F010F06FEF70E06193AE16BF06C6
:10F0A00041F700E010E0B9E7AB2EBDE1BB2E87E7EA
:10F0B000C82E8DE1D82EC801A5E0880F991FAA950A
:10F0C000E1F7DC01AE56B84F7D01912CF70181913B
:10F0D0007F011F928F93BF92AF920F949AA893943F
:10F0E0000F900F900F900F90F0E29F12EFCFDF92F2
:10F0F000CF920F949AA80F5F1F4F0F900F9000327E
:10F100001105C9F683EF9DE12AEE3BE0A2EDBBE0DD
:10F11000FC01459154914D935D9302962A173B074C
:10F12000B9F7612C712CE12CF12C10E000E0A12C3E
:10F1300040E050E0EB964FAFEB9722ED3BE0E896D6
:10F140003FAF2EAFE897A0E0B0E080E090E0B12CB8
:10F150004A01860C971C20E030E014012A0E3B1E69
:10F160006EEF6B0DE3966FAFE397B1100C94C8850B
:10F170006EEF620F683010F40C94CF852F5F3F4F15
:10F180002C30310591F7B3949096E896EEADFFAD33
:10F19000E8973296E896FFAFEEAFE897FCE0BF1233
:10F1A000DACFE816F9062CF47C010A2DEB961FAD98
:10F1B000EB974F5F5F4F4431510509F0BBCFA394EC
:10F1C00020E2620E711C34E1A312B2CFFF92EF92E3
:10F1D0001F920F931F921F9389EA9DE19F938F9334
:10F1E0000F949AA80FB6F894DEBF0FBECDBF93E47C
:10F1F000E916F10414F40C9405861F920F931F92E4
:10F200001F938AED9DE19F938F930F949AA81A5FA5
:10F21000E12EF12CA0E1EA1AF108E6E0EE0CFF1C69
:10F22000EA95E1F76896EEADFFAD6897EE0EFF1E2A
:10F230000A5FC02ED12CF0E1CF1AD108F6E0CC0C39
:10F24000DD1CFA95E1F7E0962EAD3FADE097C20EDA
:10F25000D31EA0963FADA0973F936F966FAD6F976B
:10F260006F93DF92CF92FF92EF9289EC9DE19F9393
:10F270008F930F949AA800E028EC30E0A0964EAD52
:10F280005FADA097B601C7010F9403240FB6F894A1
:10F29000DEBF0FBECDBF81E0D2011D922D01B2E0D5
:10F2A0004B16BDE05B06C1F781110C94088610E097
:10F2B00086E39EE19F938F930F949AA80F94033D4A
:10F2C00080916E00846080936E00EF9A80916F0051
:10F2D000826080936F0098E288E10FB6F894A89559
:10F2E000809360000FBE909360001092070D109203
:10F2F000060D1092050D1092040D1092030D109240
:10F30000020D0F900F90112311F40C94A38420E0B0
:10F3100030E0A9016C96EEADFFAD6C976181728112
:10F32000838194810F9426A42091DF0F3091E00F08
:10F330004091E10F5091E20F0F941AB26C96AEAD6E
:10F34000BFAD6C9711966D937D938D939C9314979D
:10F35000C090E30FD090E40FE090E50FF090E60F3F
:10F3600020E030E0A90115966D917D918D919C91E1
:10F3700018970F9426A4A70196010F941AB26C96C1
:10F38000EEADFFAD6C97658376838783908720E031
:10F3900030E040E850ECC701B6010F942EA987FF7A
:10F3A0000CC080E090E0A0E8B0EC8093E30F909375
:10F3B000E40FA093E50FB093E60F20E030E040E4C7
:10F3C00050E46091E70F7091E80F8091E90F909100
:10F3D000EA0F0F941AB26093E70F7093E80F8093CF
:10F3E000E90F9093EA0FAE968CAD9DADAEADBFAD7B
:10F3F000AE970196A11DB11DAE968CAF9DAFAEAF7D
:10F40000BFAFAE97A896AEADBFADA8971896A89619
:10F41000BFAFAEAFA8976C96EEADFFAD6C973896C8
:10F420006C96FFAFEEAF6C97AE968CAD9DADAEAD6A
:10F43000BFADAE970597A105B10509F086C980E07B
:10F4400090E00E94A59420E030E040E950EC60910B
:10F4500068157091691580916A1590916B150F94DC
:10F460002EA987FF43C0E9EEFEE184918F01882336
:10F4700039F00E947DFA0F5F1F4FF8018491F7CF9A
:10F480008AE00E947DFAE7EBFEE184918F018823F8
:10F4900039F00E947DFA0F5F1F4FF8018491F7CF7A
:10F4A000609168157091691580916A1590916B153E
:10F4B00042E00E9420FBE3EBFEE184918F01882370
:10F4C00039F00E947DFA0F5F1F4FF8018491F7CF4A
:10F4D00042E060E070E080E990EC0E9420FB0E9436
:10F4E000B2FBF2E0AF96FFAFAF9703C0AF961FAE8F
:10F4F000AF97109294151092951510929615109240
:10F500009715109298151092991510929A151092BD
:10F510009B1524E6EB962FAFEB976E961CAE1DAEB7
:10F520001EAE1FAE6E976A961CAE1DAE1EAE1FAE0F
:10F530006A97CE01019664969FAF8EAF6497DE0105
:10F54000AF5BBF4F6696BFAFAEAF66976A966CADC6
:10F550007DAD8EAD9FAD6A970F9405B3AA966CAF43
:10F560007DAF8EAF9FAFAA976A966CAD7DAD8EAD25
:10F570009FAD6A970F9494B5C457DF4F6883798322
:10F580008A839B83CC58D0406E966CAD7DAD8EAD9A
:10F590009FAD6E970F9405B3C057DF4F6883798393
:10F5A0008A839B83C059D0406E966CAD7DAD8EAD85
:10F5B0009FAD6E970F9494B5CC56DF4F68837983D7
:10F5C0008A839B83C459D0406496EEADFFAD6497A7
:10F5D00020E411922A95E9F76696AEADBFAD669725
:10F5E000E0E11D92EA95E9F780E090E00E94A594A1
:10F5F0008091941590919515A0919615B0919715BD
:10F60000C655DF4F88839983AA83BB83CA5AD040EB
:10F610008091981590919915A0919A15B0919B158C
:10F62000C255DF4F88839983AA83BB83CE5AD040CB
:10F63000DE01AF5BBF4FC856DF4FB983A883C859FF
:10F64000D040FE013196AC96FFAFEEAFAC9700E034
:10F65000CC56DF4F88819981AA81BB81C459D040A3
:10F66000B058E6968CAF9DAFAEAFBFAFE697C05730
:10F67000DF4F88819981AA81BB81C059D040B058A1
:10F68000EA968CAF9DAFAEAFBFAFEA97C457DF4FDE
:10F6900088819981AA81BB81CC58D040B058C2588A
:10F6A000DF4F88839983AA83BB83CE57D040AC9623
:10F6B0002EAC3FACAC9710E063E6462E65E1562ECB
:10F6C00074E0772EC12CD12C7601013011F40C940A
:10F6D0008686113011F40C949286002311F10230C9
:10F6E00081F4D20111962D913D914D915C91149729
:10F6F000C258DF4F688179818A819B81CE57D04083
:10F700000BC0F2012581368147815085EA966CADA8
:10F710007DAD8EAD9FADEA970F9426A44B015C01A1
:10F7200006C0812C912C50E8A52E5FE3B52E112345
:10F7300001F1123081F4D20111962D913D914D913C
:10F740005C911497C258DF4F688179818A819B81CF
:10F75000CE57D0400BC0F2012581368147815085BC
:10F76000EA966CAD7DAD8EAD9FADEA970F9426A461
:10F7700004C060E070E080E89FE39B01AC01C5013C
:10F78000B4010F9426A49B01AC01C701B6010F94EC
:10F790001AB26B017C010023E1F11123D1F1023097
:10F7A00011F00C946686D20111962D913D914D91E8
:10F7B0005C911497AA966CAD7DAD8EAD9FADAA9766
:10F7C0000F9426A44B015C01113011F40C94808637
:10F7D000123011F00C947386D20111962D913D9147
:10F7E0004D915C911497AA966CAD7DAD8EAD9FAD99
:10F7F000AA970F9426A49B01AC01C501B4010F94F4
:10F8000026A49B01AC01C701B6010F941AB26B018B
:10F810007C017A94F8E04F0E511C711056CFD10143
:10F82000CD92DD92ED92FD921D011F5F143009F023
:10F8300043CF33E6232E35E1332EEAEEFEE1A096E8
:10F84000FFAFEEAFA097CA57DF4F1882C658D0401F
:10F85000C456DF4F1882CC59D040C056DF4F1882B3
:10F86000C05AD04010E0002321F1013049F10230AC
:10F8700081F4D10111962D913D914D915C91149798
:10F88000C258DF4F688179818A819B81CE57D040F1
:10F890000BC0F1012581368147815085EA966CAD18
:10F8A0007DAD8EAD9FADEA970F9426A44B015C0110
:10F8B0000AC0812C912C20E8A22E2FE3B22E03C087
:10F8C000812C912C5401D10111964D905D906D9039
:10F8D0007C901497A3019201AA966CAD7DAD8EAD7C
:10F8E0009FADAA970F9426A46B017C01D1011596B8
:10F8F0008D919D910D90BC91A02DA6968CAF9DAF42
:10F90000AEAFBFAFA697A096EEADFFADA097859125
:10F910009591A591B491CC55DF4F88839983AA83A3
:10F92000BB83C45AD040A6962CAD3DAD4EAD5FAD65
:10F93000A697CC56DF4F688179818A819B81C45913
:10F94000D0400F9426A49B01AC01C701B6010F94CF
:10F9500019B2C655DF4F288139814A815B81CA5A65
:10F96000D0400F941AB2CC55DF4F288139814A819B
:10F970005B81C45AD0400F9419B2A50194010F9431
:10F9800026A4CA57DF4F2881C658D040C456DF4F3F
:10F990003881CC59D040C056DF4F4881C05AD04042
:10F9A000512F0F941AB2CA57DF4F688379838A8325
:10F9B0009B83C658D0400023A9F00130B9F0023033
:10F9C000D9F0A6962CAD3DAD4EAD5FADA697E696AF
:10F9D0006CAD7DAD8EAD9FADE6970F9426A46B0107
:10F9E0007C010AC0C12CD12C760106C0C12CD12CBF
:10F9F00090E8E92E9FE3F92EA096EEADFFADA0971B
:10FA0000349685909590A590B490A3019201C45727
:10FA1000DF4F688179818A819B81CC58D0400F94D7
:10FA200026A42B013C01A6962CAD3DAD4EAD5FAD9D
:10FA3000A697C057DF4F688179818A819B81C05921
:10FA4000D0400F9426A49B01AC01C301B2010F94D6
:10FA50001AB2C255DF4F288139814A815B81CE5A63
:10FA6000D0400F941AB2A50194010F9419B2A701C6
:10FA700096010F9426A4CA57DF4F288139814A8105
:10FA80005B81C658D0400F941AB2CA57DF4F6883C3
:10FA9000C658D040C456DF4F7883CC59D040C056AA
:10FAA000DF4F8883C05AD040192FA096AEADBFADAE
:10FAB000A0971896A096BFAFAEAFA097B8E02B0E58
:10FAC000311CE3E82E16E5E13E0609F0CCCEDC0160
:10FAD000CB01B058C856DF4FE881F981C859D040F2
:10FAE00081939193A193B193C856DF4FF983E88333
:10FAF000C859D0400F5FAC962EAD3FADAC97205F9C
:10FB00003F4FAC963FAF2EAFAC97043009F0CFCD4E
:10FB100025968CAD9DADAEADBFAD2597AA968CAFA9
:10FB20009DAFAEAFBFAFAA978D819E81AF81B885E3
:10FB3000AE968CAF9DAFAEAFBFAFAE9789859A85BD
:10FB4000AB85BC85A6968CAF9DAFAEAFBFAFA69779
:10FB50008D859E85AF85B889E6968CAF9DAFAEAF9B
:10FB6000BFAFE69789819A81AB81BC81EA968CAF61
:10FB70009DAFAEAFBFAFEA9729968CAD9DADAEAD50
:10FB8000BFAD2997C258DF4F88839983AA83BB836F
:10FB9000CE57D04089899A89AB89BC89C457DF4F39
:10FBA00088839983AA83BB83CC58D040898D9A8D52
:10FBB000AB8DBC8DC057DF4F88839983AA83BB83ED
:10FBC000C059D0408D8D9E8DAF8DB8A1CC56DF4FE2
:10FBD00088839983AA83BB83C459D0408D899E8929
:10FBE000AF89B88DC856DF4F88839983AA83BB83BA
:10FBF000C859D0402D968CAD9DADAEADBFAD2D9703
:10FC0000CA57DF4F88839983AA83BB83C658D040E5
:10FC100089A19AA1ABA1BCA1C456DF4F8883998367
:10FC2000AA83BB83CC59D0408DA19EA1AFA1B8A51A
:10FC3000C056DF4F88839983AA83BB83C05AD040C4
:10FC40008DA59EA5AFA5B8A9CC55DF4F8883998314
:10FC5000AA83BB83C45AD04089A59AA5ABA5BCA5ED
:10FC6000CE54DF4F88839983AA83BB83C25BD04085
:10FC700061968CAD9DADAEADBFAD6197CA54DF4FFF
:10FC800088839983AA83BB83C65BD04089A99AA93C
:10FC9000ABA9BCA9C654DF4F88839983AA83BB83D1
:10FCA000CA5BD0408DA99EA9AFA9B8ADC254DF4FA1
:10FCB00088839983AA83BB83CE5BD04089AD9AADFC
:10FCC000ABADBCADCE53DF4F88839983AA83BB8392
:10FCD000C25CD04021968CAD9DADAEADBFAD21973D
:10FCE000CA53DF4F88839983AA83BB83C65CD04005
:10FCF00014E6C12CD12C76014601570126013701AB
:10FD0000A3019201AE966CAD7DAD8EAD9FADAE9769
:10FD10000F9426A49B01AC01AA966CAD7DAD8EAD6F
:10FD20009FADAA970F9419B22B013C01A501940134
:10FD3000A6966CAD7DAD8EAD9FADA6970F9426A413
:10FD40009B01AC01C301B2010F9419B22B013C011C
:10FD5000A7019601E6966CAD7DAD8EAD9FADE697A1
:10FD60000F9426A49B01AC01C301B2010F9419B2F8
:10FD7000EA962CAD3DAD4EAD5FADEA970F9408B35A
:10FD8000A2966CAF7DAF8EAF9FAFA297C457DF4FE7
:10FD9000288139814A815B81CC58D0400F9426A4B8
:10FDA0009B01AC01C258DF4F688179818A819B81B8
:10FDB000CE57D0400F9419B22B013C01A5019401FC
:10FDC000C057DF4F688179818A819B81C059D040BB
:10FDD0000F9426A49B01AC01C301B2010F9419B288
:10FDE0004B015C01A7019601CC56DF4F68817981F8
:10FDF0008A819B81C459D0400F9426A49B01AC01F9
:10FE0000C501B4010F9419B2C856DF4F288139815A
:10FE10004A815B81C859D0400F9408B32B013C0143
:10FE2000C456DF4F288139814A815B81CC59D0404B
:10FE3000A2966CAD7DAD8EAD9FADA2970F9426A41A
:10FE40009B01AC01CA57DF4F688179818A819B8110
:10FE5000C658D0400F9419B24B015C01C056DF4F19
:10FE6000288139814A815B81C05AD040C301B201E7
:10FE70000F9426A49B01AC01C501B4010F9419B2E3
:10FE80004B015C01A7019601CC55DF4F6881798158
:10FE90008A819B81C45AD0400F9426A49B01AC0157
:10FEA000C501B4010F9419B2CE54DF4F28813981B6
:10FEB0004A815B81C25BD0400F9408B34B015C0167
:10FEC000C654DF4F288139814A815B81CA5BD040AB
:10FED000A2966CAD7DAD8EAD9FADA2970F9426A47A
:10FEE0009B01AC01CA54DF4F688179818A819B8173
:10FEF000C65BD0400F9419B26B017C01C254DF4F36
:10FF0000288139814A815B81CE5BD040C301B20137
:10FF10000F9426A49B01AC01C701B6010F9419B23E
:10FF20006B017C01CE53DF4F288139814A815B818F
:10FF3000C25CD040C501B4010F9426A49B01AC0162
:10FF4000C701B6010F9419B2CA53DF4F2881398116
:10FF50004A815B81C65CD0400F9408B36B017C0181
:10FF6000115009F0CDCEA2962CAD3DAD4EAD5FAD9A
:10FF7000A297C655DF4F688179818A819B81CA5AD1
:10FF8000D0400F941AB26093941570939515809396
:10FF9000961590939715A3019201C255DF4F688182
:10FFA00079818A819B81CE5AD0400F941AB2609396
:10FFB00098157093991580939A1590939B15A501A8
:10FFC00094016A966CAD7DAD8EAD9FAD6A970F942E
:10FFD0001AB26A966CAF7DAF8EAF9FAF6A97A701DA
:10FFE00096016E966CAD7DAD8EAD9FAD6E970F9404
:10FFF0001AB26E966CAF7DAF8EAF9FAF6E97EB96D9
:020000021000EC
:100000009FADEB979150EB969FAFEB9791119ECAE6
:100010006A966CAD7DAD8EAD9FAD6A970F9405B3BA
:10002000609384157093851580938615909387153A
:100030006A966CAD7DAD8EAD9FAD6A970F9494B509
:10004000609388157093891580938A1590938B150A
:100050006E966CAD7DAD8EAD9FAD6E970F9494B5E1
:10006000DC01CB01B05880938C1590938D15A09333
:100070008E15B0938F156E966CAD7DAD8EAD9FAD28
:100080006E970F9405B360939015709391158093BC
:100090009215909393156A962CAD3DAD4EAD5FAD24
:1000A0006A976E966CAD7DAD8EAD9FAD6E970F94D9
:1000B00019B26B017C01E894F7F8B701A60180E65C
:1000C0009FE00F94B2B12FE132E449E05BE3C70156
:1000D000B6010F9465B418166CF425E33AEF4EE8B8
:1000E0005BE3C701B6010F9465B4181634F001E064
:1000F00010E005C000E010E002C002E010E025E3DF
:100100003AEF4EE85BE36A966CAD7DAD8EAD9FAD88
:100110006A979F770F9465B418167CF025E33AEF41
:100120004EE85BE36E966CAD7DAD8EAD9FAD6E9788
:100130009F770F9465B4181614F402E010E08091D4
:10014000841590918515A0918615B0918715AE966E
:100150008CAF9DAFAEAFBFAFAE9780918C15909135
:100160008D15A0918E15B0918F15A6968CAF9DAF71
:10017000AEAFBFAFA6978091941590919515A091C1
:100180009615B0919715EE968CAF9DAFAEAFBFAF01
:10019000EE978091881590918915A0918A15B0915C
:1001A0008B15E6968CAF9DAFAEAFBFAFE697809153
:1001B000901590919115A0919215B0919315EA9692
:1001C0008CAF9DAFAEAFBFAFEA978091981590917D
:1001D0009915A0919A15B0919B15C258DF4F88834D
:1001E0009983AA83BB83CE57D040AAEEBEE1A096E6
:1001F000BFAFAEAFA09783E6282E85E1382EF10180
:1002000081809280A380B48085819681A781B0850A
:10021000AA968CAF9DAFAEAFBFAFAA97A096EEAD3A
:10022000FFADA097C590D590E590F490A5019401FD
:10023000AE966CAD7DAD8EAD9FADAE970F9426A4FE
:100240002B013C01AA962CAD3DAD4EAD5FADAA97FA
:10025000A6966CAD7DAD8EAD9FADA6970F9426A4EE
:100260009B01AC01C301B2010F941AB2EE962CAD02
:100270003DAD4EAD5FADEE970F941AB29B01AC0150
:10028000C701B6010F9419B26B017C01A096EEADC7
:10029000FFADA09734964590559065907490E69682
:1002A0002CAD3DAD4EAD5FADE697C501B4010F94E9
:1002B00026A44B015C01EA962CAD3DAD4EAD5FAD81
:1002C000EA97AA966CAD7DAD8EAD9FADAA970F94BF
:1002D00026A49B01AC01C501B4010F941AB2C25807
:1002E000DF4F288139814A815B81CE57D0400F94FE
:1002F0001AB29B01AC01C301B2010F9419B24B01B8
:100300005C01A7019601C701B6010F9426A46B01F9
:100310007C01A5019401C501B4010F9426A49B01A1
:10032000AC01C701B6010F941AB20F949FB52DEC22
:100330003CEC4CE45FE30F9465B4181614F40EEF34
:100340001FEFB8E02B0E311CA096EEADFFADA097CD
:100350003896A096FFAFEEAFA09723E835E12215BF
:10036000330509F04CCF0115110509F07AC16E96DD
:100370002CAD3DAD4EAD5FAD6E976A966CAD7DAD6B
:100380008EAD9FAD6A970F941AB220E030E040E046
:100390005FE30F9426A46B017C010F9405B32B013E
:1003A0003C01609384157093851580938615909316
:1003B0008715C701B6010F9494B56E966CAF7DAFEB
:1003C0008EAF9FAF6E976093881570938915809359
:1003D0008A1590938B15DC01CB01B058AA968CAF8F
:1003E0009DAFAEAFBFAFAA9780938C1590938D153C
:1003F000A0938E15B0938F15409290155092911541
:100400006092921570929315109294151092951512
:1004100010929615109297151092981510929915A2
:1004200010929A1510929B15A2961CAE1DAE1EAE90
:100430001FAEA2976A961CAE1DAE1EAE1FAE6A9787
:10044000CE57DF4FA881B981C258D04011968D9008
:100450009D90AD90BC90149715968D919D910D90A7
:10046000BC91A02DAE968CAF9DAFAEAFBFAFAE9797
:10047000C657DF4FE881F981CA58D040C590D59062
:10048000E590F490A5019401C301B2010F9426A454
:10049000A6966CAF7DAF8EAF9FAFA697AE962CADF4
:1004A0003DAD4EAD5FADAE97AA966CAD7DAD8EAD58
:1004B0009FADAA970F9426A49B01AC01A6966CADA4
:1004C0007DAD8EAD9FADA6970F941AB29B01AC0186
:1004D000C701B6010F9419B220919415309195156A
:1004E00040919615509197150F941AB26B017C01AB
:1004F0006093941570939515809396159093971526
:1005000020E030E040E85FE36A966CAD7DAD8EADF3
:100510009FAD6A970F941AB26A966CAF7DAF8EAF9B
:100520009FAF6A97C657DF4FE881F981CA58D0401C
:10053000349685919591A591B491A6968CAF9DAF77
:10054000AEAFBFAFA697A50194016E966CAD7DAD21
:100550008EAD9FAD6E970F9426A44B015C01AE96B5
:100560002CAD3DAD4EAD5FADAE97C301B2010F9462
:1005700026A49B01AC01C501B4010F941AB29B01E2
:10058000AC01A6966CAD7DAD8EAD9FADA6970F94D8
:1005900019B2209198153091991540919A15509162
:1005A0009B150F941AB24B015C01609398157093E0
:1005B000991580939A1590939B1520E030E040E8C0
:1005C0005FE3A2966CAD7DAD8EAD9FADA2970F940B
:1005D0001AB2A2966CAF7DAF8EAF9FAFA297CE57E7
:1005E000DF4FA881B981C258D0401896CE57DF4F4F
:1005F000B983A883C258D040C657DF4FE881F9813C
:10060000CA58D0403896C657DF4FF983E883CA5896
:10061000D0402A163B0609F013CF6A962CAD3DADAB
:100620004EAD5FAD6A97C701B6010F9408B36093F2
:100630009415709395158093961590939715A2969F
:100640002CAD3DAD4EAD5FADA297C501B4010F9489
:1006500008B3609398157093991580939A159093A9
:100660009B158090841590908515A0908615B0906C
:10067000871540909015509091156090921570904C
:1006800093158091881590918915A0918A15B09144
:100690008B156E968CAF9DAFAEAFBFAF6E9780914E
:1006A0008C1590918D15A0918E15B0918F156A962D
:1006B0008CAF9DAFAEAFBFAF6A97A3019201C501EA
:1006C000B4010F9426A46B017C016A962CAD3DAD5C
:1006D0004EAD5FAD6A976E966CAD7DAD8EAD9FAD44
:1006E0006E970F9426A49B01AC01C701B6010F942D
:1006F00019B26B017C019B01AC01C301B2010F94E3
:1007000008B32B013C016A966CAD7DAD8EAD9FADFB
:100710006A979058A70196010F9408B36A966CAF38
:100720007DAF8EAF9FAF6A976E966CAD7DAD8EAD8F
:100730009FAD6E979058A70196010F9408B3CE57BE
:10074000DF4F688379838A839B83C258D040A70197
:100750009601C501B4010F9408B36B017C01809030
:10076000941590909515A0909615B090971580913E
:10077000981590919915A0919A15B0919B156E9628
:100780008CAF9DAFAEAFBFAF6E97409284155092C5
:1007900085156092861570928715CE57DF4F888138
:1007A0009981AA81BB81C258D040809388159093CB
:1007B0008915A0938A15B0938B156A968CAD9DAD63
:1007C000AEADBFAD6A9780938C1590938D15A093B5
:1007D0008E15B0938F15C0929015D0929115E0921E
:1007E0009215F0929315C301B2019058A50194019E
:1007F0000F9426A42B013C016E962CAD3DAD4EAD61
:100800005FAD6E976A966CAD7DAD8EAD9FAD6A970C
:100810000F9426A49B01AC01C301B2010F9419B23D
:1008200060939415709395158093961590939715F2
:10083000CE57DF4F688179818A819B81C258D04031
:100840009058A50194010F9426A44B015C016E966B
:100850002CAD3DAD4EAD5FAD6E97C701B6010F94A7
:1008600026A49B01AC01C501B4010F9419B2609399
:1008700098157093991580939A1590939B1580E025
:1008800090E00E94A59417FD53C044E955E16CE83F
:1008900075E184E895E10E9441A140919415509141
:1008A0009515609196157091971585EE9FE00F94C0
:1008B000B2B1409198155091991560919A15709127
:1008C0009B1589EE9FE00F94B2B140918415509131
:1008D000851560918615709187158DED9FE00F94B9
:1008E000B2B1409188155091891560918A15709127
:1008F0008B1581EE9FE00F94B2B140918C15509111
:100900008D1560918E1570918F1585ED9FE00F9478
:10091000B2B14091901550919115609192157091DE
:10092000931589ED9FE00F94B2B10E94C6A009C053
:100930000E3F9FEF190729F4AF96AFADAF97A230E6
:1009400049F038010BC0AF961FAEAF9766246A948A
:10095000762C04C0BEEF6B2E77247A94C855DF4FF7
:1009600088819981C85AD0400E94F9F380E090E0D4
:10097000A0EAB0E48093E70F9093E80FA093E90F0B
:10098000B093EA0F2091E30F3091E40F4091E50F0F
:100990005091E60F6091DF0F7091E00F8091E10FB1
:1009A0009091E20FEAE1FDE0FF93EF93812C912C0F
:1009B000E0EAAE2EE1E4BE2EFBEECF2EFFE0DF2E0E
:1009C000E12CF12C00EA10E40F94C52E0F94AB7FBC
:1009D0000F900F9077FC22C020E030E046E153E416
:1009E0006091E70F7091E80F8091E90F9091EA0F05
:1009F0000F941AB26093E70F7093E80F8093E90F9A
:100A00009093EA0F65E575E585E591E40E9458A0AD
:100A10008AE59AE10F9479050E94D8A881E00E94A6
:100A200063AD82E00E945CA5BFEF6B167B0631F4DC
:100A30008DE19AE10F94790510E04BC0EEEF6E1650
:100A4000EFEF7E0681F4AF96FFADAF97FF2329F05D
:100A5000F23031F086ED98E1EDCF8BE599E1EACF08
:100A60008BE199E1E7CFAF962FADAF97211107C08A
:100A700033E06316710498F08BE599E117C0AF96E7
:100A80006FADAF97623019F488ED99E102C08EE83E
:100A900099E10F9479051614170454F309C0F30172
:100AA000EE0FFF1FEB52FD4F808191810F9479056E
:100AB0006720609409F286EE0E94A4F68FE59FE01D
:100AC0000F948EB1813021F08DE89AE10F94790571
:100AD00011E00F9436172BC185E29FE10F94790541
:100AE00010E025C183E0821B282F0C9439742981E2
:100AF0003A812059374F3A8329830C949875F0E94D
:100B0000CF1AF1E0DF0A0C94DA74E7968FADE7971D
:100B1000E8969FADE8970C9479768E7F0C94C57615
:100B200080E4482E512C612C712C0C94DB7687E1EB
:100B300090E00C94EF768F3F910509F014F40C943B
:100B4000F7768FEF90E00C94F7768B7F0C94FF761E
:100B5000B0E6EB16B9E0FB0614F00C940E7784E0D7
:100B60000E94ECB9EFEFEE1AFE0A0C940E77C60164
:100B70000C942E778150883011F00C9408780C94E6
:100B80000F7800E00C941D7880E090E00C9442789F
:100B9000EBE0BE1611F40C94B878222311F02B3040
:100BA00039F4E396FFADE397F83010F00C94BE787B
:100BB000B101620F731F6E56784FFB01F081A3964F
:100BC000FFAFA397E896EEADFFADE897C080D18068
:100BD00061E070E0022E02C0660F771F0A94E2F710
:100BE0006C217D21672B31F0A396FFADA397F131E6
:100BF00048F005C0A3966FADA397613118F4019634
:100C00000C94BE7801970C94BE7880E00C944C79DB
:100C100084EF91E00F944925882311F40C945779BF
:100C200014E0812C912C5401C12CD12C760188EE3A
:100C300093E00F944925882311F40C9457798091FF
:100C4000CF0F9091D00FA091D10FB091D20F092E5C
:100C5000000CAA0BBB0BC80ED91EEA1EFB1E80910E
:100C6000D30F9091D40FA091D50FB091D60F092E2C
:100C7000000CAA0BBB0B880E991EAA1EBB1E11509E
:100C8000B1F64090D70F5090D80F6090D90F709068
:100C9000DA0FC501B40122E096958795779567959F
:100CA0002A95D1F732E0F694E794D794C7943A9511
:100CB000D1F700E028EC30E0A201C6010F94032434
:100CC00011E00C94587981E00C949875F20125811B
:100CD000368147815085E6966CAD7DAD8EAD9FAD7A
:100CE000E6970C94E07BF20125813681478150859F
:100CF000E6966CAD7DAD8EAD9FADE6970C94F97B1D
:100D000060E070E080E89FE30C94FB7B112311F41A
:100D10000C94097C812C912C40E8A42E4FE3B42E36
:100D20000C94E47B01110C94CF7B0C94097C81E042
:100D30000E9463AD80E00F94DA62812FC753DF4FCA
:100D40000FB6F894DEBF0FBECDBFDF91CF911F91DC
:100D50000F91FF90EF90DF90CF90BF90AF909F905A
:100D60008F907F906F905F904F903F902F9008955D
:100D70003F924F925F926F927F928F929F92AF922B
:100D8000BF92CF92DF92EF92FF920F931F93CF9378
:100D9000DF93CDB7DEB7C855D1090FB6F894DEBFE3
:100DA0000FBECDBFB82E81E00E9463AD82E00E94ED
:100DB0005CA582EF9FE10F94FC2785EA9FE00F94EA
:100DC0008EB1A82E8DE99FE00F9496B16093DF0F4E
:100DD0007093E00F8093E10F9093E20F81EA9FE020
:100DE0000F9496B16093E30F7093E40F8093E50F37
:100DF0009093E60F22E0A21209C08AED9EE00F94C4
:100E000096B16B017C0188ED9EE008C08DE89FE003
:100E10000F9496B16B017C0183E79FE00F949BB127
:100E200067E074E0681B790BE4E076956795EA95D6
:100E3000E1F780E090E00F9432A920912F103091DB
:100E4000301040913110509132100F9408B32B01A3
:100E50003C012AE037ED43E25FE3C701B6010F949E
:100E60001AB29B01AC01C301B2010F941AB2609394
:100E7000E70F7093E80F8093E90F9093EA0F82E7F2
:100E80009FE00F948EB1882391F18EE69FE00F943E
:100E900096B16093EB0F7093EC0F8093ED0F9093EE
:100EA000EE0F88ED91E29F938F93CE0101967C0126
:100EB0009F938F930F94F2A8F70101900020E9F718
:100EC0008F01015011096091EB0F7091EC0F80912F
:100ED000ED0F9091EE0F23E046E00F94DAA460E06E
:100EE000C7010F94685C0F900F900F900F9080E1F6
:100EF000EFEDFFE0A8E0BDE001900D928A95E1F7EB
:100F0000E6EAF1E284918F01882339F00E947DFAAC
:100F10000F5F1F4FF8018491F7CF8091EA0F8F93F5
:100F20008091E90F8F938091E80F8F938091E70F65
:100F30008F938091E60F8F938091E50F8F9380912F
:100F4000E40F8F938091E30F8F938091E20F8F9343
:100F50008091E10F8F938091E00F8F938091DF0F4D
:100F60008F9388E290E29F938F930F949AA80E94A8
:100F7000B3A4109263150FB6F894DEBF0FBECDBFB9
:100F800055E7E52E5FE0F52E912C63E0762E6E019D
:100F90003FE1C30ED11C6624639477E0872E892D30
:100FA000672D0F94B8B6082F592E42E050E0B701D4
:100FB000C6010F947EB16F8D78A16115710511F096
:100FC00060926315282D020380011124050D111D67
:100FD00057FC1A95000F111F000F111F0D591A4EC3
:100FE000072E000C880B990B0F9434A92FE632E1E1
:100FF00043E85AE30F9426A4F80161837283838344
:1010000094839394F2E0EF0EF11C29E09212C7CF83
:101010008091631581110F94D1490E94A3DBE09068
:10102000E70FF090E80F0091E90F1091EA0F20917F
:10103000E30F3091E40F4091E50F5091E60F60917E
:10104000DF0F7091E00F8091E10F9091E20F0F940C
:101050004A4281E080931B0D179880931C0D1698CF
:1010600080931D0D1598E4E7F1E284918F018823A8
:1010700039F00E947DFA0F5F1F4FF8018491F7CF7E
:1010800082E00F94987F962E872E782E692E81E02D
:101090000F94987F162F072FF82EE92E80E00F94DB
:1010A000987F6F927F928F929F92EF92FF920F9311
:1010B0001F939F938F937F936F938FE490E29F93FF
:1010C0008F930F949AA88CE89FE00F948EB1E091D3
:1010D0001A0DF0E0EE0FFF1FE05AFA4E90E09183F8
:1010E00080838BE89FE00F948EB190E090931F0D6A
:1010F00080931E0D88EE9EE00F9496B160932902B6
:1011000070932A0280932B0290932C028EED9EE026
:101110000F949BB190936302809362020FB6F89490
:10112000DEBF0FBECDBF32E0A316A9F020E030E055
:1011300048EC51E46091E70F7091E80F8091E90F5E
:101140009091EA0F0F942EA987FF05C061E087EB0D
:1011500092E20F94685C61E08FEA92E20F94685C1F
:10116000E0911A0DF0E0EE0FFF1FE05AFA4E818178
:101170008F9380818F9386EA92E29F938F93DF9281
:10118000CF920F94F2A860E0C6010F94685C809142
:101190001F0D8F9380911E0D8F938DE992E29F9387
:1011A0008F93DF92CF920F94F2A860E0C6010F9464
:1011B000685C61E089E992E20F94685C0FB6F8948C
:1011C000DEBF0FBECDBFB11005C061E08EE892E278
:1011D0000F94685C61E081E792E20F94685C809113
:1011E000E60F8F938091E50F8F938091E40F8F939B
:1011F0008091E30F8F938091E20F8F938091E10FA5
:101200008F938091E00F8F938091DF0F8F938AEA05
:1012100090E29F938F930F949AA888E89FE00F9491
:101220008EB1382EBE01695A7F4F89E89FE00E9437
:1012300035C6E7E6F2E284910FB6F894DEBF0FBE42
:10124000CDBF07E612E2882339F00E947DFA0F5FD6
:101250001F4FF8018491F7CF69966EAD7FAD699706
:10126000072E000C880B990B0E9406FB0E94B2FB14
:101270008AE59FE00F948EB1482E512C682F70E0C4
:1012800080E090E00E9406FB0E94B2FB93EDC92E25
:101290009EE0D92E0AE01FE0A12CB12CA414B504C5
:1012A0003CF54E01FAE48F0E911C380128E0620EE5
:1012B000711C7401C8010F948EB1F40181934F0128
:1012C0000F5F1F4F60167106A9F7F7011086C7015F
:1012D0000E94B6FBB701C6010F9473B7C7010F9404
:1012E0009916FFEFAF1ABF0A29E0C20ED11CD6CF64
:1012F0008E01035C1F4F580185E9E82E8FE0F82E20
:10130000D02EC12EC7010F948EB1F50181935F01DC
:10131000FFEFEF1AFF0A2DE9E2162FE0F20691F730
:1013200026961FAE2697F80181918F01882319F028
:101330000E947DFAF8CF62E672E28D2D9C2D0F940B
:101340008DA7CF92DF928BE592E29F938F938E01D0
:101350000F5F1F4F1F930F930F94F2A860E0C80117
:101360000F94685C81E99FE00F9496B1D62EC72E4A
:10137000B82EA92EE0E4F2E284910F900F900F9026
:101380000F900F900F907F01882341F00E947DFA0B
:10139000FFEFEF1AFF0AF7018491F6CF4AE06D2DB7
:1013A0007C2D8B2D9A2D0E9495FA0E94B2FB61E054
:1013B0008CE392E20F94685C67E372E2C8010F94D9
:1013C00098A78DE99FE00F9496B167966CAF7DAFBB
:1013D0008EAF9FAF6797CE018D5A9F4F0F94705677
:1013E000BC01C8010F9454B764E372E2C8010F94C2
:1013F0008DA781EA9FE00F9496B167966CAF7DAFA1
:101400008EAF9FAF6797CE018D5A9F4F0F94705646
:10141000BC01C8010F9454B76DE272E2C8010F9489
:101420008DA760E0C8010F94685C68E272E2C801B1
:101430000F9498A78DE89FE00F9496B167966CAFD4
:101440007DAF8EAF9FAF6797CE018D5A9F4F0F94A0
:101450007056BC01C8010F9454B760E0C8010F94E6
:10146000685C61E08AE092E20F94685C69968FADF7
:1014700069978F9368968FAD68978F9383E092E218
:101480009F938F931F930F930F94F2A860E0C8016E
:101490000F94685C82E79FE00F948EB10F900F90DD
:1014A0000F900F900F900F90882329F061E08FEF3D
:1014B00091E20F94685C68EF71E2C8010F9498A7FD
:1014C000832D90E065969FAF8EAF6597CE018D5AC4
:1014D0009F4F0F943156BC01C8010F9454B760E080
:1014E000C8010F94685CAF92BF92CF92DF928FEEEB
:1014F00091E29F938F931F930F930F94F2A860E054
:10150000C8010F94685C61E089EE91E20F94685C19
:1015100061E08EED91E20F94685C8091EE0F8F9305
:101520008091ED0F8F938091EC0F8F938091EB0F53
:101530008F938091EA0F8F938091E90F8F93809121
:10154000E80F8F938091E70F8F9389E790E29F9345
:101550008F930F949AA80FB6F894DEBF0FBECDBF3D
:10156000C85ADF4F0FB6F894DEBF0FBECDBFDF9174
:10157000CF911F910F91FF90EF90DF90CF90BF9090
:10158000AF909F908F907F906F905F904F903F9023
:1015900008951F920F920FB60F9211240BB60F925F
:1015A0002F923F924F925F926F927F928F929F9273
:1015B000AF92BF92CF92DF92EF92FF920F931F9361
:1015C0002F933F934F935F936F937F938F939F934B
:1015D000AF93BF93EF93FF93CF93DF93CDB7DEB776
:1015E0006197DEBFCDBFEC98EFE6F1E284918F0109
:1015F000882339F00E947DFA0F5F1F4FF801849114
:10160000F7CF8AE00E947DFA80915716882309F46B
:1016100078C285EA9FE00F948EB1811172C20F9457
:101620004E866D877E878F87988BF0915716F98B42
:10163000179A10921B0D169A10921C0D64E182E00D
:101640000F94E89664E182E00F94D79664E183E01A
:101650000F94E89664E183E00F94D79683E40E94A8
:10166000F09E98878F834090391350903A13609082
:101670003B1370903C130E94F5B9481A590A61084F
:1016800071080F946157481A590A6108710877FE6A
:1016900003C0412C512C320190910C0780910B0713
:1016A000981799F0E0910B0727E5E29FF0011124CC
:1016B000EE56F84F20E030E040E752E462A173A11B
:1016C00084A195A10F9426A408C060912202709174
:1016D000230280912402909125020F9479B37E8396
:1016E0006D830F94033D83E00F94987FAB01BC01A1
:1016F0008EE69FE00F94B2B16091230E81E06827DF
:1017000082E79FE00F94A0B10F942F5D10925716BF
:10171000789420E030E040E85FE36091EB0F709157
:10172000EC0F8091ED0F9091EE0F0F9419B2698339
:101730007A838B839C83E090E70FF090E80F009111
:10174000E90F1091EA0F2091E30F3091E40F4091DF
:10175000E50F5091E60F6091DF0F7091E00F8091DF
:10176000E10F9091E20FEAE12E2EEDE03E2E3F9246
:101770002F92812C912CFEEBAF2EF2E4BF2EFE01B6
:1017800031966F010F94C52E0F94AB7F149A20E011
:1017900030E040E85FE36091EB0F7091EC0F8091D7
:1017A000ED0F9091EE0F0F9419B269837A838B83BA
:1017B0009C8367E074E02F813885621B730BA4E083
:1017C00076956795AA95E1F780E090E00F9432A9AD
:1017D00069877A878B879C872AE037ED43E25FE34E
:1017E0006091E70F7091E80F8091E90F9091EA0FF7
:1017F0000F941AB26B017C0120912F1030913010A0
:10180000409131105091321069857A858B859C8585
:101810000F9408B39B01AC01C701B6010F941AB233
:101820007B018C012091E30F3091E40F4091E50F93
:101830005091E60F6091DF0F7091E00F8091E10F02
:101840009091E20F3F922F92812C912CB0E2AB2E1F
:10185000B2E4BB2EFE0131966F010F94C52E0F949A
:10186000AB7F149A20E030E040E85FE36091EB0F3B
:101870007091EC0F8091ED0F9091EE0F0F9419B2D3
:1018800069837A838B839C832AE037ED43E25FE3AD
:101890006091E70F7091E80F8091E90F9091EA0F46
:1018A0000F941AB26B017C0120912F1030913010EF
:1018B000409131105091321069857A858B859C85D5
:1018C0000F9408B39B01AC01C701B6010F941AB283
:1018D0007B018C012091E30F3091E40F4091E50FE3
:1018E0005091E60F6091DF0F7091E00F8091E10F52
:1018F0009091E20F3F922F92FE0131966F010F946B
:10190000C52E0F94AB7F149AB301A20181E99FE029
:101910000F94B2B10F900F900F900F900F900F9007
:1019200005E71FE0712C83E0682E80916315882302
:1019300041F1872D662D0F94B8B625E18202F001A2
:10194000112433E09302E00DF11D1124EE0FFF1F6F
:10195000EE0FFF1FED59FA4E20E030E04AE754E465
:1019600061817281838194810F9426A420E030E00C
:1019700040E05FE30F941AB20F94AEB30F9479B3C3
:1019800002C060E070E0C8010F94BAB173940E5FBA
:101990001F4F49E07412C9CF6F81788583E79FE0BC
:1019A0000F94BAB14091DF0F5091E00F6091E10FB9
:1019B0007091E20F8DE99FE00F94B2B14091E30F77
:1019C0005091E40F6091E50F7091E60F81EA9FE07E
:1019D0000F94B2B14091E70F5091E80F6091E90F79
:1019E0007091EA0F8DE89FE00F94B2B1BE016B5F7A
:1019F0007F4F89E89FE00E944FC6E0911A0DF0E00A
:101A0000EE0FFF1FE05AFA4E60818CE89FE00F94C2
:101A1000A0B160911E0D8BE89FE00F94A0B1609182
:101A2000AF1988E89FE00F94A0B14091290250912E
:101A30002A0260912B0270912C0288EE9EE00F9496
:101A4000B2B160916202709163028EED9EE00F94DC
:101A5000BAB15989552329F061E085EA9FE00F94D6
:101A6000A0B10F94AB7F82E00E94F09E9F938F9372
:101A700080E290E29F938F930F949AA884E69FE070
:101A80000F948EB161E0680F84E69FE00F94A0B1DF
:101A90008FEF9EE00F949BB1BC016F5F7F4F8FEF84
:101AA0009EE00F94BAB10F944E86DC01CB012D85D8
:101AB0003E854F855889821B930BA40BB50BBF93B2
:101AC000AF939F938F9381E190E29F938F930F94B5
:101AD0009AA89DE088E10FB6F894A89580936000DD
:101AE0000FBE909360009FB7F894809102018460CC
:101AF000809302019FBF0FB6F894DEBF0FBECDBF2B
:101B0000FFCF85EA9FE00F948EB1882309F4A7C028
:101B1000179A10921B0D169A10921C0D149A64E1DC
:101B200082E00F94E89664E182E00F94D79683E414
:101B30000E94F09E3C010F94033D789467E074E0AE
:101B40006619770984E0769567958A95E1F780E0D4
:101B500090E00F9432A920912F10309130104091D5
:101B60003110509132100F9408B36B017C012AE0C0
:101B700037ED43E25FE36091E70F7091E80F8091EA
:101B8000E90F9091EA0F0F941AB29B01AC01C701C3
:101B9000B6010F941AB27B018C012091E30F3091B2
:101BA000E40F4091E50F5091E60F6091DF0F7091C7
:101BB000E00F8091E10F9091E20FEAE1FDE0FF93E9
:101BC000EF93812C912CE0E2AE2EE2E4BE2EFBEEF0
:101BD000CF2EFFE0DF2E0F94C52E0F94AB7F62E077
:101BE00085EA9FE00F94A0B1B30188ED9EE00F94C9
:101BF000BAB14091E70F5091E80F6091E90F7091F1
:101C0000EA0F8AED9EE00F94B2B184E69FE00F9454
